:1000000000800020BD010000A16C02006D6C0200A8
:100010006D6C02006D6C02006D6C02006D6C020074
:100020006D6C02006D6C02006D6C0200A16C020030
:10003000A16C02006D6C0200B18D0200B58D020052
:10004000A16C0200A16C0200A16C0200A16C020074
:10005000A16C0200A16C0200A16C0200A16C020064
:10006000A16C0200A16C0200A16C0200A16C020054
:10007000A16C0200A16C0200A16C0200A16C020044
:10008000A16C0200A16C0200A16C0200A16C020034
:10009000A16C0200A16C0200A16C0200A16C020024
:1000A0003D29020049290200A16C0200A16C020056
:1000B000A16C0200A16C0200A16C0200A16C020004
:1000C000A16C0200A16C0200A16C0200A16C0200F4
:1000D000A16C0200A16C0200A16C0200A16C0200E4
:1000E000A16C0200A16C0200A16C0200A16C0200D4
:1000F000A16C0200A16C0200A16C02008D7B0200C9
:10010000A16C0200A16C0200A16C0200A16C0200B3
:10011000A16C0200A16C0200A16C0200A16C0200A3
:10012000A16C0200A16C0200A16C0200A16C020093
:10013000A16C0200A16C0200A16C0200A16C020083
:10014000A16C0200A16C0200A16C0200A16C020073
:10015000998F0200AD8F0200C18F0200D58F02007F
:10016000A16C02003D7E0200A16C0200A16C0200A5
:10017000A16C0200A16C0200A16C0200A16C020043
:10018000A16C0200A16C0200A16C0200A16C020033
:10019000A16C0200A16C0200A16C0200A16C020023
:1001A000A16C0200A16C0200A16C0200A16C020013
:1001B000A16C0200A16C0200A16C0200564B4CF233
:1001C000205210B51A804DF628121A8000BF00BFC9
:1001D00026F06AFD514B4FF010621A60504A9A6047
:1001E000504ADA60504A136813F4807301BF4F49D4
:1001F0000B604FF4A85313604D4B4E491A7810070B
:1002000042BF1A7842F008021A704B4B2A221A7029
:100210004A4A4B4B8B4204D252F8040F43F8040B6A
:10022000F8E7484B484A0021934202D243F8041BA6
:10023000FAE7464A4648002350F8231042F82310B4
:1002400001336F2BF8D1434B434A802103F8011B44
:100250009342FBD1414B3D4A1A60414B8A221A70AE
:10026000A3F5805324225A70A0221A709A7991071C
:10027000FCD59A79D206FCD43A4A937903F00C0360
:10028000082B384BF9D103221A7140225A719A79FE
:100290009406FCD533498A79324B5006FBD5324A55
:1002A000324911600221516020221A709A7902F0BD
:1002B0000C020C2AFAD12E4B2E4A1A602E4B2F4AD2
:1002C0001A6000225A60072243F8042C2C4AC3F813
:1002D0000C2D62B627F022F9144B1B68DA0705D5FE
:1002E000284826F0DBFE284B284A1A60284B1B784A
:1002F0005B0609D5244C254B22689A4204D121483B
:1003000026F0CCFE002323602DF0FAF826F0D2FC74
:1003100029F0D1F9FEE700BF0E20054030800440EF
:10032000823F04000100002B10D0034014D0034092
:1003300002D00740188DFF1F00E0074074880300BB
:100340001C87FF1F188DFF1FBCD9FF1F0082FF1FD6
:100350000000000000E400E05FE400E008ED00E0E1
:100360000050064000400640448004400000030165
:1003700004800440C010050014E000E0FF76010096
:1003800000002020536753641CE00340A5C3945A27
:1003900000F00740FFFFFFFFFFFFFFFFFFFFFFFF32
:1003A000FFFFFFFFFFFFFFFFFFFFFFFFFFFFFFFF5D
:1003B000FFFFFFFFFFFFFFFFFFFFFFFFFFFFFFFF4D
:1003C000FFFFFFFFFFFFFFFFFFFFFFFFFFFFFFFF3D
:1003D000FFFFFFFFFFFFFFFFFFFFFFFFFFFFFFFF2D
:1003E000FFFFFFFFFFFFFFFFFFFFFFFFFFFFFFFF1D
:1003F000FFFFFFFFFFFFFFFFFFFFFFFFFFFFFFFF0D
:10040000FFFFFFFFFFFFFFFFFFFFFFFFDEF9FFFF23
:1004100010B5054C237833B9044B13B10448AFF33E
:1004200000800123237010BD188DFF1F0000000005
:1004300070880300084B10B51BB108490848AFF39A
:1004400000800848036803B910BD074B002BFBD0A0
:10045000BDE81040184700BF000000001C8DFF1FC2
:1004600070880300188DFF1F0000000070B505683C
:10047000044628460E4626F061FB864203D03146EC
:10048000284626F06FFB204670BD2DE9F0418046DE
:100490000E4614461AB3012A02D100230B701EE047
:1004A00026F04CFB01250746307097B1AC420ADDBF
:1004B00008EB050026F042FB0746192027F018F844
:1004C00077550135F1E7002D03DD3544002305F8AC
:1004D000013C192027F00CF80120BDE8F0812046EE
:1004E000BDE8F0812DE9F04112491C4600AF90466D
:1004F000054628F010FFE31D23F00703ADEB030DC5
:10050000224640466946FFF7C0FF661EE8466C4635
:10051000C8EB04039E4208DD14F8011B284628F0AE
:10052000EDFF192026F0E4FFF2E72846BD46BDE8BE
:10053000F08100BF8F110300F0B585B0002401AE3B
:100540001046234609220F463146019402948DF845
:100550000C4029F04DF830462DF08FF90130C5B22E
:10056000E3B29D420AD93B19315D00936846FFF71B
:100570007DFF192026F0BCFF0134F1E7284605B0C5
:10058000F0BD26F097BA70B5044608460D462DF02A
:1005900074F923680246294620465B68BDE870402E
:1005A000184726F087BA002070477047024A136840
:1005B00001331360704700BF98BAFF1F024A5368A7
:1005C00001335360704700BF98BAFF1F2C4B2D4A70
:1005D0001B7810B52C4C3BB12388C3F309035BB1E6
:1005E00013889BB243B10AE02388C3F30903BBB16C
:1005F00013889BB2A3B129E02449002312E021888B
:10060000128889B292B29202642392FBF3F391FBB7
:10061000F3F203FB121383B91C4B1A786AB911E089
:100620001A4901230B7013889BB223B1184B097828
:10063000187826F0B9FD00232380238801339BB26C
:10064000238010BD01221A70197813E023881288C4
:1006500099B292B29202642392FBF3F391FBF3F20C
:1006600003FB1213002BE8D1084A11780029E4D0CB
:1006700013701178064B187826F096FDDDE700BF61
:1006800020C4FF1FBAC5FF1FA0BAFF1FD78EFF1FD0
:1006900094BAFF1F10B5044628F05CFC204610BD3C
:1006A00010B5034B0360044621F094FA204610BDB8
:1006B0007022030010B50446FFF7F2FF2046142114
:1006C00029F005F8204610BD10B5034B0360044621
:1006D00021F080FA204610BDDC2E030010B5044640
:1006E000FFF7F2FF2046142128F0F1FF204610BD4D
:1006F00010B5034B0360044621F06CFA204610BD90
:10070000B42C030010B50446FFF7F2FF2046142175
:1007100028F0DDFF204610BD10B5034B03600446F2
:1007200021F058FA204610BD802A030010B5044677
:10073000FFF7F2FF2046142128F0C9FF204610BD24
:1007400026F010BA38B50C46054626F0F7F9844273
:1007500005D021462846BDE8384026F003BA38BD0A
:1007600038B50C46C1F307210546FFF7EBFF0A2019
:1007700026F0BEFE681CE1B2FFF7E4FF0A20BDE8E8
:10078000384026F0B5BE10B5029C521AE41AA242B7
:10079000A0EB0100C6BF04FB00000132604390FBE8
:1007A000F2F0184410BD10B5029C521AE41AA2428D
:1007B000A0EB0100C6BF04FB00000132604390FBC8
:1007C000F2F0184410BD10B50C4604220146204634
:1007D00026F0EAF9204610BD10B5C0F30721044603
:1007E0004FF4D170FFF7ACFF0A2026F081FEE1B292
:1007F00040F2A310FFF7A4FF0A20BDE8104026F046
:1008000077BEF8B50C460E1D0D46471A781926F02E
:1008100095F905F8010BB542F8D12046F8BD26F050
:100820008DB9FFFF10B50B4C2378042B0DD94FF475
:10083000CC70FFF7F4FF0322212888BFFF20064970
:1008400026F012FD054828F085FB2378013323703C
:1008500010BD00BF94C5FF1FA9540100388EFF1FB3
:1008600008B540F29710FFF7DAFF012126F0CAFC25
:1008700040F29710FFF7D3FF002126F095FCFA20F5
:1008800026F036FE40F29710FFF7C9FF002126F050
:10089000B9FC002008BD38B50546FFF7C0FF044687
:1008A000681CFFF7BCFF0146204628F0F1FC00B2AF
:1008B00038BD28F011BE28F013BE70B504460846B6
:1008C0000D462CF0DAFF23680246294620465B6875
:1008D000BDE87040184700230A2228F0DDBB28F04D
:1008E00016BC00230A2228F0D7BB9DF80010009107
:1008F00028F016BC38B50546FFF7DFFF044628464A
:1009000028F0A6FB204438BD38B50546FFF7E3FFC5
:100910000446284628F09CFB204438BD38B50546DF
:1009200028F0F5FB0446284628F092FB204438BD09
:10093000002A10B40BDB074B541E9C4207D830230F
:100940005A43013A232A02D910BC28F0BBBA00202E
:1009500010BC7047575555051FB50024B0F90C3031
:10096000B0F90A20B0F90810029403240194B0F9F8
:100970000E400094406824F053FB04B010BD0B8877
:1009800083834B88C3838B880384704730B502F11F
:100990001704013900F117030444A34204D011F8ED
:1009A000015F03F8015FF8E780F8242030BD0022E2
:1009B000FF238281438200F11402503022F8023F6B
:1009C0008242FBD17047FFFF10B5044621F02EF99B
:1009D000014B2360204610BD802A030010B5044659
:1009E00021F024F9014B2360204610BDDC2E0300CA
:1009F00010B5044621F01AF9014B2360204610BDC2
:100A0000B42C030010B5044621F010F9014B23600B
:100A1000204610BD7022030070B586B08DE80F002F
:100A2000194B9DF828601A78052A1D4607D069469B
:100A3000164821F01DFB011C18BF012100E0002118
:100A40002B78032B1ED1EEB11148FFF748FF009A17
:100A500010490F4828F013FB0DF107040DF10F05A5
:100A600014F8012F0C490A4828F009FBAC42F7D1D1
:100A70000A4B9DF805201B680593059B084904480F
:100A800028F0FDFA06B070BD8CBAFF1F34C5FF1FF9
:100A9000848AFF1FC0100300C610030000D8FF1F88
:100AA000CC1003002DE9F74F40F21910FFF7B7FE05
:100AB000092811D1B84BB94D01221A7108225A7177
:100AC000B74A1A600022AC5CB34998180132082A70
:100AD0000472F8D10023BEE00A2859D1B14CB24EBD
:100AE000082363714FF4DE63236033781B0103F046
:100AF000100323723378DB0003F01003A372337802
:100B00009B0003F01003237333785B00002501275B
:100B100003F0100325716572E5726573E573A373C5
:100B2000009794E80F00FFF777FFA04A657240F244
:100B3000F16323601378E5729B0003F03C0323729A
:100B4000137865731B099B00A3722573E573A57366
:100B5000009794E80F00FFF75FFF40F2F263236015
:100B60003378657203F0100323723378E572FB402B
:100B700003F01003A372337865739B0803F010032E
:100B800023733378E573DB091B01A37300973AE005
:100B90000B283BD1834C864F864D002323710823BD
:100BA00063714FF4C26323603B78A82606FB0353AE
:100BB000D3E90E012BF046FF80B2031223727B783B
:100BC000607206FB0353D3E90E012BF03BFF80B2AA
:100BD0000312A372BB78E07206FB0353D3E90E0144
:100BE0002BF030FF80B203122373FB78607306FB97
:100BF0000355D5E90E012BF025FF80B20312A37334
:100C00000123E073009394E80F00F0E20C2825D153
:100C10006449654800230B7108234B714FF4E0636E
:100C20000B60A5230B7203780478027812F0010F91
:100C3000027802F0010203F0040342F0040204F01F
:100C4000020442EA83020CBF0225002542EA840323
:100C50002B434B72012300930FC9C8E2082840F0D0
:100C6000FC80504C524F534E6071002323713B78EF
:100C7000A82202FB036393F89030FBB1DFF83881C0
:100C8000D8F804504FF48E70FFF7C9FDADB20223BF
:100C90004246D9B288420AD958F82310A94288BFDF
:100CA00052F8235003F1010388BFADB2F1E741F2DE
:100CB00088335D43AB12AD14257263727B78A82232
:100CC00002FB036393F89030FBB1DFF8EC80D8F8B7
:100CD00098514FF48E70FFF7A2FDADB2022341464A
:100CE000DAB290420AD903F16502013358F822E0E2
:100CF000AE4584BF51F82250ADB2F1E741F28833DE
:100D00005D43AB12AD14A572E372BB78A82202FB5F
:100D1000036393F89030FBB1DFF89C80D8F82C5334
:100D20004FF48E70FFF77BFDADB202234146DAB27D
:100D300090420AD903F1CA02013358F822E0AE45C5
:100D400084BF51F82250ADB2F1E741F288335D43E0
:100D5000AB12AD1425736373FB78A82202FB036604
:100D600096F890308BB3144ED6F8C0544FF48E7072
:100D7000FFF755FDADB202233146DAB290421DD9DC
:100D800003F22F12013356F82270AF4284BF51F89C
:100D90002250ADB2F1E700BF68C5FF1F83C5FF1F3A
:100DA00001C0CC1CA8C5FF1F89BAFF1FD58EFF1F2D
:100DB0008EBAFF1F8890FF1FC0C9FF1F41F2883302
:100DC0005D43AB12AD14A573E3734FF4C8632360A6
:100DD00001230093A84D94E80F00FFF71DFE05F1D5
:100DE00008062B46002203F8012F9E42FBD1A34F99
:100DF000A3483A7890F800E040F2416302F00F0215
:100E0000236041F28831531C91FBF3F20EF00F0383
:100E100013FB02F39BB263721B1223723B780278BE
:100E20001B09013391FBF3F1130913FB01F39BB28F
:100E3000E3721B12A3720123009394E80F00FFF7E3
:100E4000EBFD002305F8013FB542FBD140F24263C0
:100E500023608C4B1B7823739DE0012840F0A98010
:100E6000894C8A4908226271894A002323712372BE
:100E70006372A372E372237363731378A82000FB79
:100E80000313884693F890709146EFB1814E7568D0
:100E90004FF48E70FFF7C3FCADB202233246D9B2D5
:100EA00088420AD956F82310A94288BF52F8235025
:100EB00003F1010388BFADB2F1E741F288335D432E
:100EC000AB12AD142572637299F80130A82202FBAF
:100ED000038898F890605EB3DFF8B881D8F898512D
:100EE0004FF48E70FFF79BFCADB202234146DAB29D
:100EF00090420AD903F16502013358F822E0AE4569
:100F000084BF51F82250ADB2F1E741F288335D431E
:100F1000AB12AD14A572E3725FB95E4ED6F898516C
:100F20004FF48E70FFF77BFCADB2022331461CE01C
:100F30005FB3584F7D684FF48E70FFF770FCADB211
:100F400002233A46D9B288420AD957F82310A94257
:100F500088BF52F8235003F1010388BFADB2F1E717
:100F6000AD102573002ED8D10FE0DAB290420AD925
:100F700003F16502013356F82270AF4284BF51F885
:100F80002250ADB2F1E7AD10657340F266632360A5
:100F90003C4B1B78A373404D2B78E37301230093E4
:100FA00094E80F00FFF738FD2B780133DBB22B708C
:100FB0001FE102282ED1314F314E334B397835782D
:100FC000082201F00F015A7140F26C7241F2883030
:100FD0001A604A1C90FBF2F105F00F0212FB01F2BD
:100FE00092B211129A72274A59721278DA723A78CA
:100FF00031781209013290FBF2F00A0912FB00F27B
:1010000092B2002411121C711C7219735A739C73D2
:10101000DC732EE003280ED11B4B0821597140F2DE
:1010200002611960FF2119721649002208781A71AD
:101030005A72987217E0052830D1134B0821597164
:1010400040F2F97119600F49087800F00100187238
:1010500008780978C1F380010022C0F3400099723A
:1010600007491A7158720978D9721A735A739A73A8
:10107000DA730122B9E000BFAFC5FF1FD68EFF1F94
:10108000D58EFF1F89BAFF1FA8C5FF1F8890FF1FBD
:101090008EBAFF1FC0C9FF1FD48EFF1F062840F065
:1010A0009A80554C554FDFF86881DFF868A1082316
:1010B00063714FF4C8632360514B1A7802F0010248
:1010C00022721A78C2F3400262721A78C2F3800266
:1010D000A2721A78C2F3C002E2721A78C2F3001246
:1010E00022731A78C2F3401262731A781B78DB09F4
:1010F000E373C2F38012012300262671A2730093CA
:1011000094E80F00FFF788FC40F241632360254616
:101110004FF0A8094FF0650B16F8083009FB037370
:1011200093F89030E3B14FF48E70FFF778FB002115
:10113000002200230BFB06FC01315FFA81FE7045A3
:1011400008D90CEB010E5AF82EE012EB0E0243F117
:101150000003F1E7013892FBF0F21312237262727E
:101160000136042E04F10204D6D10123009395E840
:101170000F00FFF751FC40F242632B60214B00212E
:1011800003F1080203F8011F9342FBD11E4E1F4CCE
:101190003278207802F00F02531C41F2883191FB23
:1011A000F3F200F00F0313FB02F39BB22B721B123E
:1011B0006B72337822781B09013391FBF3F1130929
:1011C00013FB01F39BB2AB721B12EB720123009372
:1011D00095E80F000BE007280BD1074B00221A718E
:1011E0004FF4407101225A71196000920FCBFFF742
:1011F00013FC03B0BDE8F08FA8C5FF1F8890FF1F48
:1012000089BAFF1FAFC5FF1FD68EFF1FD58EFF1FE8
:101210008EBAFF1FC0C9FF1F2DE9F347C04CC14F55
:10122000C14E3B78082161714FF4D0712160BF49F4
:101230000878884601284FF0400161720BBFE92110
:10124000B321A172A1720CBF0321102103F00F037F
:101250000022E1721033FE21E373227122722173A6
:101260006173A2730023009394E80F00FFF7D4FB8F
:101270004FF4207301202360FFF7D1FAFF280546C1
:1012800000F06A813378012B40F06681A84AA823D8
:1012900003FB0025D5E90E010022A64B2BF0FAF83E
:1012A0002BF0A8FB00B2C5B2C0F307200023FE223A
:1012B000012123726272A572E07223736273A173BB
:1012C000E273009394E80F00FFF7A6FB4FF422733C
:1012D00023603378012B0ED19749984B0022D1E936
:1012E00000012AF025FF0022954B2BF0FDF92BF091
:1012F000A9FBC0B200E0C72092490A78894602F0F3
:10130000FF031AB90D222272607210E00B78012BD4
:1013100001D1702308E00B78022B01D18F2303E069
:101320000B78032B0CD1E923237260720023A37284
:10133000E37223734D236373FF23A373BF23E3730C
:10134000002694E80F000096FFF766FB0122A272C8
:101350007D4AE6724FF0FE0A4FF42873107823603E
:10136000642280233146CDF800A063722673667331
:10137000A673E673FFF707FA207294E80F00009651
:10138000FFF74AFB4FF46073236058236372FD2319
:10139000E37207232373F023267284F80AA0637391
:1013A000A67384F80FA094E80F000096FFF734FBB3
:1013B00099F800105A4D634A4FF49063236001F08E
:1013C000FF0351B996222A722C22AB72EB722B7357
:1013D0006B73AB736A72BA2328E01378012B0AD1BE
:1013E000E8232B722C236B72AE72EE722E736E7327
:1013F000AE73C4231AE01378022B0AD161232B7237
:101400002C236B72AE72EE722E736E73AE734D231D
:101410000CE01378032B0AD11B232B722C236B7245
:10142000AE72EE722E736E73AE733723EB730023BE
:10143000009394E80F00FFF7EFFA4FF491632360F5
:101440003B78424A364D03F00F030F2B14BFDBB23B
:101450000E237821D25CE1720B322272FE2262727C
:10146000A27222731B0100226273A273E3730092C3
:1014700094E80F00FFF7D0FA4FF49463236098F8D4
:101480000030012B4FF0B2032B7205D110226A728B
:10149000AB72EA722B7305E011226A72EA72AB72C8
:1014A0002B7310226A73AB73EA73002594E80F0064
:1014B0000095FFF7B1FA4FF4B1632360082323725C
:1014C00078236572A372E57225736573A573E5735E
:1014D00094E80F000095FFF79FFA3B780133DBB2E9
:1014E0003B703B7803F0FF020BB9194B1A70194A95
:1014F00013780133DBB213701378032B07D999F8F3
:1015000000300133DBB289F800300023137099F802
:101510000030032B3AD90B4B00221A7036E000BF83
:1015200068C5FF1F28C5FF1F8ABAFF1F7990FF1FDC
:101530008890FF1F000010406093FF1F000048408C
:101540000000E83F348EFF1FB8C4FF1F26220300AF
:10155000DA8EFF1F358EFF1F3378022B13D00D4913
:10156000A82303FB051100220B4BD1E90E012BF040
:1015700003FA18B1FF2D04D0002005E06020FF25FC
:1015800094E6602092E6612005468FE602B0BDE851
:10159000F08700BF8890FF1F00407F4008B54FF4E0
:1015A000CC70FFF73CF9002125F02CFE4FF4CC70F5
:1015B000FFF735F9012125F0F7FD0A20BDE80840C5
:1015C00025F096BF0B79037130B58B6883600B46AD
:1015D00000F11A0413F80C2F027300F10D0213F836
:1015E000015F02F8015B9442F9D1CB69C36130BD60
:1015F00010B5042894BF044603242146084821F06E
:1016000087FA032C074A084B15BFF0214FF4A0714D
:101610001180118014BF4FF4A072F0221A8010BD07
:1016200008C6FF1F0488FF1F3E88FF1F2DE9F041F9
:10163000044690B003200F46FFF7DAFF012C25D1B6
:10164000974B98481B6804930499974E974DFFF762
:1016500048F997499348FEF796FF002332785C1CBF
:10166000DBB29A420FD9A82202FB03530222009256
:10167000D3E90E238B48FFF738F98D498948FEF7E7
:1016800082FF2346EAE78B498648B4E0022C40F00B
:10169000B480894B1B78FF2B40F0AF80804E874988
:1016A00033680293029B0A689A1A854B18784EF6A3
:1016B000602343439A4202D9FF2F00F0A580002403
:1016C000804B04AA03F1080C154618685968964621
:1016D000AEE80300083363457246F6D1186899886E
:1016E000DFF804829B79CEF80000AEF804108EF883
:1016F000063098F80030FF2F18BF3B4630338DF886
:101700001930BCB170496748FEF73DFF98F80010EA
:101710006448FFF7E0F86D496248FEF734FF294658
:101720006B481FF015F908B16A4900E06A495D4845
:10173000FFF7E0F869481EF07AFF98B92946644837
:101740001FF0FAF8132300282A46614908A808BFA9
:1017500001241FF0ADF808A96048FFF733FF08A87F
:101760001EF022FFFCB15E495C484F4DFEF70BFFB7
:1017700000242B78E1B2994204F101040FD2002237
:1017800008A818F021FC08A9544827F041FC08A833
:1017900027F081FD46495148FEF7F5FEE9E7454946
:1017A0004E48FFF7A7F84D481EF041FF28B33368B5
:1017B0000893089949483C4E3C4DFFF792F83C4944
:1017C0004648FEF7E0FE002332785C1CDBB29A420A
:1017D0000FD9A82202FB035302220092D3E90E2361
:1017E0003E48FFF782F832493C48FEF7CCFE2346DC
:1017F000EAE730493948FFF77DF83A4B1878FFF7A8
:10180000F7FE10B0BDE8F08133680393364D039BBB
:101810000B602B780133DBB2092B00D900232B702E
:101820002978DFF8D8804FF4D070FEF78BFF2F486F
:1018300021F08AFA09224FF6E0738DE80C0032217C
:101840001F230122294823F093FB0121274821F07F
:1018500006FA0124002302223621244888F8004099
:1018600022F0D6FC0021214821F0FFF920491F4831
:10187000FEF789FE29781D48FFF72DF81D4A1E49FD
:10188000B2F90020B1F900101848002322F0C0FC82
:101890000021164821F0E9F9002388F800300FE70D
:1018A00000D8FF1F848AFF1F22C4FF1F8890FF1FDC
:1018B000401103008F1103000C88FF1F2CC5FF1F70
:1018C00060C5FF1F02110300DF100300F3100300C7
:1018D000E0D4FF1FF0130300511D0300F0C4FF1FED
:1018E000F71003002888FF1F4188FF1F08C6FF1F4D
:1018F000FB1403003E88FF1F0488FF1FBCC5FF1FA9
:101900002DE9F04F814689B06848694D694F884696
:10191000002121F0AAF90121644821F0A0F9032057
:10192000FFF766FE0B2444F2082301930094BC23C6
:10193000012246215D4823F01BFB46F22C33019324
:1019400000940F2301223721584823F011FB002374
:1019500002223B21554822F05BFC57495348FEF7D1
:1019600012FE2C782CB1FF2C08BF3C78013CA4B2AD
:1019700000E0FF24514A0392702606FB09264644E4
:1019800046F22C3A337E4948A34214BF53464FF4E3
:10199000FC634FF00B0B0193012233234B21CDF855
:1019A00000B023F0E5FA002302224D213F4822F047
:1019B0002FFC3B780822E1B204A818F005FB04A92B
:1019C0003A4827F025FB04A827F065FC327E2B78E7
:1019D0003648CDF800B09A4214BF53464FF4FC632A
:1019E000019301223323832123F0C2FA0023022230
:1019F00085212E4822F00CFC3B782978082204A887
:101A000018F0E2FA04A9294827F002FB04A827F0FD
:101A100042FC2C78FF2C06D0264B1B78013B9C42C5
:101A200003D0013402E0002400E0FF24039A1F48A1
:101A3000702303FB0929C84446F22C3698F8183065
:101A40000B25A34214BF33464FF4FC63019300956A
:101A500033230122BB2123F08BFA00230222BD2174
:101A6000124822F0D5FB3B780822E1B204A818F016
:101A7000ABFA04A90D4827F0CBFA04A827F00BFC19
:101A80008DE860000F230122F321084823F070FA4B
:101A900000230222F721054822F0BAFB0849034837
:101AA000FEF771FD09B0BDE8F08F00BF08C6FF1F4B
:101AB00094C5FF1F22C4FF1F11110300B0BCFF1FFC
:101AC00013110300013808B5052810D8DFE800F02D
:101AD000050305090709522104E0062102E0D2218D
:101AE00000E0C6210648BDE8084024F065BCD221CC
:101AF000034824F061FC034B00221A7008BD00BFAC
:101B000010C5FF1FE88EFF1F10B5074A0023702184
:101B100001FB0324D8B294F858401CB10133112BB7
:101B2000F6D1FF2010BD00BFB0BCFF1F38B5074D78
:101B30000024281990F858301BB1FF2200211EF014
:101B400011F97034B4F5EE6FF3D138BDB0BCFF1F9E
:101B500010B58CB01B49684627F0DDFB5323009A73
:101B6000194904A81EF0A4FE04A91848FFF72AFD8D
:101B700004A81EF019FD00242046FEF750FE013493
:101B800002461349114827F07AFAB4F5BE7FF3D123
:101B900010490E48FEF7F7FC4FF4C8742046FEF7D4
:101BA0003EFE013402460A49084827F068FAB4F5B7
:101BB000167FF3D105481EF02EFD684627F06BFB1B
:101BC0000CB010BD15110300E0D4FF1FF0C4FF1FBF
:101BD000C6100300261103000D4B03600B7903713F
:101BE0008B6883600B7B037303460A4A30B543F866
:101BF0000D2B01F1190401F10D0252F8045B43F8B9
:101C0000045BA242F9D112781A70CB69C36130BD6E
:101C100074820300587303001B4B73B50122044602
:101C2000014600201A7018F0A7F910B1174B1B7865
:101C3000DBB9174B1B782BB32146012018F09CF918
:101C400000B32146022018F097F9D8B901212046A7
:101C500018F07EF90F4A1378013313700E4B1B688E
:101C600001930E4B019A1A600CE00D4B14201D6875
:101C700027F029FD0646FEF7A7FE3146284620F04C
:101C800071F8D6E702B070BD8BBAFF1F3D88FF1F09
:101C900029C5FF1F5AC7FF1F00D8FF1FD0D4FF1F41
:101CA0004CD7FF1F2DE9F347384EA82202FB0067EF
:101CB0008246D7E90E4500293ED097F89130FF2B98
:101CC00008D002FB0361D1E90E01D7E926232AF0EF
:101CD00067FED0B1D7E91689204642464B462946D1
:101CE0002AF05EFE30B9D7E91223204629462AF0B1
:101CF0004DFE50B100220023404649462AF032FEF4
:101D000018B95046FFF788FF16E0A82303FB0A63C3
:101D100093F8A12082B193F8A2206AB11C4A1D4811
:101D2000126801921C4A019912680078891A64228B
:101D300010FB02F2914222D8A82707FB0A67D7E9D5
:101D40001423204629462AF035FE10B1C7E9144570
:101D500019E0D7E91089204642464B4629462AF029
:101D60000BFE30B900220023404649462AF0FAFD16
:101D700048B1A82303FB0A66C6E9104503E0002228
:101D800083F8A220D8E702B0BDE8F0878890FF1F53
:101D900000D8FF1F29C5FF1FD0D4FF1F73B51446FD
:101DA00003EB430203EB8203CA1805B200230C20A5
:101DB0008DE809000E46052312B229460B4823F090
:101DC000D7F8FF2C0FD004EB440204EB82020B2166
:101DD0004FF6E07332448DE80A0012B2052329461B
:101DE000024823F0C5F802B070BD00BF08C6FF1F4F
:101DF000022938B50346084605D1FF222C21FFF7FA
:101E0000CDFF002038BD1D4A1D491278A82404FBCF
:101E1000021494F86840012C14BF0B240D24013CDB
:101E200003B918B3A34203DB01280CD100241EE040
:101E300020B95C1EE4B2042C0AD114E0012804D1BC
:101E40005C1CE4B202E00028F3D01C46042C0CD049
:101E5000072C0CD1A82505FB0212516840F6FF7231
:101E6000914204D008B9013C00E00134E4B22246BA
:101E70002C210220FFF792FF204638BD94C5FF1F9A
:101E80008890FF1F2DE9F0430B88FF2B89B0054692
:101E90000C4617460CD14888092809D8864B8A88F1
:101EA000C0B21870854B1A70FFF7A2FB002000E14A
:101EB0002389834E092B0ED1824A142303FB052369
:101EC00001221A7440F2AB10FEF7A9FC7E4B187089
:101ED0001B78A38153E00B2B3BD16389092B04D1E1
:101EE0007A4B7B4A1B78DBB205E00A2B0AD1774B91
:101EF000784A1B78DBB21278934211D00023A38179
:101F0000E28113E00B2B05D1704B1B78FF2B64D0C3
:101F1000002363E00C2B09D16C4B1B78FE2BF6E7FA
:101F20000122A2816C4A9BB21380E3816B4B1B7828
:101F3000FF2B10D0654A117864290CD81078684AB4
:101F40004FF0A80808FB03282AF02EFAC8E90E0172
:101F500001E0052B13D13A78002A40F09F807023CE
:101F60006B43F2544FF0700808FB05684FF000090E
:101F700088F8089038462BF080FC08F80090702311
:101F800003FB05666389ADF818300125A389ADF818
:101F90001A3006A9E38986F858503046ADF81C304F
:101FA000FEF7EDFC0020A388628821880290207A49
:101FB0000190E088009030461DF010FF2389112B1E
:101FC0000ED10320FEF72BFC464B1B7883425BD9D6
:101FD00008A92A4601F80C0D51E00123A381A5E7C9
:101FE0000B2B2FD163890E2B14D13F4F3B7803F07D
:101FF000F002A37B13433B70397840F2C510FEF723
:10200000A1FB3B7803F00F033384384B1B7803F0BC
:102010000F0315E00F2B37D1334FE2893B7803F0E4
:102020000F0343EA0213DBB23B70397840F2C5106C
:10203000FEF788FB3B781B0933842C4B1B781B096C
:1020400073841FE005AF7BB9294A106805900E34F0
:1020500034F8021FFF29DAB204D0F9540133042BFB
:10206000F6D11A46394614E0072B0DD12846FEF763
:10207000D6FBFF2808D08DF814002A463946304692
:10208000FEF784FC284614E008A9238A01F80C3DD9
:1020900001223046FEF77AFC01200AE038462BF098
:1020A000ECFB02467020394600FB05602BF002FC79
:1020B00058E709B0BDE8F0832888FF1F0F88FF1F8D
:1020C000B0BCFF1FA4BAFF1F7990FF1F95BAFF1F76
:1020D00088BAFF1F96C9FF1FBAC5FF1F0A88FF1FD6
:1020E0008890FF1F22C4FF1FD68EFF1FD58EFF1FB3
:1020F000580E03002DE9F04F0246BDB072B65323CF
:1021000004A8A1491EF0D4FB04A81EF090FA30B137
:102110009E4FDFF8ACA24FF00008B946CEE062B6A1
:102120009B499C48FEF72FFA27E1A826DFF874B2F6
:1021300099496643BD19002358468BF800302BF0AF
:1021400094FB2B7A062B06F1100640F0BF803E442C
:102150000636EB7A01966A7D0092904922460CA8D9
:102160002BF038FB0CA958462BF058FBA82303FB97
:1021700004948B4994F868200CA82BF02BFB0CA935
:1021800088482BF04BFBD4E91C012AF07BFC0CABFC
:102190000822012124F0FEFD0CA982482BF03EFB11
:1021A000814980482BF03AFBD4E91E012AF06AFCF1
:1021B0000CAB0822012124F0EDFD0CA979482BF08D
:1021C0002DFB794977482BF029FBD4E920012AF02F
:1021D00059FC0CAB0822012124F0DCFD0CA971484C
:1021E0002BF01CFB70496F482BF018FBD4E922013F
:1021F0002AF048FC0CAB0822012124F0CBFD0CA9ED
:1022000068482BF00BFB684966482BF007FB94F8F5
:10221000902066490CA82BF0DDFA0CA961482BF040
:10222000FDFAD4E912012AF02DFC0CAB02220121A7
:1022300024F0B0FD0CA95B482BF0F0FA5A4959483C
:102240002BF0ECFAD4E916012AF01CFC0CAB0222AC
:10225000012124F09FFD0CA952482BF0DFFA94F8DD
:1022600091204F490CA82BF0B5FA0CA94D482BF042
:10227000D5FAD4E926012AF005FC0CAB0222012193
:1022800024F088FD0CA947482BF0C8FA94F8A31055
:1022900094F8A13094F8A02000910CA844492BF0A8
:1022A00099FA0CA93F482BF0B9FA3E4904A8FEF769
:1022B0006AF904A81EF011F908F101089AF8003033
:1022C0005FFA88F4A3423FF630AF4FE06A683949BD
:1022D0000CA82BF07FFA0CA958462BF09FFA297B0B
:1022E0006B7A2A7A0291E97A0191A97A00910CA875
:1022F00031492BF06FFA0CA958462BF08FFA2A6956
:102300002C490CA82BF066FA0CA958462BF086FA3B
:102310006A7D26490CA82BF05DFA0CA958462BF0D3
:102320007DFABA19063225490CA82BF053FA0CA9EC
:1023300058462BF073FAD5E90A012AF0A3FB0CAB3F
:102340000822012124F026FD0CA958462BF066FA3C
:10235000154958462BF062FAD5E90C012AF092FB98
:102360000CAB0522012124F015FDFBE604A81EF0AC
:10237000B4F804A81EF04FF962B604A81EF014F9D0
:102380003DB0BDE8F08F00BFE0D4FF1F8890FF1F75
:1023900028110300848AFF1F3F110300421103002C
:1023A0007F11030097C6FF1F401103008011030037
:1023B0008411030061110300681103007811030008
:1023C00022C4FF1FF0B5334B1C7891B007460E4670
:1023D000002C5BD008230A222F496846FEF782F8BA
:1023E0000622694604A827F04DF92C4908A826F0D2
:1023F00092FF08A904A827F022F9054608A826F0AC
:102400004AFF04A826F047FF65B906232A46694615
:1024100008A827F017F908A9684626F0F1FF08A8D0
:1024200026F039FF1E4904A826F075FF694604A866
:10243000FEF73FFA1B4904A8FEF73DFA049D1A492E
:1024400001232A4608A81EF033FA9FB11EB117488F
:10245000FFF750FE0AE008A81EF0CAF830B108A83D
:102460001EF04FF8C0B226F0F9FBF4E708A81EF002
:10247000D2F802E02846FFF73DFE08A81EF094F8C7
:1024800004A826F008FF684626F005FF204611B094
:10249000F0BD00BFDBD4FF1F30C5FF1FA91603002E
:1024A0009011030096110300E0D4FF1F9B1103005D
:1024B0002DE9F0438DB00E461746984608AC544DB2
:1024C0000C2800F28280DFE800F0071B232B333B4F
:1024D000434B535B636B73004E49204626F01BFF52
:1024E00046F22C33029314202823009300FB06505D
:1024F00001943C234246394617F00AF8204682E010
:102500000DF110094349484626F005FF424956E0BF
:102510000DF110093F49484626F0FDFE3F494EE0C7
:102520000DF110093B49484626F0F5FE3C4946E0CE
:102530000DF110093749484626F0EDFE39493EE0D5
:102540000DF110093349484626F0E5FE364936E0DC
:102550000DF110092F49484626F0DDFE33492EE0E3
:102560000DF110092B49484626F0D5FE304926E0EA
:102570000DF110092749484626F0CDFE2D491EE0F1
:102580000DF110092349484626F0C5FE2A4916E0F8
:102590000DF110091F49484626F0BDFE27490EE0FF
:1025A0000DF110091B49484626F0B5FE244906E006
:1025B0000DF110091749484626F0ADFE2149204685
:1025C00026F0A9FE4FF4FC630BE00DF11009114950
:1025D000484626F0A0FE1C49204626F09CFE4FF6F9
:1025E000E073039314202823009342463C2339468A
:1025F00000FB06500294CDF8049017F02EF8204608
:1026000026F049FE484626F046FE0DB0BDE8F083B0
:10261000A4BAFF1FAA110300B4110300BA110300EA
:10262000C2110300CA110300D5110300D911030020
:10263000E1110300EA110300F0110300F811030097
:10264000FE110300061203000E12030038B50D46FA
:102650000B49044626F05FFE0DB90A490AE0092D30
:1026600001D1094906E00A2D01D1084902E0072DF0
:1026700003D10749204626F0CBFE204638BD00BFD7
:10268000161203001A1203001E1203002212030086
:1026900026120300F7B5002A46F22C360C4618BF66
:1026A0004FF4FC668A1C0623411C054600930196E4
:1026B000032312B209B2134822F05AFC6B1D04F135
:1026C00008011BB2621C09B200910196194612B2B0
:1026D0000C4820F057FD27B2AB1D09341BB224B2C1
:1026E0003A4619468DE85000064820F04BFDEB1D98
:1026F0001BB28DE850003A461946024820F042FDD0
:1027000003B0F0BD08C6FF1F2DE9F34146F22C339C
:102710000D4604464FF6E071002A0CBF1A460A46E1
:10272000671C09236E1C073424B236B24FF0000830
:10273000019200932AB201B23FB21048073522F04D
:1027400017FC2DB22346324639468DE840010B482E
:1027500020F018FD2346324621468DE82001074827
:1027600020F010FD8DE820013B463246214603480B
:1027700020F008FD02B0BDE8F08100BF08C6FF1FD1
:10278000F0B5032087B0FEF733FF00214C484D4ED3
:1027900020F06BFA01214A4820F061FA484820F005
:1027A000D3FA00240C238DE8180022460F2321467B
:1027B000434822F0DDFB3378032B4BD140F2AD10C0
:1027C000FEF72DF8002845D03F4F3D886D083E3D6F
:1027D000EDB2E30229199BB20134009300220C23CD
:1027E000C9B23748A4B222F0C7FC202CF1D13988F5
:1027F00049080C204FF478431E398DE80900002267
:102800003C2309B22E4822F0B3FB3C8864083D34D7
:10281000E4B20025EB02611B9BB2009300220C2363
:10282000C9B22748013522F0A7FC202DF2D13C88FF
:1028300026496408053C02A826F06DFDA4B20523D4
:102840000093234802AB0222214617F023FF02A87F
:1028500026F021FD1F4C3078FEF7CAFE23780B2BA3
:102860002CD01D4B1A78003218BF012201211420F0
:10287000FFF74AFF194B01211A782320FFF70AFFBF
:102880000A2246F22C338DE80C00012211460D235A
:102890000B4822F06DFB002302220521084821F09D
:1028A000B7FC2378092B05D90222002311460448DE
:1028B00021F0AEFC21780248FEF70DF807B0F0BD1C
:1028C00008C6FF1F2888FF1F0488FF1F2E12030061
:1028D000B0BCFF1F0688FF1F29C5FF1F3D88FF1FD3
:1028E00007B5002A0CBF4FF478434FF4FC63019303
:1028F000072300930AB2042301B2034822F038FBF5
:1029000003B05DF804FB00BF08C6FF1F012808B52F
:1029100003D0022803D1044902E0044900E004493D
:102920000448FDF730FE08BD4112030039120300D0
:102930004812030008C6FF1F2DE9F84306460F465C
:10294000DDE908019046994629F0F0FB00220023BA
:1029500004460D462AF006F8E8B942464B46304692
:10296000394629F0E3FBDDE90A2306460F46DDE997
:102970000C0129F0DBFB02460B463046394629F0B4
:1029800089FD22462B4629F0AFFEDDE90A2329F016
:10299000CFFBBDE8F883DDE90A01BDE8F883FFFF5E
:1029A0002F4B37B501221A7000242E4B05462146C5
:1029B0002D481C7021F0B0FCFFF7E2FE012D07D17D
:1029C0002A4B224623F814200134112CFAD11BE0A3
:1029D000022D19D1264B2448B3F900304FF6FF726F
:1029E00001920C220092214622F0C2FA23460F22C5
:1029F000DC211D4821F00CFC21461B4820F035F954
:102A00001C491948FDF7BFFD4FF6FF71164820F02D
:102A10002CF9194B1B78042B1FD1134820F094F983
:102A20000321114820F01BF9002314220A210E482B
:102A300021F0EEFB4FF6FF710B4820F016F90F491D
:102A40000948FDF7A0FD0A21074800233C2221F098
:102A5000DFFB0B490448FDF796FD03B030BD00BF16
:102A60003C88FF1F96BAFF1F08C6FF1F26C4FF1F22
:102A70000488FF1F501203008CBAFF1F5512030079
:102A80006012030073B504B20DB20023164621464E
:102A90002A460E4821F0BCFB0D4B1B7803F0FF02C9
:102AA00093B90A232146019200932A461E23074820
:102AB00022F05EFA074B05481A783241D30754BF1B
:102AC00005490649FDF75FFD02B070BD08C6FF1F4E
:102AD000BCC5FF1FE8C4FF1F761203007912030074
:102AE0002DE9F34107B20FFA81F800231446394665
:102AF00042461A4821F08CFB194B1B785BBB194AE4
:102B0000194D115D2B5D994204D0631CD25CEB5CC6
:102B10009A4202D1154B1B78EBB100260A238DE8AF
:102B200048004246394628230C4822F021FA295D04
:102B30000A483346102226F0AFFA01340C49074800
:102B4000FDF721FD295D05483346102202B0BDE89E
:102B5000F04126F0A1BA02B0BDE8F08108C6FF1F1F
:102B6000BCC5FF1F75C7FF1FE8C4FF1F3C88FF1FC0
:102B7000A91603002DE9F04F504B514E00271F704E
:102B80009846504B8DB005460C46FAB2052A19D826
:102B9000DFE802F0030818180D123178C80711D5C4
:102BA00001210DE0317889070CD5022108E0317848
:102BB000C80607D5032103E03178890602D5042130
:102BC00088F800101978DFF8FC90002940F0708137
:102BD0003D48317890F800E0DFF8E4A08EEA01018A
:102BE000394111F0010F834640F0378137490978A8
:102BF000002940F03281013704F10A02072F92B216
:102C000001D01446C1E799F8003003F0FF08002B0B
:102C100040F04E8105F11E073FB216B243463246E0
:102C200039462B4821F0F4FA9AF800301B0607D5F4
:102C3000264B1B7803F0FF02002B40F015819046D5
:102C400099F8002002F0FF03002A40F031812FB2F2
:102C50001F483246394621F0DBFA9AF80100B8F1F4
:102C6000000F0CD02AF018F81A492AF069F81A490E
:102C700029F05CFF29F0BAFB8046894634E0C0EBBE
:102C8000C0006523A0F56070584340F2EB1390FB41
:102C9000F3F029F099FB002200238046894629F0B1
:102CA0006BFEE8B900220D4B4046494629F082FEF2
:102CB000D0B14FF00008DFF8249015E08CC7FF1F5B
:102CC000E8C4FF1FBCC5FF1F75C7FF1F3C88FF1F5F
:102CD00008C6FF1F96434B3F9643CB420000594026
:102CE0004FF000084FF000099AF801209BF80130DE
:102CF0009A4240F0CA80704B1B78002B40F0C58090
:102D000004F11401022289B22846FFF7E9FE04F11A
:102D10001E01042289B22846FFF7E2FE674E04F145
:102D20002801062289B22846FFF7DAFE3378FF2B06
:102D30002AD0634A12789A4226D95F4A614F1278A4
:102D400007920122069205220592002004F13C021E
:102D500009904FF0A8084FF6FF7092B208FB03717C
:102D60000890049203950293D1E91823CDE900233A
:102D70005548D1E90E2318F0C5FF337808FB0371DD
:102D8000D1E90E23C1E918237378FF2B2BD04C4ACD
:102D900012789A4227D9484A4A4F1278079201225C
:102DA000069205220592002004F1460209904FF098
:102DB000A8084FF6FF7092B208FB037108900492C6
:102DC00003950293D1E91823CDE900233E48D1E9C8
:102DD0000E2318F097FF394B5B7808FB0371D1E99C
:102DE0000E23C1E918230120FDF719FDFF285FD04C
:102DF000334B1B7883425BD93378834258D02F4BB7
:102E00005B78834254D02C4B2E4F1B7807930022C3
:102E100050340992A8264FF6FF724FF0010805239F
:102E2000A4B206FB007102900892CDF818800593B9
:102E300004940395D1E91823CDE900232248D1E970
:102E40000E2318F05FFF4046FDF7E9FC06FB00701B
:102E5000D0E90E23C0E918232AE0214628460B9327
:102E6000FFF710FE0B9BC6E60A23CDF80480009303
:102E7000324619233946154822F07AF81449134886
:102E8000FDF781FB4FF00108DAE64FF0000A0A2354
:102E90008DE8080432461E2339460C4822F068F8B3
:102EA000CDF800A042464B460848FDF71EFD27E737
:102EB0000DB0BDE8F08F00BF3C88FF1F2688FF1FC4
:102EC00022C4FF1F8890FF1FB0BCFF1F08C6FF1F52
:102ED000D31703002DE9F04F9C4B9D4D1B7813F049
:102EE000FD0087B001D1287014E09A4A1278C82AF0
:102EF00015D9DB0713D5984B187880B9974B1B78F9
:102F0000FF2B0CD1964B05221A70964A137843F08A
:102F1000010313708E4B187007B0BDE8F08F924B11
:102F20001A78012A1E4627D01B78042B14D18F4B08
:102F30008F4A5B7812789A420ED98E4AA82404FBF5
:102F400003248D4B586829F051FA02460B46D4E908
:102F50000E0129F025FD78B93378042B05D1834B78
:102F6000834A1B7812789A4208D832787E4B022A1C
:102F700014D01A78042A13D10020CBE77D4AA82464
:102F800004FB03247C4B186829F030FA02460B46F8
:102F9000D4E90E0129F004FD0028E6D06420B9E749
:102FA0001A78052A14D01A78062A13D01A78072A14
:102FB00012D01A78082A11D01B78092B40F0C28051
:102FC0006E4B6B491A78097891429A4608D8B9E055
:102FD00050209FE73C209DE728209BE7142099E79D
:102FE0001B78DFF890B1A82101FB03B3D3E90E678A
:102FF0009AF8003001FB03B3D3E912459AF8003088
:1030000001FB03B122462B46D1E9160129F08EF8C7
:10301000002200238046894629F0A4FC90B922466C
:103020002B463046394629F081F80022544B29F0CE
:1030300031FA42464B4629F057FB0022002329F083
:1030400077F801E00020002129F0FCFCC6B2092E2F
:1030500075D89AF800109AF80030DFF82881A82770
:1030600007FB01B107FB03B3D3E91223D1E9160132
:1030700029F05CF80022424B29F036FB9AF8003028
:1030800007FB03B3D3E90E23CDE900239AF8003000
:1030900007FB03BBDBE9122304460D463046CDE9AE
:1030A000022329F091F922462B4629F0F3F98246B2
:1030B00018F806008B4629F077F906F10109064653
:1030C00048460F4629F080F922462B4629F0E2F9BE
:1030D00052465B4629F02AF80022002318F809809E
:1030E000CDE9040129F03EFC20BBDDE90223DDE946
:1030F000000129F01BF852465B4629F017F80446F8
:1031000040460D4629F050F932463B4629F00EF86C
:1031100002460B462046294629F0BCF9DDE9042386
:1031200029F0E2FA02460B463046394629F000F80B
:1031300006460F463046394629F05CFC03E0114B49
:10314000987AE7E62878C0B2E4E600BF5BC7FF1FC5
:10315000B8C4FF1F28C5FF1FDA8EFF1F0C88FF1F92
:103160008CC7FF1FE8C4FF1F7990FF1F2688FF1F31
:1031700022C4FF1F8890FF1F8CC5FF1F21C4FF1FA3
:103180000000244078C5FF1F244B33F8102044F280
:1031900008239A423AD00FD81F2A2FD001D8B2B3B1
:1031A00039E0B2F5FC6F23D040F2FF739A4232D17E
:1031B000FF22114600202CE04FF6C0439A4221D056
:1031C00009D8B2F5784F16D04FF61F039A4222D194
:1031D000FF2200211CE04FF6E0739A4205D04FF623
:1031E000FF739A4217D1FF2211E00022FF2107E06E
:1031F0000022FF210CE00022114605E0FF22002101
:10320000084606E00022A521FF2002E0A522114683
:10321000104623F0F4B90020704700BF1288FF1F4A
:10322000F8B50E4B1B780546BBB10D4F0024FF2DA2
:103230000ABF07EB440328465878FFF7A5FFA6B25C
:10324000024631460748013423F0A7F9082CEED195
:103250000448BDE8F84023F0D3B8F8BDFC87FF1F51
:103260002988FF1F10C5FF1F0D4B30B51B889B1A07
:10327000994285B011DA5408031B0A44044412B27F
:103280004FF6E07524B202928DE8140003950AB25D
:103290001BB201B2034820F0F9FE05B030BD00BFFB
:1032A0003E88FF1F08C6FF1F064B82B01A680092B7
:1032B00000991A680192019A521A8242F9D902B011
:1032C000704700BF00D8FF1F13B504461DF019F961
:1032D0008DF8060020461DF014F98DF80700BDF8A2
:1032E000060002B010BD13B504461DF00AF98DF8B2
:1032F000040020461DF005F98DF8050020461DF05C
:1033000000F98DF8060020461DF0FBF88DF8070047
:10331000019802B010BDFFFFF8B5234CA82303FBB2
:10332000004408460D4629F04FF8D4E9222329F03D
:10333000B1F80646C5F57F7003300F4629F044F812
:1033400002460B463046394629F0CEF926F020FBDE
:10335000D4E9202306460F4629F09CF832463B4626
:1033600029F098F8D4E91E2328F0E2FE32463B46C5
:1033700029F090F8D4E91C2328F0DAFE02460B4627
:1033800000200A4929F0B0F905A3D3E9002328F069
:10339000CDFE29F02FFB00B2F8BD00BFAFF30080D7
:1033A00000000060661271408890FF1F0000F03F2F
:1033B0002DE9F04FA14B90461A78032A95B00646A6
:1033C0000C4699461AD19E4D9E499F482F4605F1BD
:1033D0000F0A57F8072B25F052FE17F8012F9B49CB
:1033E000994825F04CFE5745F7D1994B6A791B68EF
:1033F0000A930A9B9749944825F041FE99F80030BA
:10340000042B2BD11323944A94490CA81DF050FA95
:103410000CA99348FEF7D6F80CA81DF0C5F8904803
:103420001DF005F9B8B1324686498D4825F027FED2
:10343000651EE71D15F8012F8449894825F01FFEF8
:10344000AF42F7D1824B83491B680B930B9B844897
:10345000424625F014FE82481DF0DDF8814B1D79AF
:1034600019680023DAB2AA4208D2DA0088188A580A
:10347000964203F10103F5D103799BB97A4B5B685E
:103480009E4240F0808100230CE093F80890B9F14F
:10349000060F15D0B9F1070F14D122781B6993429A
:1034A00012D0019B704A0133DBB20193019B5D1E78
:1034B000EDB2A82303FB05235A689642E5D062E1EA
:1034C000012102E0494600E0002100230022CDE96D
:1034D0000C23654B4FF0A80808FB053898F80A3014
:1034E000012B0DD198F80B301BB998F80930E25632
:1034F00010E098F80930E25C0023CDE90C235CE091
:1035000001291DD1022B0BD198F80B3023B998F863
:103510000930E25ED317F0E798F80930E25AEBE79A
:10352000042B4AD198F80B301BB998F80930E258AF
:10353000F0E798F80930E3580C9300230D933CE032
:1035400011BB022B0BD198F80B301BB998F809303E
:10355000E25E0CE098F80930E35A5BBA11E0042B04
:103560002BD198F80B3023B998F80930E258D2BA29
:10357000D0E798F80930E3585ABA1B0C5BBA43EA13
:1035800002430C930D9118E0042916D1042B14D199
:1035900098F80930E118E25C4878CB78120642EAE4
:1035A00000421A438B7842EA0322D317CDE90C2359
:1035B0000C9828F01BFFC8E90E012B4B4FF0A80B0D
:1035C0000BFB053BDBF8100000286BD09BF80B10C1
:1035D00002460023CDE90423DDE90C9A002945D1F8
:1035E0009BF81420002A41D09BF80C304FF00008C3
:1035F0001A444FF0010E0EFA02F200EA090708EA37
:103600000A08CDE90278174008EAE27857EA08028A
:103610002CD01A46049328F06BFD049B6FEA000837
:103620006FEA01091A46DDE9020128F06DFD40EA62
:10363000080041EA0901CDE90C013DE08CBAFF1F09
:10364000ACC9FF1FC1100300848AFF1FC61003000E
:1036500000D8FF1FCC1003009B110300E0D4FF1F14
:10366000F0C4FF1FA0C9FF1F8890FF1F474BDDE973
:1036700004014FF0A80808FB053800EA090098F893
:103680000C2001EA0A0128F03FFD28F0D5FED8E918
:103690000A2328F0FFFED8E90C2328F049FDC8E9E9
:1036A0000E0115E0B9F1040F04D1DBE90A23DBE9CF
:1036B0000E0105E0DDE90C0128F0BEFEDBE90A237E
:1036C00028F0E8FEDBE90C2328F032FDCBE90E01FF
:1036D0002E4B4FF0A80808FB053898F86830012BEE
:1036E00041D1D8E90E23CDE90423D8E91C23CDE943
:1036F0000223D8E92223D8E91E01CDE90623DDE91A
:10370000022328F013FD00220023D8E920ABCDE9E5
:10371000080129F027F9F8B9DDE90223DDE9040100
:1037200028F004FD52465B4680468946DDE90601E5
:1037300028F0FCFC02460B464046494628F0AAFE0B
:10374000DDE9082328F0D0FF02460B4650465946D3
:1037500028F0EEFC82468B460C4AA82303FB052387
:10376000C3E90EAB0AE0022B08D1BDF930102846A0
:10377000FFF7D2FD28F028FEC8E90E0101212846F6
:10378000FEF790FA8DE615B0BDE8F08F8890FF1F28
:103790002DE9F04FA34AA82303FB00238BB05E7AE8
:1037A0000592042E05460F4600F2DC809E4B985D84
:1037B00023F0F0F816F0FD0F04B23ED140F28E3344
:1037C0009C423ADC40F27A339C4202DDA0F10804CC
:1037D00032E040F266339C4202DDA0F10D042BE0A2
:1037E000B4F5517F02DBA0F1120425E0B4F5397F76
:1037F00002DDA0F119041FE040F276239C4202DDB5
:10380000A0F1240418E040F262239C4202DDA0F102
:10381000280411E0B4F5117F02DDA0F122040BE0D1
:10382000B4F50C7F02DDA0F11C0405E040F2062394
:103830009C4202DDA0F1180424B24FF4CA73734312
:103840007A4AD058652101FB06014FF0650E42F817
:103850002140D1580131D150D158B94224BF012162
:10386000D1500020002300210EFB06F601335FFA41
:1038700083FE774508D906EB030E52F82EE010EBD5
:103880000E0041F10001F1E77A1ED31729F07AFC0E
:1038900028F0CAFD059B4FF0A80808FB053806462E
:1038A00098F86830022B0F460ED129F0A3F801B228
:1038B0002846FFF731FD28F087FDD8E90A2328F0D4
:1038C000E9FDD8E90C232EE0012B33D1D8E91C23E4
:1038D000D8E91E01CDE9022328F028FC00220023AC
:1038E000D8E920ABCDE9060129F03CF800BB5246EF
:1038F0005B46D8E9220128F019FCDDE90223804665
:1039000089463046394628F011FC02460B464046AF
:10391000494628F0BFFDDDE9062328F0E5FE024612
:103920000B465046594628F003FC06460F4601E078
:1039300056465F463E4B1B78032B04D14FF4D6709E
:10394000FCF76DFF88B9374AA82303FB0525D5E9A5
:103950000A233046394628F09DFDD5E90C2328F08E
:10396000E7FB5CE00020002159E032493248FCF7D7
:103970000AFE29463048FCF7AEFF30492E48FCF7D6
:1039800002FE21462C48FCF7AAFF02242B492A48B4
:10399000FCF7F9FD32463B4600942748FCF7A5FFAB
:1039A00026492548FCF7EFFD059A0094A82303FB60
:1039B000052ADAE91C232048FCF797FF1F491E4817
:1039C000FCF7E1FD0094DAE91E231B48FCF78DFFAC
:1039D0001A491948FCF7D7FD0094DAE92023164864
:1039E000FCF783FF15491448FCF7CDFD0094DAE994
:1039F00022231148FCF779FF10490F48FCF7C3FD5B
:103A00000F490D48FCF7BFFD0E4B0B481B6809938F
:103A10000999FCF766FF084825F01AFB93E70BB0FD
:103A2000BDE8F08F8890FF1F5CC7FF1FC0C9FF1F54
:103A30008CBAFF1F7D120300848AFF1FA9160300A2
:103A40008712030000D8FF1F2DE9F04FAB4DDFF8C0
:103A5000B09289B005F105084FF0A80A15F8017F6A
:103A6000A74C0AFB079696F890306BB14FF48E7016
:103A7000FCF7D5FE01463846FFF78AFEC6E90E017F
:103A800001212878FEF70EF9A845E7D19D4E9E4DFD
:103A900032782B789A4219D2262022F07BFF377891
:103AA00040F21D13C0F1D8005843A82606FB074674
:103AB00000F6FC0028F088FCD6E90A2328F0EAFC8E
:103AC000C6E90E0101213846FEF7ECF88F4B029350
:103AD0001A78FF2A53D08E4B2F781E78BE424ED2D2
:103AE0000120FCF79CFE8742824648D90320FCF760
:103AF00096FE874243D9A82707FB0040D0E90E89EC
:103B00000022844B4046494628F054FF002800F02C
:103B1000BE807B4B07FB0A3A42464B46DAE90E0170
:103B200028F0E2FD28F08EFFC0B229F0B5F87A49FE
:103B3000009029F005F9794901904FF0000A07FB40
:103B40000646D1F80080764F0391D346029B13F8C6
:103B50000B0029F0A1F881460146019829F0ACFA42
:103B600000287AD10BF101035FFA83FBBBF1050F4B
:103B7000ECD9BAF1000F02D0039BC3F80080694B67
:103B800093F800A0BAF1010F3BD1674B2A781B785C
:103B90009A4255D9A82202FB0343D3E90E67634B2F
:103BA000186828F023FC8046894602460B463046BA
:103BB000394628F0F5FE40B15D4B1A78012A00F035
:103BC000078183F800A051460CE042464B46304640
:103BD000394628F0DBFE48B1554B1B7833B1544BC6
:103BE00000211970534B187823F0DEFA524B2A78D3
:103BF0001B789A4224D9A82606FB03464C4B18781A
:103C00001AE0BAF1030F04D1494F3B78C3B901213F
:103C100007E0BAF1020F13D1454F3B78012B0FD1CA
:103C20000021444B3970187823F0BEFA424B3878A3
:103C30001B78A82606FB034628F0B6FBC6E90E0152
:103C40003E4B1E78FF2E00F0CD800520FCF7E7FDEF
:103C50002D78A842074634D3C4E03949009829F0AA
:103C60006FF80146484629F027FA00283FF47AAF5A
:103C70000BF1010028F0A8FB3B680593C6E90E0193
:103C8000DDF814804FF0010A4FF0060B6AE70022BE
:103C9000204B4046494628F079FE50B9204B1F4A38
:103CA0001B680693069B12689B1AB3F57A7F7FF612
:103CB00066AFA82303FB064600220023C6E90E23B5
:103CC0005DE70420FCF7ABFD85423BD9A82303FB4D
:103CD000074703FB004003FB0645D0E90E23D7E965
:103CE0000E0128F023FAD5E90A2328F0D3FBD5E901
:103CF0000C2328F01BFAC5E90E0164E08DBAFF1F02
:103D00008890FF1F0288FF1F22C4FF1FD4D4FF1F0B
:103D10004288FF1F000008403333933FCCD4FF1F7D
:103D200000D8FF1FA4C5FF1FBCC9FF1F64C7FF1F2A
:103D30000E88FF1FD88EFF1F4388FF1F0788FF1FB5
:103D40009A99593F40F21D10FCF769FD012849D1AD
:103D5000264A274B12681B680792079A03F5FA73E5
:103D60009A423FD90520FCF75AFDA82303FB0040E7
:103D7000D0E90E89002200234046494628F0F2FD92
:103D80001C4D50B90021286829F06EF928B1404631
:103D9000494628F077FE286024E0A82000FB06446E
:103DA000286828F023FB02460B464046494628F087
:103DB000BDF9D4E90A2328F06DFBD4E90C2328F0DF
:103DC000B5F9C4E90E0101213046FDF76BFF09E0AA
:103DD00042464B463046394628F0D8FD00283FF48D
:103DE00005AFFCE609B0BDE8F08F00BF00D8FF1FAB
:103DF000D08EFF1FE48EFF1F10B572B60C4B41240E
:103E00001C7003F8010C073B80201870187800061E
:103E1000FCD5084B1B788B54074B0A441B78537016
:103E2000064B1B789370064B1B78D37062B610BD9F
:103E3000070002400B0002400A0002400900024055
:103E40000800024073B50F490F4801AEFCF79BFB19
:103E5000002231460F20FFF7CFFF4FF4C675002434
:103E60002846FCF7DCFCA5F5C6730135F35C8342FC
:103E70001CBF0134E4B2B5F5C87FF1D1204602B0D1
:103E800070BD00BF8E120300848AFF1FF0B595B08D
:103E90002C22002109A822F077FCA94901A825F0CD
:103EA0003AFA4FF4C6750A272846FCF7B8FC0928E9
:103EB000044608D8A34901A8FCF7FDFCA14901A8C4
:103EC000FCF7F9FC22E0632820D89E4901A8FCF702
:103ED000F2FCB4FBF7F60A22F1B205A825F04EFA7F
:103EE00005A901A8FCF7E5FC05A825F0D4F907FB16
:103EF00016410A22C9B205A825F040FA05A901A871
:103F0000FCF7D7FC05A825F0C6F903E0214601A877
:103F100025F002FB0135B5F5C87FC5D12C22002361
:103F200009A901A825F064FB09A821F0C4FE10210D
:103F3000054621F035FA0446284629F043FB2022A5
:103F40002146814829F058FB80B9804905A825F011
:103F5000E2F905A94FF4FC627D4815F0FFF905A8C8
:103F600025F099F901214FF48B7067E0794901A898
:103F700025F04EFA4FF4C6750A272846FCF74FFC89
:103F80000928044608D86F4901A8FCF794FC6D493C
:103F900001A8FCF790FC22E0632820D8694901A819
:103FA000FCF789FCB4FBF7F60A22F1B205A825F06C
:103FB000E5F905A901A8FCF77CFC05A825F06BF93B
:103FC00007FB16410A22C9B205A825F0D7F905A9B1
:103FD00001A8FCF76EFC05A825F05DF903E0214679
:103FE00001A825F099FA0135B5F5C87FC5D12C2275
:103FF000002309A901A825F0FBFA09A821F05BFE1E
:104000001021054621F0CCF90446284629F0DAFAB9
:10401000202221464C4829F0EFFAA8B94E4905A8BC
:1040200025F079F905A94FF4FC62494815F096F995
:1040300005A825F030F901214FF48D70FCF782FBC3
:10404000204629F0BFFA75E0444901A825F0E0F9BF
:104050004FF4C6750A272846FCF7E1FB09280446F9
:1040600008D8384901A8FCF726FC364901A8FCF716
:1040700022FC22E0632820D8324901A8FCF71BFC6F
:10408000B4FBF7F60A22F1B205A825F077F905A9E5
:1040900001A8FCF70EFC05A825F0FDF807FB16416A
:1040A0000A22C9B205A825F069F905A901A8FCF7FB
:1040B00000FC05A825F0EFF803E0214601A825F053
:1040C0002BFA0135B5F5C87FC5D12C22002309A9EB
:1040D00001A825F08DFA09A821F0EDFD1021054673
:1040E00021F05EF90446284629F06CFA2022214688
:1040F000154829F081FA80B9194905A825F00BF96E
:1041000005A94FF4FC62124815F028F905A825F01E
:10411000C2F802214FF4E77090E7124905A825F094
:10412000FAF80B484FF4784205A915F017F905A8DD
:1041300025F0B1F801A825F0AEF815B0F0BD00BF2C
:104140009C12030049150300C4C4FF1FBA120300E8
:10415000E0BAFF1FDB120300F9120300171303007C
:10416000351303005C13030038B546F22C311248B6
:104170001EF07BFD012110481EF071FD0F490E4815
:10418000FCF701FA4FF4C6742046FCF748FB0928F7
:10419000054601D80A4902E0632803D809490648C0
:1041A000FCF7F1F9294604480134FCF794FBB4F517
:1041B000C87FE9D138BD00BF08C6FF1F6A130300DE
:1041C000681B0300491503002DE9F041074688B03C
:1041D00068B9C34BC34AB3F90030019012880D3A55
:1041E00012B2009201460D22BF4820F0C1FEBF4B23
:1041F00000221A70BE4B00221A60BE4BFF221A70BA
:104200003FB93B46DC222821B74820F001F8FFF7F0
:10421000ABFFB924052646F22C3300258DE850006B
:1042200002931E22E6232821AF4820F0F9FE8DE8F4
:104230005000E6231E2204AC2821AB4802951FF053
:1042400003FDAD49AD4E204625F065F80F2323222E
:104250002D210093AA480295DC23019415F058F90A
:10426000204625F018F829469F481EF0FEFC012143
:104270009D481EF0F4FC2B46272232219A481FF05D
:10428000C7FF7019143514F0D3FFB5F5027FF8D1CC
:10429000002519269B49204625F03DF82823372282
:1042A0008721994802950194009615F031F920462E
:1042B00024F0F1FF9549204625F02DF828233722D8
:1042C000B421934802950194009615F021F92046F7
:1042D00024F0E1FF8F49204625F01DF828233722DE
:1042E000E1218D4802950194009615F011F92046C0
:1042F00024F0D1FF8949204625F00DF828235522C6
:104300008721874802950194009615F001F920460F
:1043100024F0C1FF8349204624F0FDFF28235522C5
:10432000B421814802950194009615F0F1F82046D9
:1043300024F0B1FF7D49204624F0EDFF28235522CB
:10434000E1217B4802950194009615F0E1F82046A2
:1043500024F0A1FF7749204624F0DDFF28237322B3
:104360008721754802950194009615F0D1F82046F2
:1043700024F091FF7149204624F0CDFF28237322B9
:10438000B4216F4802950194009615F0C1F82046BB
:1043900024F081FF6B49204624F0BDFF28237322BF
:1043A000E121694802950194009615F0B1F8204684
:1043B00024F071FF6549204624F0ADFF28239122A7
:1043C000B421634802950194009615F0A1F82046A7
:1043D00024F061FF5F49204624F09DFF2823372207
:1043E0002D215D4802950194009615F091F8204624
:1043F00024F051FF5949204624F08DFF28235522EF
:104400002D21574802950194009615F081F8204619
:1044100024F041FF5349204624F07DFF28237322D6
:104420002D21514802950194009615F071F820460F
:1044300024F031FF4D49204624F06DFF2823372218
:104440005A214B4802950194009615F061F82046D8
:1044500024F021FF4749204624F05DFF2823552200
:104460005A21454802950194009615F051F82046CE
:1044700024F011FF4149204624F04DFF28237322E8
:104480005A213F4802950194009615F041F82046C4
:1044900024F001FF4FF023083A49204624F03BFF67
:1044A0004423AF222D21384802950194CDF8008095
:1044B00015F02EF8204624F0EEFE3449204624F074
:1044C0002AFF4423AF227621314802950194CDF88A
:1044D000008015F01DF8204624F0DDFE5AE000BFF4
:1044E0000488FF1F3E88FF1F08C6FF1F0088FF1FAC
:1044F000C0C5FF1F0988FF1F8F110300A4BAFF1F4B
:10450000E0BAFF1FCC1603006CBBFF1F871303002C
:1045100080BBFF1FD416030094BBFF1FD8160300F7
:10452000A8BBFF1FBF1A0300BCBBFF1F90180300EE
:10453000D0BBFF1F5D150300E4BBFF1FF712030094
:10454000F8BBFF1F731303000CBCFF1F49150300CA
:1045500020BCFF1FE814030034BCFF1F6E2F0300B4
:104560005CBCFF1FF41D030084BCFF1F7513030018
:1045700048BCFF1F462F030070BCFF1F1D880300AF
:1045800098BCFF1FF013030030BBFF1F771303001D
:10459000F4BAFF1F1549204624F0BDFE14480295C9
:1045A0000194CDF800804523AF22BF2114F0B0FF65
:1045B000204624F070FE0FB90E4902E0012F11D100
:1045C0000D49204624F0A7FE4FF6E07302930B48F6
:1045D00001940096282391222D2114F099FF204662
:1045E00024F059FE08B0BDE8F08100BF7F1303003E
:1045F00008BBFF1F86130300D81603001CBBFF1F58
:104600002DE9F043A14D89B006460F46904600249F
:104610002819143414F00CFEB4F5027FF8D19C4B29
:104620009C4800251D709C4B00221A609B4BB924AE
:104630001D701E2246F22C334FF0050911460293DD
:104640008DE810028C2320F0EBFC1E2211468C23F7
:104650008DE810028F48029504AC1FF0F5FA9049DE
:10466000204624F058FE23220F23114600938D4844
:1046700002958223019414F04BFF204624F00BFE98
:10468000294684481EF0F1FA012182481EF0E7FA1B
:104690002B46272228217F481FF0BAFDB8F1000FD2
:1046A00002D1CDF8008001E00223009332463B4660
:1046B000784800261925FCF718F97B49204624F094
:1046C0002AFE282337222321784802960194009558
:1046D00014F01EFF204624F0DEFD7549204624F02C
:1046E0001AFE282337225021724802960194009521
:1046F00014F00EFF204624F0CEFD6F49204624F032
:104700000AFE282337227D216C48029601940095E9
:1047100014F0FEFE204624F0BEFD6949204624F038
:10472000FAFD28235522232166480296019400951C
:1047300014F0EEFE204624F0AEFD6349204624F03E
:10474000EAFD2823552250216048029601940095E5
:1047500014F0DEFE204624F09EFD5D49204624F044
:10476000DAFD282355227D215A48029601940095AE
:1047700014F0CEFE204624F08EFD5749204624F04A
:10478000CAFD2823732223215448029601940095E0
:1047900014F0BEFE204624F07EFD5149204624F050
:1047A000BAFD2823732250214E48029601940095A9
:1047B00014F0AEFE204624F06EFD4B49204624F056
:1047C000AAFD282373227D21484802960194009572
:1047D00014F09EFE204624F05EFDB8F1010F1FD1BB
:1047E0004349204624F097FD282391222321414864
:1047F00002960194009514F08BFE204624F04BFDA8
:104800003D49204624F087FD3C48029601940095DE
:10481000282391227D2114F07BFE204624F03BFDCD
:104820003749204624F077FD002619239122009372
:104830005021282302960194324814F069FE204644
:1048400024F029FD23253049204624F064FD3E2331
:10485000AF2229460296019400952C4814F058FE88
:10486000204624F018FD2A49204624F054FD3E231A
:10487000AF226721029601940095264814F048FE65
:10488000204624F008FD09B0BDE8F083A4BAFF1F5C
:104890000088FF1F08C6FF1FC0C5FF1F0988FF1F34
:1048A0008F110300E0BAFF1FCC1603006CBBFF1F83
:1048B0008713030080BBFF1FD416030094BBFF1FA8
:1048C000D8160300A8BBFF1FBF1A0300BCBBFF1F05
:1048D00090180300D0BBFF1F5D150300E4BBFF1F52
:1048E000F7120300F8BBFF1F731303000CBCFF1F7C
:1048F0008913030020BCFF1F8B13030048BCFF1F5C
:104900004915030034BCFF1FF0130300F4BAFF1F66
:104910007F13030008BBFF1F10B5074C20461EF095
:1049200013FA204601211EF09AF920464FF6FF7136
:10493000BDE810401EF099B908C6FF1F2DE9F041EF
:1049400090B00446FFF7E8FF0021AE48AE4E1EF0DF
:104950008CF9AE4B1878FCF74BFE3278012A33D134
:104960000A234FF4FC668DE8480032211F23A54836
:10497000A74D20F0FDFA002302223821A1481FF0A4
:1049800047FCA4499F48FBF7FEFDA349A348FBF75A
:10499000FAFD00242B78E1B2994204F101040FD210
:1049A000002208A815F010FB08A99C4824F030FB51
:1049B00008A824F070FC9A499848FBF7E4FDE9E761
:1049C000964824F045FBC0E0022A03D1954B1B78A2
:1049D00013B9A2E0092C76D80A234FF6E0758DE8CA
:1049E000280001221F233221864820F0C1FA8E4B75
:1049F00084481D780222002336211FF009FCFF2C79
:104A000018BF254689497F48FBF7BDFD29467D48EB
:104A1000FBF761FF864B1B680393864B039A1A6072
:104A2000854B04AC03F10802A04618685968274674
:104A300003C7083393423C46F7D118689A889B799C
:104A40003860BA80BB7130357C488DF819501BF046
:104A5000EEFD60B913234246794908A81BF028FFF0
:104A600008A97648FCF7AEFD08A81BF09DFD734829
:104A70001BF0DDFD044600B367497048644DFBF749
:104A800082FD00242B78E1B2994204F101040FD297
:104A9000002208A815F098FA08A9684824F0B8FA86
:104AA00008A824F0F8FB5E496448FBF76CFDE9E7D1
:104AB00064496248FBF71EFF47E063495748FBF72C
:104AC00019FF347041E0032A12D10A234FF6E07433
:104AD0008DE8180001221F2332214A4820F048FAAD
:104AE00033210023022247481FF092FB574929E057
:104AF000042A15D10A204FF478438DE809000122D9
:104B00001F2332213F4820F033FA332100230222B1
:104B10003C481FF07DFB4E4914E0092C7FF65CAF4A
:104B20000A2146F22C338DE80A0001221F2332218C
:104B3000344820F01DFA33210023022231481FF0AF
:104B400067FB44492F48FBF71EFD434B1B78002BA6
:104B500051D0424B2B481C886408323421B2A4B295
:104B60000A224FF6E073671C02264FF478458DE861
:104B70000C003FB20E23012220F0FAF939460096CC
:104B80000C2308221F48019520F0F2F933463946DC
:104B9000009606221B48019520F0EAF9A71D04F1B2
:104BA0000B014FF0040833460096062209B215485F
:104BB00001953FB220F0DCF93346324639461148C0
:104BC0000195CDF8008020F0D3F9062604EB08010A
:104BD0003B46424609B20B48019500961EF0D2FAB8
:104BE000E31D04F10901019500961BB2424609B28A
:104BF00004481EF0C7FA0320FCF7FAFC10B0BDE829
:104C0000F08100BF08C6FF1F8CBAFF1F2888FF1F56
:104C100022C4FF1F8D130300F7100300848AFF1FB7
:104C200040110300DBD4FF1F4188FF1FFB1403006A
:104C300000D8FF1F2CC5FF1F02110300F0C4FF1F87
:104C4000E0D4FF1F8F110300911303009F13030093
:104C5000A5130300AB13030068C7FF1F0488FF1FE1
:104C60002DE9F0413B4C07462046FBF7A0FE3A4AAF
:104C7000012313702372394B394A00261E70394BB9
:104C800010781E70384B1978884215461C4612D28F
:104C9000DFF8E080022198F8000022F0B3FA98F8DB
:104CA0000000324B32491E6022284FF0030228BF19
:104CB000FF2022F0D9FA6A7823789A420FD22D4C3D
:104CC0000221607822F09EFA6078284B2A4900225F
:104CD00022285A6028BFFF20032222F0C5FA274B62
:104CE000274D00241C70274B2E681C70264B142067
:104CF0001C7024F0E8FC8046FBF77AFE4146304603
:104D00001DF030F8A7F16403012B07D814202C689C
:104D100024F0D9FC0546FBF775FE13E01B4B384623
:104D20001C70FFF70BFE1A4B1878FCF761FC194B4F
:104D30001B78042B0CD014202C6824F0C4FC0546EE
:104D4000FBF74CFE29462046BDE8F0411DF00AB8AD
:104D5000BDE8F0814CC4FF1F3C88FF1F74C7FF1FD4
:104D60003988FF1FDAD4FF1F22C4FF1F98BAFF1F24
:104D7000AD05000069C7FF1FBD05000095C6FF1FF8
:104D80004CD7FF1FC4C5FF1FBCC5FF1F96C6FF1F22
:104D90002888FF1F8CBAFF1F37B54FF6E074002834
:104DA00008BF00240546FFF7B7FD154B1B7801949B
:104DB000032B4FF00B0300934FF000024FF014034E
:104DC00007D0AA210F4820F0D3F800230222AC21FB
:104DD00006E0E6210B4820F0CBF800230222E82170
:104DE00008481FF015FA012D07D1002105481DF0D4
:104DF0003CFF05490348FBF7C6FB03B030BD00BFCD
:104E00002888FF1F08C6FF1F8D1303002DE9F043FC
:104E10008D4F8E4C3B78032B87B0054609D00C2173
:104E20000022B4F900308A488DE80600114620F0CF
:104E30009FF80320FCF7DCFB44F208260C22B4F9AF
:104E4000003083488DE844000022114620F090F89D
:104E5000FFF762FD3DB1032D00F0F080012D4FF40E
:104E600078460BD801E046F22C360B2300930196CE
:104E70002E2301220521764820F07AF8754902A8F0
:104E800024F049FA05230093032202AB192172484A
:104E900015F000FC02A824F0FEF915F0FD0F08D172
:104EA0000B23009301962E2301223721684820F01E
:104EB0005FF86A4902A824F02EFA05230093032222
:104EC00002AB4B21644815F0E5FB02A824F0E3F99E
:104ED000012D73D100215E481DF0C7FE604B1A788A
:104EE000012A1E4607D14FF6FF7159481DF0BDFE3D
:104EF0004FF4784301E04CF218634FF00B090122A4
:104F00000193A8212A235248CDF8009020F030F8D0
:104F10004FF00508534902A824F0FDF902AB032223
:104F2000BD214D48CDF8008015F0B4FB02A824F057
:104F3000B2F9002146481DF098FE3378012B56D077
:104F4000FCF7E2FD4CF21866FF2814BF4FF4FC6337
:104F50003346012201936F2134233D48CDF8009060
:104F600020F006F8404902A824F0D5F902AB03224C
:104F70008B213948CDF8008015F08CFB02A824F075
:104F80008AF93B783248CDF80090032B18BF4FF4D4
:104F9000FC662B230122D72101961FF0E9FF33493C
:104FA00002A824F0B8F92C48CDF8008002AB032207
:104FB000ED2115F06FFB02A824F06DF94FF6FF719B
:104FC00023481DF052FE032D16D121880B2046F2F6
:104FD0002C3332398DE8090009B22D2301221C48F7
:104FE0001FF0C6FF248822491E3CA4B215E04FF6EC
:104FF000FF7117481DF039FE218815480B2246F233
:105000002C3332398DE80C0009B22D2301221FF018
:10501000AFFF248817491E3CA4B202A824F07BF9F4
:1050200005230093032202AB21460B4815F032FB07
:1050300002A824F030F907B0BDE8F0834FF6FF7105
:1050400003481DF012FEC0E72888FF1F0488FF1FD9
:1050500008C6FF1FB1130300B0BCFF1F50120300AE
:105060000F88FF1FB9130300BE130300C71303000B
:10507000251B0300CE1303002DE9F0437E4B187867
:10508000A7B0002800F0F5807C4F7D4839880023C8
:1050900001937C4B1B88423B1BB26539009328224D
:1050A000652309B21FF064FF0123774A774916A8E8
:1050B0001BF0FEFBFFF730FC08230DEB03000A2278
:1050C0007349FBF70FFA062202A912A824F0DAFAB4
:1050D00070491EA824F01FF91EA912A824F0AFFAE7
:1050E00004461EA824F0D7F812A824F0D4F864B916
:1050F0000623224602A91EA824F0A4FA1EA902A88B
:1051000024F07EF91EA824F0C6F8DFF89C81FF2465
:105110000025012216A91EA81BF026FC1EA81BF0C4
:1051200086FA06461EA8002E00F081801BF03DFA8C
:10513000014606A824F0EFF81EA81BF038FA8146B5
:1051400000286DD154490AA824F0E5F80AA906A858
:1051500024F075FA002816DB01234A4606A90EA89A
:1051600024F070FA4D4912A824F0D5F812A90EA81F
:1051700024F065FAB0FA80F612A824F08CF80EA894
:10518000760924F088F80AA824F085F8002E47D183
:1051900098F80020AB1A0C2B01DC954202D20135A5
:1051A000EDB23DE003EB43023988354803EB820260
:1051B00029325D39334612B209B205F101091FF0F7
:1051C00027F849462E48FBF78AFB35492C48FBF760
:1051D000DAF906A92A4823F01BFF2F4912A824F068
:1051E0009AF812A906A824F02AFA3246034606A91C
:1051F0000EA824F027FA0EA824F04BFA014602A8C4
:1052000024F0C8F906460EA824F045F812A824F0A8
:1052100042F81EB198F800402C1BE4B25FFA89F501
:1052200006A824F038F81EA81BF0BEF971E71BF0A1
:10523000BBF91C4B16A81D701BF0EDF9FF2C11D00B
:10524000398804EB440204EB82020A204FF47843CD
:1052500028325E398DE8090012B25F2309B208488E
:105260001DF0D0FF02A824F016F816A81BF09CF938
:10527000204627B0BDE8F083DBD4FF1F0488FF1F62
:1052800008C6FF1F3E88FF1F90110300E0D4FF1FD8
:1052900030C5FF1FA9160300D31303007A140300BF
:1052A000D713030093BAFF1FE08EFF1F2DE9F043D1
:1052B000454B1978A1B0064619B90A2224F05EF8C8
:1052C0007DE00123414A4249DFF81481DFF814915F
:1052D00010A81BF0EDFAFFF71FFB0025012210A913
:1052E00018A81BF041FB18A81BF0A1F9044618A848
:1052F000002C58D01BF059F90146684624F00BF8F1
:1053000018A81BF054F90746002845D1314904A8D4
:1053100024F001F804A9684624F091F9002816DB6E
:1053200001233A46694608A824F08CF92A490CA8BA
:1053300023F0F1FF0CA908A824F081F9B0FA80F459
:105340000CA823F0A8FF08A8640923F0A4FF04A870
:1053500023F0A1FF04BB98F8002099F80030134413
:105360009D4217D11B490CA823F0D5FF0CA9684614
:1053700024F065F9224603466946304624F062F976
:105380000CA823F088FF684623F085FF18A81BF0BF
:105390000BF911E00135EDB2684623F07CFF18A847
:1053A0001BF002F99AE71BF0FFF810A81BF033F985
:1053B0000A49304623F0AFFF10A81BF0F5F830463D
:1053C00021B0BDE8F08300BFDBD4FF1F90110300C4
:1053D000E0D4FF1FD31303007A1403004915030020
:1053E00094C5FF1FE08EFF1F2DE9F0438B4C8C4EC0
:1053F0002288338891B00A210025653B0A3A8DE85E
:1054000022001BB212B20121804686481FF0B0FD77
:10541000228884480A3A2B4612B201211EF0F8FE77
:10542000814B1B7843B981497E48FBF7ACF84FF4B8
:105430007A7022F05DF8EDE072B6FFF76DFA7C4B02
:1054400002AD03F1100E2A46186859682F4603C7AB
:10545000083373453D46F7D118689B883860BB8098
:105460007449532308A808F130088DF818801BF000
:105470001FFA08A81BF0DBF80546002800F09C8006
:105480006D4B6E4A1B7812786D496E4C08A823F05C
:10549000F6FD04F5EE670026A04694F85830002B80
:1054A0007DD094F827300B2B05D1A38B093B9BB201
:1054B000022B40F2A380B4F9101008A8FBF70FFAF2
:1054C000614908A8FBF75FF8B4F9121008A8FBF7C8
:1054D00006FA5D4908A8FBF756F8B4F9141008A8B5
:1054E000FBF7FDF9584908A8FBF74DF8B4F9161079
:1054F00008A8FBF7F4F9544908A8FBF744F894F816
:10550000271008A8FBF7E7F94F4908A8FBF73BF875
:10551000A18B08A8FBF7E3F94B4908A8FBF733F880
:10552000E18B08A8FBF7DBF9474908A8FBF72BF844
:10553000218C08A8FBF7D3F9434908A8FBF723F807
:10554000217E08A8FBF7C7F93F4908A8FBF71BF81D
:1055500094F82730ABB94FF07009012509FB068993
:1055600094F82430AB4213D909EB050308A8197E3F
:10557000FBF7B1F90135344908A8FBF704F8EDB29F
:10558000EEE70B2B01D0052B02D12378002B38D16D
:105590002E4908A8FBF7AEF908A81AF09EFF703450
:1055A000A74206F101067FF478AF08A81AF095FF2C
:1055B00008A81BF030F81CE022880A3A034612B211
:1055C000012118481EF024FE3388228815480195D1
:1055D0000A21653B0A3A00911BB212B201211FF069
:1055E000C7FC1B490F48FAF7CEFF4FF4FA6021F0D1
:1055F0007FFF62B608A81AF0D7FF0BE00023E38311
:1056000059E7214608A8FAF7BEFF0F4908A8FAF79C
:10561000BAFFBDE711B0BDE8F08300BF3E88FF1FB1
:105620000488FF1F08C6FF1FDBD4FF1FF31303000E
:1056300020140300E0D4FF1F0F88FF1F2888FF1FDE
:10564000FF130300B0BCFF1F401103008F110300C4
:105650000C1403002DE9F04FC24EA3B0934604AFE3
:1056600032883B610A3A002312B28A4680461946C4
:10567000BD4897F8A0901EF0CBFDFFF74DF907F15C
:1056800018001AF083FFB8481DF0DAF9824580F25D
:10569000AE81B5481DF0D7F90A38834580F2A7815D
:1056A00001234246B14907F158001BF001F907F107
:1056B000580107F11800FBF785FF1AF0B8FF044600
:1056C00007F158001AF070FF2CB94246A849A648C5
:1056D00023F0D5FC90E107F1180107F15800FCF721
:1056E0007BFA07F15800FDF7EFFD044607F158007B
:1056F0001AF05AFF44F642539C4240F03F8107F1B2
:10570000180107F15800FCF767FA07F15800FDF798
:10571000EAFD07F158001AF047FF07F1180107F1F9
:105720005800FCF759FA07F15800FDF7DCFD07F1C6
:1057300058001AF039FF07F1180107F15800FCF77B
:105740004BFA07F15800FDF7CEFDF86007F158005D
:105750001AF02AFF07F1180107F15800FCF73CFA8C
:1057600007F15800FDF7BFFD07F158001AF01CFFC4
:1057700007F1180107F15800FCF72EFA07F158005D
:10578000FDF7B1FD054607F158001AF00DFF07F1CE
:10579000180107F15800FCF71FFA07F15800FDF750
:1057A000A2FD786107F158001AF0FEFE07F118011A
:1057B00007F15800FCF710FA07F15800FDF784FDD7
:1057C000044607F158001AF0EFFE012C40F0D68095
:1057D00007F1180107F13800FCF7FEF907F138006E
:1057E000FDF772FD182811D107F1180107F15800D3
:1057F000FCF7F2F907F15800FDF775FDB0FA80F4F7
:1058000007F1580064091AF0CFFE00E0002407F108
:1058100038001AF0C9FE002C00F0B080C7F808D09C
:10582000ADB2BC8ABAF1000F11D1BBF1000F0ED19D
:10583000504B1A8833881B1B0221521B0A3B92FBD8
:10584000F1F293FBF1F31FFA82FA1FFA83FB3B6933
:105850007C612E467BB1484B702000FB093090F8EC
:105860002530428A018A029390F8273001930094F0
:105870002B461AF0B3FA05F1010909EB490929F0A1
:10588000030339483B611DF0DBF85544854205DDD3
:1058900035481DF0D5F8CAEB000086B232481DF03D
:1058A000D2F80BEB0405854206DD2F481DF0CBF83E
:1058B000CBEB000083B27B6106EB4605EB1D23F0CA
:1058C0000703ADEB030DABB2FA687B603B69013CAB
:1058D000564403FB0429B3B20DF110080024FB6009
:1058E0007B69A6B2B34239D907F118001AF075FEE8
:1058F000484504D0494607F118001AF065FE7A6859
:10590000414607F118001AF05AFE0BEB060292B25C
:105910000092FB68144851461FF012FC0026B54265
:1059200014DD08EB0603104899785B780902DB0068
:1059300001F4784103F4FC630B4318F806100336B6
:1059400043EAD1011DF052F9B6B2E8E706481DF06E
:1059500059F93B690134C3EB0909C1E7D7F808D00D
:105960003FE000BF3E88FF1F08C6FF1FE0D4FF1FB7
:10597000361403000488FF1FB0BCFF1F3288234B7E
:105980000B204FF6E0710B3AB3F9003012B28DE8FC
:10599000030000211E481FF0EBFA4FF478411C4829
:1059A0001DF063F941461A48FAF7EDFD1949184808
:1059B000FAF7E9FD414618481AF0CAFF4FF4FA70A9
:1059C00021F096FD154A702303FB0922938B0133C6
:1059D0009BB2FD2B938304D84A465946504600F0AB
:1059E00021F807F118001AF016FE012404E00C4912
:1059F0000748FAF7C8FD002407F118001AF0D4FD93
:105A000020467C37BD46BDE8F08F00BF0488FF1FED
:105A100008C6FF1F50140300E0D4FF1FB0BCFF1FD7
:105A2000431403002DE9F04F774B1C78A3B0814657
:105A30008A469046002C00F0E280744B7449702531
:105A400005FB023502A8AF8B23F065FC95F82730E3
:105A5000052B01D16F4902E00E2B03D16E4902A83C
:105A600023F0D6FC95F82730052B05D1284627F0E2
:105A700004FF012800F2BA80FFB2FF2F19D1049869
:105A8000013023F022FE049A04460146002301322D
:105A900002A823F0ADFD049B234400225A70204647
:105AA000CDF80080012352464946FFF7D3FD044656
:105AB00098E0DDF808B0594901235A4612A81AF0B7
:105AC000F7FE0026012212A91AA81AF04DFF1AA803
:105AD0001AF0ADFD044600287BD0594606A823F0F5
:105AE0001AFC1AA81AF061FD014606A8FAF7E3FEAF
:105AF0001AA81AF05CFD002864D149490AA823F0CD
:105B00000AFC0AA906A823F09AFD00280CDB4549E7
:105B10000EA823F000FC0EA906A823F090FDC443B4
:105B20000EA8E40F23F0B7FB0AA823F0B4FB002C67
:105B300048D1BE4241D10898013023F0C6FD089AF1
:105B4000014601320646234606A823F051FD089B74
:105B500033441AA85C701AF05EFD12A81AF05BFDBF
:105B60002B4906A823F054FC1AA81AF01EFD014682
:105B700006A8FAF7A0FE0898033823F0A6FD089AB5
:105B8000234607460146033A06A823F031FD089A4A
:105B90003946033A284620F05DFD01235246494626
:105BA000CDF800803046FFF755FD044606A823F0E7
:105BB00072FB1AA81AF0F8FC11E01AA81AF02BFDD3
:105BC0000136F6B206A823F066FB1AA81AF0ECFC20
:105BD00078E71AA81AF0E8FC12A81AF01CFD12A81F
:105BE0001AF0E2FC02A823F056FB08E0294602A8BE
:105BF000FAF761FE0A4902A8FAF75DFE3FE7204680
:105C000023B0BDE8F08F00BFDBD4FF1FB0BCFF1F87
:105C10008F110300651403006B140300E0D4FF1F11
:105C2000731403007814030073B51C4B1C4A1D4801
:105C30001D4D1E4E00241C701D4BB3F90030019405
:105C400012880C3A12B2009221460C221FF090F9F1
:105C5000184B1878FBF7CCFC174B01221A7095F8FB
:105C60005830E2B26BB195F8273013B926F81430EA
:105C700003E0052B0CD00E2B0AD0002128461AF089
:105C80005FF80134112C05F17005E8D102B070BD48
:105C9000698A288AFFF7C6FEF3E700BFBCC5FF1F6D
:105CA0003E88FF1F08C6FF1FB0BCFF1F26C4FF1F92
:105CB0000488FF1F2888FF1F3C88FF1F2DE9F04F35
:105CC000BA4FBB4E3A883388DFF83C939FB000242C
:105CD0000D46653B0A210A3A80468DE812001BB248
:105CE00012B20121B3481FF043F93A88B1480A3A89
:105CF000234612B201211EF08BFAFEF70DFEAE4BC9
:105D000099F800001C70AD4B1C70FBF771FCB8F1EA
:105D10000A0F40F09E803A88B6F80090A84BA94937
:105D200016AD243A4FF00B0B92B24FF0050A4FEA32
:105D30005909284683F800B0049223F0ECFA2B4668
:105D4000049ACDF800A049469F4814F0A3FC2846C9
:105D500023F0A1FA3A889D491A3A4FF01A0992B2F3
:105D60002846049223F0D7FA049A02942146282365
:105D70000195CDF80090964813F0CAFB284623F011
:105D80008AFA33883A889349293B1A3A9BB292B2ED
:105D900028460493059223F0BEFA059A04990294CA
:105DA00028230195CDF800908B4813F0B1FB2846CD
:105DB00023F071FA33883A88022044F20821703BBC
:105DC0000C3A8DE803001BB212B2332179481FF060
:105DD000CFF8824B187833883E3B22460093FA2155
:105DE0003223FAF7D0FC3F8804901A3FBFB27C49B7
:105DF000284623F090FA43463A46BDF81010029424
:105E00000195CDF80090774813F082FB284623F0E7
:105E100042FA31886748CDF800B046F22C33323967
:105E2000019301222D2309B21FF0A2F836886E4992
:105E30001E3EB6B2284623F06EFACDF800A02B46DF
:105E400003223146604814F025FC284623F023FA4B
:105E50000BE1B8F1080F26D1644E33781BB3DFF89D
:105E6000A081594F4FF0140909FB048013F0E0F9A9
:105E7000702303FB047301340025112C524883F86E
:105E80005850F1D1012380F85830DC2210238DE8DE
:105E90000C0002954FF49B730F22052119F09EFF11
:105EA0002C463570E1E0524B1C78002C00F0DD8070
:105EB000504B09AA03F11007164618685968144692
:105EC00003C40833BB422246F7D118689B88206080
:105ED000A38008F13008314647488DF834801AF025
:105EE0002BFD28B930238DF83430444B01221A7031
:105EF00001233246404916A81AF0DAFC032089F83B
:105F00000000FBF775FB16A81AF091FB0446002869
:105F100000F09F803A4F2C4E00244FF0140808FBED
:105F2000047013F085F9702303FB0463013400222D
:105F3000112C83F85820F2D1324B0FAA03F1180626
:105F4000904618685968144603C40833B342224681
:105F5000F7D100261868206037463446B14616A8A7
:105F60001AF046FB00286FD016A81AF0CAFA5FFA9A
:105F700080FA15B1504622F071FEBAF13B0F45D1BF
:105F8000072C06D81EAB2344013403F8609CE4B20E
:105F9000F6E706A827F082FA1EAB03EB46030136AC
:105FA00023F83C0CF6B20024D9E700BF3E88FF1F5F
:105FB0000488FF1F08C6FF1F96BAFF1FB9C5FF1F41
:105FC000FD87FF1F7C140300B0BCFF1F11110300ED
:105FD000E0BAFF1F13110300F4BAFF1F65C5FF1FCE
:105FE000A916030008BBFF1FCE1303003C88FF1F48
:105FF000DBD4FF1FB7140300E0D4FF1F0688FF1F88
:10600000A4BAFF1F5C0E03002888FF1FBAF10D0F12
:1060100002D0BAF10A0F10D17EB1092E384606AA75
:10602000414694BF8DF818908DF82090FBF72AFF19
:1060300000263844C7B2344691E71EAB23440134EE
:1060400003F860ACE4B28AE716A81AF0E4FA012477
:1060500008E008490848FAF796FA3246074908481E
:1060600023F00DF816A81AF09FFA20461FB0BDE8DD
:10607000F08F00BF8614030008C6FF1F9D140300A5
:10608000848AFF1FFFFFFFFF2DE9F04F8B469FB073
:106090000646002840F024830146BB48BB4DDFF88C
:1060A00080A31CF0E2FD0121B7481CF0D8FDB84BDD
:1060B000B548B3F9003001962A880C3A12B21AACEE
:1060C000314600920C2228271EF052FFB14920468B
:1060D00023F021F93C233A4650210296AE48019420
:1060E000009713F015FA204623F0D5F8AB49204667
:1060F00023F011F93E233A469A210296A8480194CA
:10610000009713F005FA204623F0C5F8A54920466C
:1061100023F001F93E23E22102963A46A248019477
:10612000009713F0F5F9204623F0B5F89AF80030FF
:106130009E49A84612AE16AD2046002B39D04FF42A
:10614000FC6923F0E8F83C235A2205219848CDF851
:1061500008900194009713F0DBF9204623F09BF898
:106160009249284623F0D7F80A229AF80010B1FB8A
:10617000F2F10EA823F002F90EA9304623F035F90A
:106180008C49304623F0E2F90146204623F02DF9F0
:106190004B4622462946864813F016F9204623F03E
:1061A0007AF8304623F077F80EA823F074F82846E2
:1061B0000DE023F0B0F846F22C3302937C480194B2
:1061C00000973C235A22052113F0A2F9204623F020
:1061D00062F8794B79491B78204623B123F09BF86C
:1061E0004FF4FC6303E023F096F846F22C3302935D
:1061F000282300935A223C2350217148019413F024
:1062000087F9204623F047F86E4B1B78012B06D107
:106210006D49204623F07FF84FF4FC631BE0022B0E
:1062200001D16A4902E0032B06D16949204623F0D7
:1062300072F84FF6E0730EE0042B06D16549204654
:1062400023F069F84FF4784305E06349204623F0D2
:1062500062F846F22C33029328235A229A210093A3
:106260005E4801943E2313F053F9204623F013F8BF
:106270004CF218695A492827204623F04CF83E234F
:106280005A22E2215748CDF808900194009713F064
:106290003FF9204622F0FFFF5349204623F03BF808
:1062A0003C2305218C225148CDF808900194009799
:1062B00013F02EF9204622F0EEFF4D4B4D491B788E
:1062C00020462BB123F027F84FF6E073029303E04A
:1062D00023F021F8CDF808903E238C22E22100978C
:1062E0004548019413F014F9204622F0D4FF4349A5
:1062F000284623F010F84CF2186941492827204617
:1063000023F009F83C23BE2205213E48CDF80C902D
:1063100002940195009713F0A0F9204622F0BBFFEC
:10632000284622F0B8FF3849204622F0F4FF5021D9
:106330003C238C223548CDF808900194009713F047
:10634000E7F8204622F0A7FF40F21B10FAF767FAA1
:106350002F490A2800F28480DFE800F06E060B1057
:106360006469828282827800284622F0D4FF29491B
:1063700070E0284622F0CFFF27496BE0284622F044
:10638000CAFF264966E000BF08C6FF1F3E88FF1F00
:106390000488FF1FCD140300B8BAFF1FD5140300F3
:1063A000CCBAFF1FE0140300E0BAFF1FEA14030099
:1063B000F4BAFF1F411603003D88FF1FF0140300CD
:1063C00008BBFF1F8CBAFF1FF7140300FF14030064
:1063D0009F130300A5130300061503001CBBFF1F3A
:1063E0000D15030058BBFF1F1715030030BBFF1F1F
:1063F00068C7FF1F20150300BCBBFF1F2915030042
:106400005A19030094BBFF1F2F150300F8BBFF1F91
:106410003715030040150300451503004B15030015
:1064200029C5FF1F284622F076FF974912E028462B
:1064300022F071FF95490DE0284622F06CFF944947
:10644000204622F068FF4CF2186312E0284622F042
:1064500062FF9049204622F05EFF4FF4FC6308E0A3
:10646000284622F058FF8C49204622F054FF4FF670
:10647000E073039328235021BE220093874802949F
:106480003C23019513F0E9F8204622F004FF28464A
:1064900022F001FF824B83491B78012B04D128464F
:1064A00022F039FF804905E0022B09D1284622F06D
:1064B00032FF7749204622F02EFF4CF218630AE0A3
:1064C000032B18D1284622F026FF7849204622F0D7
:1064D00022FF40F2FF73039328230093BE223C2344
:1064E0009A2173480294019513F0B7F8204622F0E0
:1064F000D2FE28460FE0204622F00DFF46F22C3354
:106500000293282300936A4801943C23BE229A21D7
:1065100012F0FEFF204622F0BEFE664B1B880BB336
:106520006549304622F0F7FE6449284622F0F3FE22
:106530006349204622F0EFFE4FF47843049328236A
:10654000BE22E22100935F4803943C23029501960A
:1065500013F01EF8204622F09EFE284622F09BFEF5
:10656000304643E0584B1B78022B0AD1524928464B
:1065700022F0D1FE5149204622F0CDFE4FF6E073C5
:1065800025E003F0FD02012A0AD14B49284622F0FA
:10659000C2FE4A49204622F0BEFE4FF4FC6316E0DC
:1065A000042B0AD14949284622F0B5FE434920462A
:1065B00022F0B1FE40F2FF7309E03F49284622F085
:1065C000AAFE3E49204622F0A6FE46F22C33039353
:1065D00028230093BE223C23E2213A4802940195ED
:1065E00013F03BF8204622F056FE284622F053FED8
:1065F000B8F800203648083A002312B201211DF0F5
:1066000007FEFDF7B1FD08230A2232493046F9F7AB
:1066100069FF06223146284623F034F82E492046E9
:1066200022F079FE2146284623F009F80746204645
:1066300022F031FE284622F02EFE67B906233A46A4
:106640003146204622F0FEFF2146304622F0D8FE99
:10665000204622F020FE46F22C311D481CF005FB9E
:10666000B8F800201A48083A002312B2C8211DF0D9
:10667000CFFD1A491648F9F786FF3146144822F033
:10668000C7FC01F034BE00BF4F15030057150300CF
:10669000B21B03005F1503000E12030044BBFF1F73
:1066A0005BC7FF1F671503009E1B0300F211030069
:1066B000E4BBFF1FC08EFF1F6E1503000117030010
:1066C000BB190300D0BBFF1F64C5FF1F7415030077
:1066D00008C6FF1F30C5FF1FA91603007815030069
:1066E000431E012B45F28D81DFF80C83B8F8004082
:1066F0000328A4F165091FFA89F940F0CF8000272B
:10670000DFF8F8820197B8F80030B3480D3B1BB2B0
:1067100000930D2223B239461EF02AFC32463B4636
:106720008221AD481DF074FD1AADAC49AA48F9F7B5
:106730002AFF4FF01A0AAA49284622F0ECFD6423EA
:106740000E224946A74802970195CDF800A012F005
:10675000DFFE284622F09FFDB8F80080A249A8F18C
:106760001A081FFA88F8284622F0D5FD424664230D
:1067700049469E4802970195CDF800A012F0C8FE48
:10678000284622F088FD4FF6FF719348DFF87482A7
:106790001CF06BFA32463B4682218F481DF038FDD3
:1067A0008E498D48F9F7EFFE2A260797904B9DF802
:1067B0001C701B78711EBB4289B203D800210520D2
:1067C00000F029BC2FB98B4A3B4612784846FBF7AC
:1067D000E5FAA4F15E0B4FF6FF717F481FFA8BFBC1
:1067E0000FFA86FA1CF041FA002352460FFA8BF199
:1067F00079481DF00DFDD8F8042040F6FF739A4249
:1068000014D198F80930032B10D8A4F1570152463F
:10681000002309B270481DF0FBFC3946032013F039
:10682000ABFB314602465846FCF75AF8724B3946E4
:10683000B3F800A0012013F09FFBAAF1140A1FFA7D
:106840008AFA024631465046FBF75EFF6A4B3946EC
:10685000B3F800A0002013F08FFBAAF10A0A1FFA78
:106860008AFA024631465046FBF714FF604B0B2272
:106870001B783946284613F0A7FB2946564822F0D4
:10688000C7FB284622F007FD079B01330D360D2B71
:106890000793B6B208F1A80888D18FE7042840F022
:1068A000B3800025554E019533884B48544F423BE9
:1068B0001BB20FFA89F10093282264231EF058FBC3
:1068C0004D4B32881B88444801951A21643B1A3A83
:1068D00000911BB2294612B21EF04AFB32883E4894
:1068E000DFF80C910A3A2B4612B201211DF090FC00
:1068F0004FF6FF7138481CF0B8F93D782A26CB4690
:106900003B780C33AB42C5F27C8099F80030AB4247
:1069100045F27780A4F15E084FF6FF712E481FFA0A
:1069200088F80FFA86FA1CF0A0F9002352460FFAF5
:1069300088F129481DF06CFC324AA82303FB05238B
:1069400040F6FF725968914213D15B7A032B10D83D
:10695000A4F157015246002309B21F481DF058FC0C
:106960002946032013F008FB314602464046FBF758
:10697000B7FF214B2946B3F80080012013F0FCFA41
:10698000A8F114081FFA88F8024631464046FBF782
:10699000BBFE194B2946B3F80080002013F0ECFA37
:1069A000A8F10A081FFA88F8024631464046FBF76C
:1069B00071FE9BF800300B2229461AA813F004FB45
:1069C0001AA9054822F024FB01351AA80D3622F039
:1069D00062FCEDB2B6B293E708C6FF1FCD14030008
:1069E00083150300A4BAFF1F86150300B8BAFF1F62
:1069F00022C4FF1F94C5FF1F0488FF1F3E88FF1F8E
:106A0000E08EFF1F8890FF1F052840F0A58200251B
:106A1000C34A01951288C348DFF848930D3AA4F1A0
:106A2000660312B21BB2009229460D221EF0A0FA94
:106A30004FF6FF71BB48BC4C1CF017F90121B94857
:106A40001CF00DF9B949B7481CF064F931462B46E2
:106A50002422B448B64E1DF0DBFB99F800302178B3
:106A60000F221AA813F0B0FA1AA9AE4822F0D0FAF1
:106A70001AA822F010FCAB481CF066F94CF2186121
:106A8000A8481CF0F2F82B462D220D21A5481DF038
:106A9000BFFBA849A348F9F776FD2B462D225F21BD
:106AA000A0481DF0B5FBA4499E48F9F76CFD23787A
:106AB0009C48A8274FF00208CDF8008007FB03632D
:106AC000D3E91023F9F711FF4FF6FF7195481CF039
:106AD000CCF82B463A220D2192481DF099FB97499C
:106AE0009048F9F750FD2B463A225F218D481DF062
:106AF0008FFB91498B48F9F746FD2378CDF800804C
:106B000007FB0363D3E912238648F9F7EEFE4CF244
:106B1000186184481CF0A9F82B4647220D218148B2
:106B20001DF076FB86497F48F9F72DFD2B4647225D
:106B30005F217C481DF06CFB7F497A48F9F723FD03
:106B40002378CDF8008007FB0363D3E9142375484D
:106B5000F9F7CBFE4FF6FF7172481CF086F82B4612
:106B600054220D216F481DF053FB76496D48F9F70B
:106B70000AFD2B4654225F216A481DF049FB6E49ED
:106B80006848F9F700FD2378CDF8008007FB036320
:106B9000D3E916236348F9F7A8FE2B466E220D2190
:106BA00060481DF035FB68495E48F9F7ECFC2B4660
:106BB0006E225F215B481DF02BFB5F495948F9F7B6
:106BC000E2FC2178284613F0D7F9FBF79FFE2178E5
:106BD000284613F0D1F96D2102465120FBF75AFDEA
:106BE0002B467B220D214F481DF012FB57494D4883
:106BF000F9F7C9FC2B467B2233214A481DF008FBDC
:106C000053494848F9F7BFFC7B222B463D214548B4
:106C10001DF0FEFA4F4B43481978F9F75CFE2B46FE
:106C20007B2247213F481DF0F3FA4B493D48F9F7D5
:106C3000AAFC2B467B225F213A481DF0E9FA3E4927
:106C40003848F9F7A0FC2178012013F095F9FBF7FB
:106C50005DFE2178012013F08FF97A210246512040
:106C6000FBF752FD237807FB036340F6FF72596878
:106C70009142B04625D15B7A032B22D82B4688223D
:106C80000D2128481DF0C4FA34492648F9F77BFC49
:106C900088222B465F2123481DF0BAFA2649214855
:106CA000F9F771FC2178032013F066F9FBF72EFE4B
:106CB0002178032013F060F9892102465120FBF767
:106CC0000FFE002395220D2116481DF0A1FA24493C
:106CD0001448F9F758FC002395225F2111481DF054
:106CE00097FA15490F48F9F74EFC217899F80030CA
:106CF000A82505FB0181002291F891101AA813F034
:106D000063F91AA9074822F083F91AA822F0C3FAF6
:106D10000023A2220D2103481DF07AFA24E000BFCF
:106D20003E88FF1F08C6FF1F94C5FF1F6C26030087
:106D30008890FF1F89150300911503009515030026
:106D4000A2150300AA150300B7150300EA140300F7
:106D5000BC1503006BC7FF1F572F0300BE150300B0
:106D6000C515030022C4FF1FAD49AE48F9F70BFC5F
:106D70000023A2225F21AB481DF04AFAAA49A94884
:106D8000F9F701FC237805FB038393F89120FF2A90
:106D900004D1A649A348F9F7F6FB06E002220092C7
:106DA000D3E926239F48F9F7A0FD0023AF220D2148
:106DB0009C489F4E9F4F1DF02BFA9F499948F9F729
:106DC000E2FB0023AF225F2196481DF021FA96498D
:106DD0009448F9F7D8FB2378A82505FB038393F89B
:106DE0006800FBF793FD237805FB038898F868306B
:106DF000012B36D10023BC220D218A481DF008FA50
:106E00008E498848F9F7BFFB0023BC225F218548E3
:106E10001DF0FEF984498348F9F7B5FB3B788148BA
:106E2000022405FB03630094D3E92023F9F75DFDF9
:106E30000023C9220D217B481DF0EAF980497948D9
:106E4000F9F7A1FB0023C9225F2176481DF0E0F984
:106E500075497448F9F797FB3B78009405FB036587
:106E600073E0022B44F0CD850023BC220D216D4838
:106E70001DF0CEF973496B48F9F785FB0023BC225E
:106E8000172168481DF0C4F967496648F9F77BFB8C
:106E90003B786448082405FB03630094D3E91C2372
:106EA000F9F723FD0023C9220D215E481DF0B0F93A
:106EB00065495C48F9F767FB0023C9221721594847
:106EC0001DF0A6F958495748F9F75DFB3B78009447
:106ED00005FB0363D3E91E235248F9F706FD00239F
:106EE000BC2271214F481DF093F958494D48F9F7DC
:106EF0004AFB0023BC227B214A481DF089F94A49FC
:106F00004848F9F740FB3B78009405FB0363D3E95D
:106F100020234448F9F7E9FC0023C92271214148A4
:106F20001DF076F94A493F48F9F72DFB0023C922A5
:106F30007B213C481DF06CF93B493A48F9F723FBAB
:106F40003B7805FB036500230093D5E922233548F0
:106F5000F9F7CBFC04F055BD062840F08D800025E4
:106F60003C4E019533882F48443B1BB21AAC282273
:106F700000930FFA89F164231DF0FAFF3649204689
:106F800022F0C9F93423422249460093334802953E
:106F90006423019412F0BCFA204622F07CF91A27EF
:106FA0002F49204622F0B7F96423AA2249462D48EA
:106FB00002950194009712F0ABFA204622F06BF98B
:106FC0002949204622F0A7F964230E224946274882
:106FD00002950194009712F09BFA204622F05BF98B
:106FE000368823491A3EB6B2204622F094F964232B
:106FF000324649461F4802950194009712F088FADC
:10700000204622F048F92C2102202B465A46FAF756
:10701000C5FE29460720FFF737F804F0F2BC00BF91
:10702000CF15030008C6FF1F91150300D8150300F4
:107030008890FF1F94C5FF1FDC150300E3150300B4
:10704000E6150300DA1503008F130300E54403007F
:10705000761403003E88FF1FF0130300CCBAFF1F15
:10706000E915030058BBFF1F83150300A4BAFF1FD7
:1070700086150300B8BAFF1F072829D161B9114A44
:10708000128801911A20A4F164031A3A00901BB2ED
:1070900012B20D481DF06CFF00210B481BF0E5FDFE
:1070A0000A4B1A78052A1AAC1D4604F091811A7809
:1070B000062A04F08D811A78072A44F0AE8104F084
:1070C00087B900BF3E88FF1F08C6FF1F96C6FF1F77
:1070D000092840F06F83FF2940F0C2810025DFF8C6
:1070E00078A3BF4EDFF874B3FDF716FCB8F9003093
:1070F0000195BAF80020BB480D3A12B20092294619
:107100000D221DF035FFB849B6481BF003FE2B4693
:1071100024220521B3481DF07BF8B449B148F9F7A2
:1071200032FAFDF7F9FBB2481AAC12F081F8B14817
:1071300012F07EF8B049204622F0EDF834234222C6
:10714000494601940093AD480295642312F0E0F99A
:10715000204622F0A0F8AA49204622F0DCF87378F5
:10716000A8483BF8133002931A2764237922494632
:107170000194009712F0CCF9204622F08CF8A24935
:10718000204622F0C8F8642349460E2201949F4805
:107190000295009712F0BCF9204622F07CF8BAF86C
:1071A00000209B491A3A92B22046079222F0B3F887
:1071B0006423079A0194494696480295009712F075
:1071C000A7F9204622F067F8BAF800909249A9F191
:1071D0001A091FFA89F9204622F09DF813234A461E
:1071E000294601948D480295009712F091F92046A6
:1071F00022F051F8B8F80090BAF800208849A9F1B7
:107200007D091A3A92B21FFA89F92046079222F0B4
:1072100082F849461323079A019482480295009701
:1072200012F076F9204622F036F8B8F80030BAF8B5
:1072300000206C4844F2082E0221A03B0C3A8DE855
:1072400002401BB212B219211DF092FEB8F80000E4
:10725000963825F0B9F80022734B24F067FF80467A
:107260003078894625F0A0F802460B46404649464C
:1072700025F010F900226D4B25F036FA00226A4BFA
:1072800024F056FF25F0DEFBBAF800806849A8F12B
:107290001A081FFA80F91FFA88F8204622F03BF8F6
:1072A0000A2342464946019462480295009712F02B
:1072B0002FF9204621F0EFFFFDF72EFB2D2427B2FA
:1072C0003A4600230D2147481CF0A2FF05F10108B2
:1072D00059494448F9F757F941464248F9F7FFFA46
:1072E00006EB4503621E5B783E483BF81330019382
:1072F0000923009312B20A2373211DF039FE3A4686
:1073000000233F2137481CF083FF16F8151035483D
:107310006423594345461F460D34F9F7E0FA082D1A
:10732000A4B2CCD1A22200230D212E481CF070FF64
:1073300042492C48F9F727F9414B187825F034F8E1
:107340000323002467250293A223019302460B46E0
:107350000494039400953B4814F014FC2346AF2298
:107360000D2120481CF054FF37491E48F9F70BF94E
:10737000364B187810FB07F025F026F80526AF23CA
:10738000019302460B4604940394029600952D48FF
:1073900014F0F8FB2346BC220D2112481CF038FFE4
:1073A0002B491048F9F7EFF8BC2301930494039498
:1073B0000296009500220023224814F0E3FB2346A6
:1073C000C9220D2107481CF023FF22490548F9F77F
:1073D000DAF8234622462D210220FAF7DFFCBCE131
:1073E0002988FF1F08C6FF1F6C260300D514030061
:1073F00030BBFF1F44BBFF1FF9150300CCBAFF1FB2
:10740000FE1503001CBBFF1F83150300A4BAFF1F5A
:1074100086150300B8BAFF1F11110300E0BAFF1F61
:1074200013110300F4BAFF1F0000394000005E4052
:10743000A916030008BBFF1F04160300091603006A
:10744000FC87FF1FB0BCFF1F151603003B88FF1F02
:1074500021160300291503003E88FF1F1288FF1F15
:10746000012940F07A81C14D2E78082E5ED8C04F98
:10747000963C17F816000094192378220021F9F79A
:1074800082F9BC4EA3B281B2192206F1640012F057
:1074900035F9FDF741FA2B78B74803EB430203EBCC
:1074A000820200240A232D328DE8180012B21E2316
:1074B0003F211DF05DFD2B78AF4803EB430203EB4A
:1074C00082022D3212B223463F211CF0A1FE2B78FE
:1074D000A94817F81310642359431AACF9F7FFF9B8
:1074E000A649B6F88080B6F88290B6F884A0B6F8BF
:1074F00086B0204621F00FFF2B7807EB4307A04B07
:107500007A7833F8123002934A465346414606F1E0
:1075100078000194CDF800B011F0FAFF204621F078
:10752000BAFE06F18C00F9F717FA88E0092E27D188
:10753000944E963C307800941923FF220021F9F7ED
:1075400022F9A3B281B219228F4812F0D7F8FDF7C1
:10755000E3F92B78884803EB430203EB8202002413
:107560000A232D328DE8180012B21E2367211DF068
:10757000FFFC307824F018FF0494039403234EE0BA
:107580000A2E21D1814F963C387800941923782215
:107590000021F9F7F8F8A3B281B219227A4812F063
:1075A000ADF8FDF7B9F92B787348009603EB430269
:1075B00003EB82022D32002401941E2312B26721B4
:1075C0001DF0D6FC387823E00B2E38D1704E963C57
:1075D00030780094192378220021F9F7D4F8A3B267
:1075E00081B21922684812F089F8FDF795F92B78D5
:1075F000614803EB430203EB82022D320A2300248D
:107600008DE8180012B21E2367211DF0B1FC3078FE
:107610006423584324F0D8FE049403940523029372
:107620002B7803EB430203EB82032D339BB20193D0
:107630006723009302460B46564814F0A3FA2B78B2
:107640000C2B40F08A804FF4D470F9F7E8F8494CDD
:107650005149B4F88060B4F88270B4F88480B4F80A
:10766000869001281AAD0CBF4FF01F0A4FF4FC6A38
:10767000284621F050FE3A4643463146CDF808A050
:10768000CDF8009004F17800019511F041FF2846F3
:1076900021F001FE4149B4F88690B4F88080B4F836
:1076A00084A0B4F8826016A821F035FE3C4B12A8E5
:1076B000197821F050FE12A916A821F03FFF4E4480
:1076C00003360146B6B20027284621F08EFE324628
:1076D00053464146CDF8009004F18C000297019585
:1076E00011F016FF284621F0D6FD12A821F0D3FD97
:1076F00016A821F0D0FDB4F89A30B4F89660B4F82A
:107700008080B4F88490B4F886A01E44254B12A85B
:10771000197821F020FE12A916A821F066FE224950
:1077200016A821F013FF03360146B6B2284621F011
:107730005CFE4B463246414604F1A000029701959B
:10774000CDF800A011F0E4FE284621F0A4FD16A813
:1077500021F0A1FD12A803F0AABF1448F9F7FCF824
:107760001348F9F7F9F804F04CB900BF94C5FF1FAE
:107770002988FF1FA4BAFF1F08C6FF1FFE150300BC
:107780001288FF1FFC87FF1F08BBFF1F3B88FF1FDE
:10779000368EFF1FB0BCFF1F2D16030037160300E7
:1077A000E88EFF1F23C4FF1F3D16030030BBFF1FE1
:1077B00044BBFF1F0A286FD100220C2044F208238B
:1077C00011468DE8090023B2AF481DF0D1FBFDF74B
:1077D000A3F8002303228221AB481CF019FDAB491A
:1077E000A948F8F7D0FEB8F80010A7480B2646F2D3
:1077F0002C3732392D23012209B28DE8C0001DF04B
:10780000B7FBB8F80040A2491E3C0525A4B21AA84F
:1078100021F081FD1AAB032221469E48009512F00B
:1078200039FF1AA821F037FDBBF1000F0CBF3B4612
:107830004FF478430122019329462E239248009663
:107840001DF096FB94491AA821F065FD1AAB03229E
:1078500019219048009512F01DFF1AA821F01BFD78
:10786000BBF1000F0CBF4FF478433B46012201935C
:1078700037212E23844800961DF07AFB87491AA8E9
:1078800021F049FD834800951AAB03224B2112F0E9
:1078900001FF1AA803F00BBF0B2804F0B2800C28DC
:1078A00040F0A68100267E4F01963B8876480D3B2E
:1078B0001BB20D220093314623B21DF059FB4FF647
:1078C000FF7171481BF0D1F901216F481BF0C7F916
:1078D00074496D481BF01EFA3346242205216A487C
:1078E0001CF096FC70496848F8F74DFE66481BF09E
:1078F0002BFA3A8864480A3A334612B205211AAC88
:107900001CF086FC69496048F8F73DFE08230A220E
:1079100067492046F8F7E6FD21465B4821F078FBF1
:10792000204621F0B8FC3A8857480A214FF47843A2
:107930000B3A12B28DE80A0016AD782331461BF0DF
:1079400061FC5C49284621F0E6FC40F29F10F8F704
:1079500066FF24F029FD02460B4600204FF08041CF
:1079600022F094F8544B002224F094FD25F08AF87C
:107970004FF0280801460222204621F052FD3C2308
:10798000912205214D48039602940195CDF800807F
:1079900011F063FE204621F07EFC284621F07BFC9E
:1079A0004749204621F0B7FC05213C232D224548BC
:1079B00002960194CDF8008011F0AAFD204621F036
:1079C0006AFC4FF4E570F8F72AFFBA463E493F4F8C
:1079D00048B1284621F09FFC3D49204621F09BFC00
:1079E0004FF4FC6308E0284621F095FC3849204616
:1079F00021F091FC46F22C335F2205210393CDF850
:107A000000803C2307F164000294019511F025FEEB
:107A1000204621F040FC284621F03DFC2D49284617
:107A200021F079FC2C49204621F075FC4FF0280804
:107A30004CF2186350215F220393284802943C23A0
:107A40000195CDF8008011F008FE204621F023FCBE
:107A5000284621F020FC4FF4D870F8F71CFF12AE36
:107A600083461F493046BBF1000F3FD021F053FC45
:107A70001C49284621F04FFC1B49204621F04BFCB5
:107A80004FF4FC6304933DE008C6FF1FE0140300BD
:107A900043160300B0BCFF1F131503004816030074
:107AA0003E88FF1F6C260300171503004F160300C6
:107AB00030C5FF1F6216030000405F40CCBAFF1FB5
:107AC0006C160300E0BAFF1F71160300A4BAFF1F73
:107AD00079160300C8150300981603001CBBFF1F8E
:107AE000EE180300CE190300AB1E030021F013FCB7
:107AF0003649284621F00FFC3549204621F00BFC81
:107B0000CDF810B03C239122502102950196CDF87A
:107B1000008003942F4811F03BFD204621F0BBFB71
:107B2000284621F0B8FB304621F0B5FB40F2191091
:107B3000F8F775FE2D239B220821FAF7B9FC264998
:107B4000204621F0E8FB002628235F2200939B219A
:107B50003C2302960194214811F0DAFC204621F0E2
:107B60009AFB4FF01A081E49204621F0D4FB6423EB
:107B70000E22494602960194CDF80080194811F072
:107B8000C7FC204621F087FBBAF8005016491A3D81
:107B9000ADB2204621F0BFFB2A4649466423029637
:107BA0000194CDF80080114811F0B2FC204621F07C
:107BB00072FBFDF761FAFB897989388919443246ED
:107BC000334689B2FAF7EAF803F01BBFCE19030077
:107BD0008116030030BBFF1F8A16030058BBFF1F2E
:107BE00083150300A4BAFF1F86150300B8BAFF1F50
:107BF0000D2840F00485FF2940F0DD83BC4D0024B2
:107C00002819143411F014FBB4F5027FF8D1B94BE4
:107C1000B94AB3F90030B948B94EBA4F00240194BB
:107C200012880D3A12B2009221460D221DF0A0F9E1
:107C300046F22C35032202238DE82C0005214FF457
:107C40009B738C22AD481DF0EBF94FF6FF71AB48EA
:107C50001BF00BF80121A9481BF001F8AA49A7481D
:107C60001BF058F8234624220521A4481CF0D0FA22
:107C7000A649A248F8F787FCA0481BF065F82946FA
:107C80009E481AF0F2FF3068716832890EAB03C368
:107C900001201A80F8F7C3FD3B7883420CD99C4B36
:107CA000A82202FB003000F110030EAA53F8060FC1
:107CB00059681B7A03C2137016AC1AAD4FF0000856
:107CC00094498DF84180204621F025FB0EA92846D5
:107CD00021F021FB28232D22052100938448CDF893
:107CE0000C803C230295019411F0B7FC284621F04A
:107CF000D2FA204621F0CFFA30687168327A0EABA2
:107D000003C303201A70F8F78AFD3B7883420CD92D
:107D10007F4BA82202FB003000F110030EAA53F89B
:107D2000060F59681B7A03C213704FF000087A4996
:107D30008DF84180204621F0EEFA0EA9284621F068
:107D4000EAFA28232D22502100937448CDF80C80A4
:107D50003C230295019411F080FC284621F09BFA07
:107D6000204621F098FA30687168327A0EAB03C36E
:107D700004201A70F8F753FD3B7883420CD9644B0A
:107D8000A82202FB003000F110030EAA53F8060FE0
:107D900059681B7A03C213704FF0000860498DF8D0
:107DA0004180204621F0B7FA0EA9284621F0B3FA07
:107DB00028232D229B2100935A48CDF80C803C2388
:107DC0000295019411F049FC284621F064FA2046FE
:107DD00021F061FA30687168327A0EAB03C3052076
:107DE0001A70F8F71CFD3B7883420CD9484BA82247
:107DF00002FB003000F110030EAA53F8060F596879
:107E00001B7A03C213704FF0000847498DF8418078
:107E1000204621F080FA0EA9284621F07CFA28237A
:107E20002D22E62100934148CDF80C803C23029599
:107E3000019411F012FC284621F02DFA204621F081
:107E40002AFA30687168327A0EAB03C306201A70C2
:107E5000F8F7E5FC3B7883420CD92D4BA82202FBB6
:107E6000003000F110030EAA53F8060F59681B7A70
:107E700003C2137000272E498DF84170204621F06F
:107E80004AFA0EA9284621F046FA039728273C23F0
:107E90005A220521274802950194009711F0DDFB35
:107EA000284621F0F8F9204621F0F5F9306871688C
:107EB000327A0EAB03C31A701F4B20491E78012E75
:107EC000204603D121F027FA1D4958E0022E03D1A4
:107ED00021F021FA1B4952E0032E03D121F01BFAB5
:107EE00019494CE0042E33D121F015FA174946E028
:107EF000A4BAFF1F0488FF1F3E88FF1F08C6FF1F8C
:107F0000A116030022C4FF1F6C2603009116030074
:107F10008890FF1F9D16030066160300CCBAFF1F52
:107F2000AB160300E0BAFF1FB2160300F4BAFF1F3E
:107F3000B9160300D0BBFF1F348DFF1FBE16030010
:107F4000CA160300CE160300D2160300D61603008D
:107F5000052E0FD121F0DFF9B349284621F0DBF9D6
:107F60004FF4FC6303930295019400973C239622FF
:107F7000314619E0062E08D121F0CDF9AB4928464B
:107F800021F0C9F94FF4FC6307E021F0C4F9A849D6
:107F9000284621F0C0F946F22C3303930295019450
:107FA00000973C2396220521A24811F056FB284653
:107FB00021F071F9204621F06EF99F4B9F491B7803
:107FC00012AE012B304607D121F0A5F99C4920467D
:107FD00021F0A1F99B4930E0022B07D121F09BF958
:107FE0009749204621F097F9974926E0032B07D1BE
:107FF00021F091F99249204621F08DF993491CE036
:10800000042B07D121F087F98D49204621F083F90F
:108010008F4912E0052B07D121F07DF988492046D0
:1080200021F079F9804908E0062B0CD121F073F991
:108030008349204621F06FF97C49284621F06BF9ED
:108040004FF4FC630BE021F066F97D49204621F0F6
:1080500062F97749284621F05EF946F22C33049301
:1080600028239622E62100937A4803953C23029424
:10807000019611F08DFA284621F00DF9204621F0E5
:108080000AF9304621F007F9734BDFF8E4911A78CA
:1080900099F80080FF2A4FF4CD709A464FF6E077AA
:1080A00018BF4FF4FC67F8F7BAFB804505D16B4960
:1080B000204621F030F963493EE040F29B10F8F78A
:1080C000AEFB804505D16549204621F024F95E4983
:1080D00032E04FF4CE70F8F7A2FB804505D15F493E
:1080E000204621F018F9594926E040F29D10F8F792
:1080F00096FB80455949204603D121F00CF954499B
:108100001AE0B8F1000F03D121F005F9464913E058
:10811000B8F1010F03D121F0FEF844490CE0B8F1A9
:10812000090F03D121F0F7F84D4905E0B8F10A0F26
:1081300007D121F0F0F84B49284621F0ECF80397DD
:1081400008E021F0E8F83A49284621F0E4F846F240
:108150002C33039328239622502100934248029502
:108160003C23019411F079FA284621F094F8204636
:1081700021F091F89AF8013099F80180FF2B4FF423
:10818000CD704FF6E07718BF4FF4FC67F8F747FB68
:10819000804505D13549204621F0BDF829493EE00A
:1081A00040F29B10F8F73BFB804505D12F49204654
:1081B00021F0B1F8244932E04FF4CE70F8F72FFBEC
:1081C000804505D12949204621F0A5F81F4926E020
:1081D00040F29D10F8F723FB80452449204603D147
:1081E00021F099F81A491AE0B8F1000F03D121F0F3
:1081F00092F80D4913E0B8F1010F03D121F08BF88B
:108200000A490CE0B8F1090F03D121F084F81449B0
:1082100005E0B8F10A0F2DD121F07DF8114928466B
:1082200021F079F803972EE01A12030016120300CA
:10823000E6180300B8BAFF1FE4C4FF1FDA160300F4
:10824000C3160300CA160300CE160300D21603009D
:10825000D61603006CBBFF1F3988FF1FE51603000D
:108260001E1203002212030094BBFF1FED16030031
:1082700069C7FF1F21F04FF86849284621F04BF8E5
:1082800046F22C33039328239B21962200936448C3
:1082900002953C23019411F0E0F9284620F0FBFF01
:1082A000204620F0F8FF5F4B5F491F78012F3046D2
:1082B00020D121F030F85D49204621F02CF85C49AE
:1082C000284621F028F84FF4FC63049328230093F8
:1082D0000395029401963C23C3220521554811F0D1
:1082E00057F9284620F0D7FF204620F0D4FF30462B
:1082F00003F0DDB9022F07D121F00DF84B492046DC
:1083000021F009F84C49DBE7032F07D121F003F8EE
:108310004649204620F0FFFF4849D1E7042F07D106
:1083200020F0F9FF4149204620F0F5FF4449C7E716
:10833000052F15D120F0EFFF3C49204620F0EBFF40
:108340004049284620F0E7FF4FF4FC6304932823BC
:1083500000930395029401963C23C3223946BDE75E
:10836000062F07D120F0D7FF3049204620F0D3FF59
:108370003549A5E7072F07D120F0CDFF2B4920462F
:1083800020F0C9FF31499BE7082F07D120F0C3FF38
:108390002649204620F0BFFF2D4991E720F0BBFF82
:1083A0002249204620F0B7FF1C49284620F0B3FFA1
:1083B00046F22C3389E72749274B0A781B78DFF8E8
:1083C0009C90501E9842884616D00AB9FF2B13D0B5
:1083D0009A4217D099F800108A4201D1FF2B11D090
:1083E000501C834213D08A4200D183B101398A42A2
:1083F00036D1FF2B34D10AE044F208252E464FF443
:10840000FC6731E044F208254FF4FC662BE044F2AF
:1084100008264FF4FC65374626E000BFE618030047
:10842000A8BBFF1F94C6FF1FF516030058120300D8
:10843000CA160300BCBBFF1FCE160300D2160300F2
:10844000D61603001A120300161203001E120300B0
:108450002212030094C5FF1FE08EFF1F22C4FF1FDE
:1084600044F208252E462F46DFF860A28A49BAF862
:1084700000B01AACABF11A0B204620F04CFF1FFAEB
:108480008BFB02971A275A463323372183480194DE
:10849000009711F03DF8204620F0FDFEBAF80020CC
:1084A0007F48113A002312B239211BF0B1FE98F82F
:1084B000001099F8003001390822C9B2204611F0A5
:1084C00083FD2146764820F0A3FD204620F0E3FE00
:1084D000BAF800B07049ABF11A0B1FFA8BFB2046BB
:1084E00020F019FF33235A46702102966D480194FB
:1084F000009711F00DF8204620F0CDFEBAF80020CC
:108500006748113A002312B273211BF081FE99F8DB
:10851000003098F800100822204611F055FD214641
:108520005F4820F075FD204620F0B5FEBAF80060E7
:1085300059491A3EB6B2204620F0EDFE32463323AA
:10854000A921029558480194009710F0E1FF2046B8
:1085500020F0A1FEBAF800205148113A002312B2CF
:10856000AC211BF055FE98F8001099F8003001314D
:108570000822C9B2204611F027FD2146484820F0C4
:1085800047FD204620F087FEBAF8005047491A3DC3
:108590000026ADB2204620F0BEFE2A4633233146E7
:1085A000434802960194009710F0B2FF204620F055
:1085B00072FEBAF800503F491A3DADB2204620F095
:1085C000AAFE2A463323E2213B48029601940097F3
:1085D00010F09EFF204620F05EFEBAF800503749AA
:1085E0001A3DADB2204620F096FE02960194009707
:1085F00027232A464FF48C71314801F09ABC142885
:1086000040F03984FF29DFF8C8804FF0000600F001
:1086100032812D22631F009201961BB2C3220521D5
:108620001F481CF0A5FC08EB0600143610F000FEF5
:10863000B6F5027FF7D12349234B0A781B78DFF880
:108640009490501E9842884615D00AB9FF2B12D03C
:108650009A4216D099F800108A4201D1FF2B10D00F
:10866000501C834212D08A4200D17BB1884233D160
:10867000FF2B31D10AE044F208252E464FF4FC6767
:108680002EE044F208254FF4FC6628E044F2082668
:108690004FF4FC65374623E0A916030008BBFF1F13
:1086A00008C6FF1F1CBBFF1F30BBFF1F11110300BB
:1086B00044BBFF1F1311030058BBFF1FF01303003F
:1086C00080BBFF1F94C5FF1FE08EFF1F3E88FF1F6A
:1086D000A4BAFF1F22C4FF1F44F208252E462F46CE
:1086E000DFF82CA3BF49BAF800B01AACABF11A0BF3
:1086F000204620F010FE1FFA8BFB02971A275A46DD
:1087000033233721B8480194009710F001FF204629
:1087100020F0C1FDBAF80020B448113A002312B28B
:1087200039211BF075FD98F8001099F800300139D7
:108730000822C9B2204611F047FC2146AB4820F080
:1087400067FC204620F0A7FDBAF800B0A549ABF1C0
:108750001A0B1FFA8BFB204620F0DDFD33235A460F
:1087600070210296A2480194009710F0D1FE204695
:1087700020F091FDBAF800209C48113A002312B273
:1087800073211BF045FD99F8003098F8001008227D
:10879000204611F019FC2146944820F039FC20466F
:1087A00020F079FDBAF800608E491A3EB6B2204634
:1087B00020F0B1FD32463323A92102958D48019462
:1087C000009710F0A5FE204620F065FDBAF80020C5
:1087D0008648113A002312B2AC211BF019FD98F81B
:1087E000001099F8003001310822C9B2204611F07A
:1087F000EBFB21467D4820F00BFC204620F04BFD92
:10880000BAF800507C491A3D0026ADB2204620F04F
:1088100082FD2A4633233146784802960194009718
:1088200010F076FE204620F036FDBAF8005074496C
:108830001A3DADB2204620F06EFD2A463323E221D8
:10884000704802960194009710F062FE204620F0D6
:1088500022FDBAF800506C491A3DADB2204620F016
:108860005AFD02960194009727232A464FF48C71F3
:10887000664801F05EBB664B01961B885B480D3B6A
:108880001BB20D220093314623B21CF071FB4FF650
:10889000FF7156481AF0E9F9012154481AF0DFF93E
:1088A0005C4952481AF036FA3346242205214F48D3
:1088B0001BF0AEFC58494D481AADF7F764FE4B4823
:1088C0001AF042FA5549284620F025FD544B16ACC3
:1088D000282719880A22204620F050FD2D223C230B
:1088E00005214046039602940195009710F0B5FECD
:1088F000204620F0D0FC284620F0CDFC49492846EF
:1089000020F009FD484B20461978F9F79FFE2D22EB
:108910003C23502108F1140003960294019500971E
:1089200010F09BFE204620F0B6FC284620F0B3FC59
:108930003E49284620F0EFFC3D4B2046197820F0B8
:108940000AFD2D223C239B2108EB0700039602948D
:108950000195009710F081FE204620F09CFC2846EF
:1089600020F099FC3349284620F0D5FC324B2046B4
:10897000197820F0F0FC3C2308EB03002D22E621BF
:10898000039602940195009710F067FE204620F0B0
:1089900082FC284620F07FFC284A1378012B914660
:1089A0000AD12749204620F0B6FC2649284620F067
:1089B000B2FC4FF4FC6355E0032B05D1204920465F
:1089C00020F0A9FC204906E0042B41D11F49204694
:1089D00020F0A1FC1B49284620F09DFC40F2FF73CB
:1089E00040E000BFA91603006CBBFF1F08C6FF1FB5
:1089F00080BBFF1F94BBFF1F11110300A8BBFF1F0B
:108A000013110300BCBBFF1FF0130300D0BBFF1FFB
:108A10003E88FF1F6C260300FB16030009170300A6
:108A2000E6C4FF1F1317030094BAFF1F18170300B3
:108A300088BAFF1F2317030096C9FF1F64C5FF1FD5
:108A40002E170300D4180300351703007415030014
:108A5000A749204620F05FFCA649284620F05BFC91
:108A60004FF6E0735A220521039308F150003C238E
:108A700002950194009710F0F0FD284620F00BFCC1
:108A8000204620F008FC9C4B1E7876B9314640F217
:108A9000CF10F7F757FE9949204620F03CFC954946
:108AA000284620F038FC03960FE0012140F2CF1059
:108AB000F7F748FE9149204620F02DFC90492846C2
:108AC00020F029FC4FF4FC63039328235A22502101
:108AD00000938C4802953C23019410F0BEFD28467B
:108AE00020F0D9FB204620F0D6FB99F80030032B6C
:108AF00040F081808449204620F00DFC0027282684
:108B00008249284620F007FC3C235A229B218048BA
:108B1000039702950194009610F09FFD284620F0DF
:108B2000BAFB204620F0B7FB7A49284620F0F3FB39
:108B3000794B0A221988204620F020FC3C2387220A
:108B400005217648039702940195009610F085FD63
:108B5000204620F0A0FB284620F09DFB70492846C7
:108B600020F0D9FB6F4B0A221988204620F006FC22
:108B70003C23872250216C4803970294019500966C
:108B800010F06BFD204620F086FB284620F083FB8A
:108B90006649284620F0BFFB654B0A22198820460B
:108BA00020F0ECFB3C2387229B2162480397029430
:108BB0000195009610F051FD204620F06CFB2846F0
:108BC00020F069FB5C49284620F0A5FB5B4B0A229C
:108BD0001988204620F0D2FB3C238722E621584802
:108BE000039702940195009610F037FD204620F07F
:108BF00052FB284617E05349204620F08CFB52498F
:108C0000284620F088FB00230393282300935A2250
:108C10003C239B213E480295019410F01EFD2846FE
:108C200020F039FB204620F036FB4849484F2046CB
:108C300020F071FB0026444928464FF0280820F018
:108C40006AFB3C235A22E62103964248029501948E
:108C5000CDF8008010F001FD284620F01CFB2046D6
:108C600020F019FB46F22C390A234FF0030B8DE854
:108C70000808B6224FF49B7305213748CDF80890B9
:108C80001CF0CEF93346B7222D2133481BF0C0FA31
:108C9000FBF742FE31493048F7F775FC0722B72150
:108CA0002520FAF7E1FAB721FA200722FAF7DCFAD1
:108CB0003E782B492046002E58D020F02CFB294925
:108CC000284620F028FB4FF4FC630393C7223C2383
:108CD000052102950194CDF80080234810F0BDFCD9
:108CE000284620F0D8FA204620F0D5FA5CE000BFF4
:108CF0002E170300E618030020C4FF1F39170300D6
:108D0000D418030008BBFF1F401703006E150300B3
:108D1000E4BBFF1F7614030062C5FF1F0CBCFF1FDE
:108D200076150300368DFF1F20BCFF1F331A03008A
:108D3000DCD4FF1F34BCFF1F4717030054C6FF1FBE
:108D400048BCFF1F531703001E4503005B170300B9
:108D5000A4C5FF1FF8BBFF1F08C6FF1F6217030053
:108D600092170300AB1E03001CBBFF1F20F0D3FAB9
:108D7000BC49284620F0CFFA3C23C7220521BA4837
:108D8000CDF80C9002950194CDF8008010F065FCB0
:108D9000284620F080FA204620F07DFA31464FF434
:108DA000E870F7F7CFFC3E70B049284620F0B3FAE0
:108DB000AF4B20461978F9F749FC00262823C72233
:108DC00050210093AB4803963C230294019510F088
:108DD00044FC204620F05FFA284620F05CFAA64AC0
:108DE00051681068128912AB03C3A4491A80A44BBE
:108DF00009781A78914202D2FF221A700DE0A14B35
:108E0000A82101FB0233103312AA53F8060F596848
:108E10001B7A03C213708DF851609B49204620F0E5
:108E20007AFA002712A92826284620F074FA3C2353
:108E3000C7229B219548039702950194009610F054
:108E40000CFC284620F027FA204620F024FA90490E
:108E5000204620F060FA8F4B02221968284620F045
:108E6000E0FA03970295019400963C23C722E6217D
:108E7000894802F070B8162840F08E82FF294FF022
:108E8000000440F04581854D2819143410F0D0F9C4
:108E9000B4F5027FF8D10A240025C02601944FF4CE
:108EA0009B73302205217E48029500961CF0B8F88D
:108EB0004CF218633022029301944FF49B73052106
:108EC000774800961AF0C0FE4FF6FF71744819F00B
:108ED000CCFE0121724819F0C2FE7249704819F0A7
:108EE00019FF2B464A2221466D486F4C1BF090F922
:108EF0006E496B48F7F747FB694819F025FF0221D7
:108F0000674819F005FE2378694AD25C5B4B1B78F1
:108F10009A424ED227262378DFF89491217822783E
:108F2000584F19F80110DBB20793237819F8033072
:108F30004FF0A80808FB037308FB017193F815A014
:108F400019F8023008FB0373D3E91223D1E91601A3
:108F500023F0ECF80022574B23F0C6FBCDE90801C3
:108F6000284623F031FA02460B46DDE9080123F0DA
:108F700091FA079B19F8033008FB0377D7E912230E
:108F800023F0D6F823F07EFD1AAB524601211DF0E6
:108F900001FF32B200231A2141481BF039F9013593
:108FA0001AA93F48F7F7EFFA18360B2DB6B2B2D12F
:108FB00005E02078FF2100F5F770F7F7C3FB0321E8
:108FC0003748DFF80481DFF8B490DFF800A119F02A
:108FD0009FFD46F22C31324819F047FE00236522EE
:108FE0000C212F481BF014F933492D48F7F7CBFA21
:108FF00000237A2210212A481BF00AF92F49284819
:10900000F7F7C1FA00238F221E2125481BF000F933
:1090100000212348F7F763FC0023A32210212048F6
:109020001BF0F6F826491E48F7F7ADFA0023B722E1
:109030000C211B481BF0ECF822491948F7F7A3FA5A
:1090400007250024184B1A78E3B29A4208D198F801
:10905000013099F800209A423AD98AF8003037E076
:10906000002737E0811603001CBBFF1F1317030006
:10907000D88EFF1F30BBFF1FA116030022C4FF1FA5
:10908000BCC9FF1F8890FF1FC815030044BBFF1F0A
:10909000D215030064C7FF1F58BBFF1FA4BAFF1FF0
:1090A00008C6FF1F6C26030096C6FF1F9A17030011
:1090B000C88EFF1F00002440AC170300B217030046
:1090C000B7170300BC170300C78EFF1F94C5FF1F0F
:1090D0004FF4FC671AAE99F8003018F8011F0A2205
:1090E000304610F071FF9F4A142303FB04202946E9
:1090F0008DE8C8004D223A233C3010F009FA0134C3
:10910000304620F0C8F83E35052CADB29AD108E0C3
:109110005C2300930194F8236422272192481BF0DA
:1091200027FF672441F2A20522B215340095F123EE
:109130002A218D48A4B21CF07DF8D02CF4D12A2429
:1091400041F2A20521B218340095542368228648C2
:10915000A4B21CF011F8B4F5997FF3D1834C844E7E
:109160002378844DF25C2B789A4206D3BBF10B0F27
:10917000DFF820825FD902F0B8BA22787E4F0B2345
:109180005A434FF00B08BA56642AC1BF22785343A2
:109190000022FA54237808FB03F34FF02A09FA5609
:1091A0006FF0530364325A43C92392FBF3F2BC328B
:1091B00092B24FF0010A237808FB037313F90A30C7
:1091C000642B02F38A82694B6B491B7808FB0313FB
:1091D00013F90A306433C2F28082237808FB0373E8
:1091E0006FF0530113F90A3064334B43C92193FBE9
:1091F000F1F3BC33662B03DDBC2BA8BFBC2300E01E
:10920000672399B207910FFA89F109F118091FFA3A
:1092100089F94FF478401BB20190009312B20FFA13
:1092200089F3514819F0AEFFB9F58D7F0AF1010AB3
:109230009CD0079ABFE723784C4FF25C2B789A4278
:1092400082F053823B784C4C47480B2505FB034387
:109250000BEB4B0113F90B206FF0530364324FF407
:1092600078465A43C900C92392FBF3F2BC320096F8
:10927000032312B22A311AF07DFC4FF00309029643
:10928000152632233522F92137488DE840021BF09C
:10929000C7FE4FF6FF71344819F0E7FC37493248F2
:1092A00019F038FD4A220023FA212F481AF0B0FFA6
:1092B0003B782D4805FB03441AAD14F90B10F7F762
:1092C0000EFB294819F040FD00242D49284624278B
:1092D00020F021F8182364224FF49371019521485E
:1092E0000294009710F014F928461FF0D4FF254986
:1092F000284620F010F81823CC224FF493710195E2
:1093000021480294009710F003F928461FF0C3FF8C
:109310001E4928461FF0FFFF3C238C224FF4937117
:10932000019500931A480294182310F0F1F828468A
:109330001FF0B1FFB8F800200B480294183A8DE8EE
:1093400040024FF48A7312B211211BF069FE054DE1
:1093500004F1C800284414340FF06AFF642CF7D1DC
:1093600002F04FBBA4BAFF1F08C6FF1F96C6FF1F1F
:10937000C88EFF1F22C4FF1F57C6FF1F6C260300A5
:109380008315030086150300B8BAFF1FE717030013
:10939000CCBAFF1F3E88FF1F182840F06283FF29C8
:1093A0004FF0000440F08281B24D281914340FF0C0
:1093B0003FFFB4F5027FF8D10024AC250A2640F225
:1093C0002B1330221421AC4802948DE860001BF06E
:1093D00027FE4CF2186330220293142140F22B1323
:1093E000A5488DE860001AF02FFC4FF6FF71A248E7
:1093F00019F03BFC0121A04819F031FC9F499E481F
:1094000019F088FC23464A2219219B481AF000FFD4
:109410009B499948F7F7B7F89A4A9B4910780B7817
:109420000891984292460BD211781AA8082210F09F
:10943000CBFD1AA990481FF0EBFD1AA81FF02BFFD7
:109440008D4819F081FC02218B4819F061FB002343
:109450001A22582188481AF0DBFE8C498648F7F713
:1094600092F827270026089A9AF800301278DFF839
:1094700014829A4240F2C58000233AB216217E48F7
:10948000834C1AF0C5FE98F80030A82505FB03436D
:109490005B7D8BBB98F8001098F8003098F800209E
:1094A00005FB014105FB0343D2B20792D1E9160146
:1094B000D3E9122322F03AFE0022764B23F014F96E
:1094C00080463046894622F07FFF02460B464046E2
:1094D000494622F0DFFF079B05FB0344D4E9122332
:1094E00022F026FE23F0CEFA23F006FE6A4902B2ED
:1094F0001AA824F06FF980E098F8003098F800106E
:1095000005FB034305FB01415B7D012B98F800300F
:1095100098F8002005FB0343D2B20792D1E9160167
:10952000D3E9122333D122F001FE0022594B23F05C
:10953000DBF880463046894622F046FF02460B465D
:109540004046494622F0A6FF079B05FB0344D4E9A9
:10955000122322F0EDFD23F095FA0021054623F0B9
:109560008DFD10B105F1004000E028464B4923F085
:10957000E7FB23F0C1FD0A2390FBF3F404FB130483
:10958000284623F0B9FD234602B2454932E022F0D5
:10959000CDFD00223F4B23F0A7F880463046894698
:1095A00022F012FF02460B464046494622F072FF67
:1095B000079B05FB0344D4E9122322F0B9FD23F0F5
:1095C00061FA0021054623F059FD10B105F1004074
:1095D00000E02846334923F0B3FB23F08DFD6423DC
:1095E00090FBF3F404FB1304284623F085FD2E4979
:1095F000234602B21AA824F0EDF81AA91E48F6F77D
:10960000C2FF013618370B2EBFB27FF42CAF0321F7
:10961000194819F07DFA46F22C31174819F025FB4C
:1096200000234D22172114481AF0F2FD642112483C
:10963000F7F755F9002362221A210F481AF0E8FDC6
:1096400050210D48F7F74BF90023A4221A210A48AC
:109650001AF0DEFD14210848F7F741F90023BA2279
:10966000202105481AF0D4FD00210348F7F737F907
:1096700025E000BFA4BAFF1F08C6FF1F6C26030029
:10968000C217030021C4FF1F22C4FF1FCE1703000F
:109690008890FF1F00002440634503000000204124
:1096A000D51703000000C842DE170300752300939E
:1096B0000194F8234D2227219A481BF059FC50248D
:1096C00041F2A20522B216340095F1232A219548D1
:1096D000A4B21BF0AFFDD42CF4D12A2441F2A20590
:1096E00021B2183400956D2351228E48A4B21BF08C
:1096F00043FDB4F5997FF3D18B4D2E46502716F8D4
:10970000010B0097BE2364220021F7F73CF82A24BE
:109710001FFA80F916F8010B0097BE23642200217E
:10972000F7F731F880B24F2803DDBE28A8BFBE206E
:1097300000E0502021B21834A4B21FFA80FA4FF48E
:10974000784800B20090CDF8048023B20FFA89F275
:10975000744819F017FDB4F58D7F01D0D146D9E7D3
:10976000ABF16503DBB2992B00F2FA806F4B0BF182
:109770003807FFB21B787A1E9A4216D00FB9FF2B1A
:1097800013D09F4217D06A4A1278974201D1FF2B1B
:1097900011D0791C8B4213D0974200D183B1013A8A
:1097A000974213D1FF2B11D10AE044F20824264638
:1097B0004FF4FC690EE044F208244FF4FC6608E024
:1097C00044F208264FF4FC64B14603E044F2082456
:1097D0002646A146DFF88481B8F800201920052329
:1097E0000025303A8DE8290012B2DB234F214D4885
:1097F0001BF016FC4FF0030C4FF0000E94238DE885
:1098000008503C2218234FF4937146481BF008FC83
:10981000B8F800A0464B1AAD0BF137011B780822AF
:10982000C9B22846AAF1300A10F0CEFB1FFA8AFA14
:10983000CDF808904FF01A09524633234F213D4886
:109840000195CDF800900FF063FE28461FF023FD30
:10985000B8F800A0364BAAF1300A1B780822394626
:1098600028461FFA8AFA10F0AFFB332352468721AD
:10987000029631480195CDF800900FF049FE284638
:109880001FF009FDB8F80060294B303E0BF139019B
:109890001B780822C9B22846B6B210F095FB3323D4
:1098A0003246BF21029425480195CDF800900FF073
:1098B0002FFE28461FF0EFFCB8F800402049303C4E
:1098C00028461FF028FDA4B2002322461721029348
:1098D0001C4801953323CDF800900FF019FE28465F
:1098E0001FF0D9FCB8F800401749303C28461FF05B
:1098F00012FDA4B200232246F721029313480195DA
:109900003323CDF800900FF003FE28461FF0C3FC70
:109910000F480FF08DFC0F480FF08AFC0E4800F046
:10992000BCBD00BF08C6FF1F78C5FF1FE08EFF1F2C
:1099300022C4FF1F08BBFF1F1CBBFF1F30BBFF1F44
:109940001111030044BBFF1F1311030058BBFF1F7D
:10995000A4BAFF1FB8BAFF1FCCBAFF1F3E88FF1F73
:10996000BBF1C70F02F24D80502315F80B00009396
:109970006422BE230021F6F706FF0BEB4B01C90062
:1099800002B203232A31C048CDF800801AF0F2F861
:109990001521032335228DE80A00BB48CDF8088045
:1099A0002A23F9211BF03CFB4FF6FF71B64819F052
:1099B0005CF9B649B44819F0ADF900234A22FA21FE
:1099C000B1481AF025FC15F80B10AF481AACF6F7A1
:1099D00082FFAD4819F0B8F90025AD49242620468C
:1099E0001FF099FC18233C224FF49371A94802956B
:1099F000019400960FF08CFD20461FF04CFCA64908
:109A000020461FF088FC1823AC224FF49371A34822
:109A10000295019400960FF07BFD20461FF03BFC61
:109A20009F4920461FF077FC442364224FF4937132
:109A300000939C480295182301940FF069FD20467D
:109A40001FF029FC98480FF0F3FB98480FF0F0FB4B
:109A500097480FF0EDFB97480FF0EAFB964800F0AF
:109A60001CBD152840F08882FF294FF0000440F00B
:109A70006781884D281914340FF0DAFBB4F5027FA2
:109A8000F8D1AC240A25002640F22B1330221421F1
:109A90007D488DE870001BF0C3FA4CF21863302249
:109AA0000293142140F22B1377488DE830001AF00E
:109AB000CBF84FF6FF71744819F0D7F801217248BE
:109AC00019F0CDF87149704819F024F933464A224B
:109AD00019216D481AF09CFB784916A81FF01BFC51
:109AE000774B1A78032A9A4617D176496648F6F7D3
:109AF0004AFD754B75491B78097832461AA810F053
:109B000063FA1AA960481FF083FA1AA81FF0C3FB72
:109B10006F4916A81FF07CFC03E06E495A48F6F71F
:109B200032FD594819F010F90221574818F0F0FF9A
:109B300000231A22532154481AF06AFB16A95248EE
:109B40001FF066FA272500272AB2002316214E4867
:109B5000614E1AF05DFB0120F6F761FEA82404FBBC
:109B6000006000225D4BD0E9160122F0BDFD804669
:109B70003846894622F028FC02460B4640464946B4
:109B800022F088FC22F05EFF013781B23E48F6F7F2
:109B9000A6FE18350B2FADB2D6D103213A4818F0E6
:109BA000B7FF46F22C31384819F05FF89AF80030C8
:109BB000032B4FF04D024FF0000340F09780434FCE
:109BC00031481A211AF024FB3B782F48012504FB69
:109BD00003630095D3E91623F6F787FE002362227C
:109BE0001A2129481AF014FB397804FB0161D1E9E4
:109BF0001289D1E9160142464B4622F097FA00221B
:109C0000374B22F047FC0022364B22F06DFD4246D6
:109C10004B4622F08DFA009502460B461A48F6F79D
:109C200064FE0023A4221A2117481AF0F1FA3978A9
:109C300004FB0161D1E91289D1E9160142464B4684
:109C400022F074FA0022284B22F024FC0022254B3B
:109C500022F04AFD42464B4622F06AFA009502463F
:109C60000B460948F6F741FE0023BA221A2106489E
:109C70001AF0CEFA3B78009504FB0364D4E9122372
:109C80000148F6F732FE57E008C6FF1F6C260300B6
:109C900083150300A4BAFF1F86150300B8BAFF1F7F
:109CA000E7170300CCBAFF1F08BBFF1F1CBBFF1F39
:109CB00030BBFF1F44BBFF1F58BBFF1FEA17030049
:109CC00064C5FF1FF417030022C4FF1FFE87FF1F98
:109CD00040170300021803008890FF1F0000244073
:109CE00000005440000059400000344017219648BD
:109CF0001AF08EFA64219448F6F7F1FD00236222EF
:109D00001A2191481AF084FA50218F48F6F7E7FD9E
:109D10000023A4221A218C481AF07AFA14218A48C6
:109D2000F6F7DDFD202188480023BA221AF070FAE8
:109D300000218548F6F7D3FD16A81FF0ACFA08E01D
:109D4000752300930194F8234D2227217E481BF0B0
:109D50000FF9502441F2A20522B216340095F123E6
:109D60002A217948A4B21BF065FAD42CF4D12A2414
:109D700041F2A20521B2183400956D235122724898
:109D8000A4B21BF0F9F9B4F5997FF3D16F4B704D84
:109D90001A7807932E46032A16F8012B6FF06C07EA
:109DA00014BF4FF065094FF480797A4392FBF9F2C2
:109DB000BE3292B22A2416F8013B7B4393FBF9F39F
:109DC000BE339BB24F2B03DDBE2BA8BFBE2300E0EA
:109DD000502321B21834A4B21FFA83FA4FF4784802
:109DE0001BB20093CDF8048023B212B2564819F08A
:109DF000C9F9B4F58D7F01D05246DCE7BBF1FF0F06
:109E000001F0FF8515F80B204F48CDF800806FF06A
:109E10006C030BEB4B015A43C90092FBF9F2BE32C3
:109E2000032312B22A3119F0A5FE152203238DE86F
:109E30000C00EF21342335224348CDF808801BF075
:109E4000EFF84FF6FF71404818F00FFF41493E48C8
:109E500018F060FF00234A22F0213B481AF0D8F99D
:109E6000079B15F80B401B78032B29D13A4B3B4A33
:109E70001B78A82101FB0321D1E91267D1E9160162
:109E800032463B4622F052F980462046894622F06F
:109E90008BFA02460B464046494622F0FBFA28A3BD
:109EA000D3E9002322F020FC32463B4622F040F961
:109EB0000223009302460B462348F6F716FD03E003
:109EC00021462148F6F707FD1AAC1F4818F03CFF61
:109ED00000252349242620461FF01DFA18233C2282
:109EE0004FF493711F480295019400960FF010FBF8
:109EF00020461FF0D0F91C4920461FF00CFA182309
:109F0000AC224FF4937119480295019400960FF01A
:109F1000FFFA20461FF0BFF9154920461FF0FBF954
:109F200044231448009302950194182364224FF4AB
:109F300093710FF0EDFA01F0B9BB00BFAFF30080F1
:109F40000000000000E06F4008C6FF1F64C5FF1F4F
:109F5000B9C4FF1F6C260300FE87FF1F8890FF1FF8
:109F600083150300A4BAFF1F86150300B8BAFF1FAC
:109F7000E7170300CCBAFF1F172840F0E480A04D7C
:109F80000024281914340FF053F9B4F5027FF8D1E6
:109F90000026AC240A258DE8700040F22B133022F5
:109FA00014219848DFF8B4821BF03AF84CF2186399
:109FB00030228DE830000293142140F22B13914897
:109FC00019F042FE4FF6FF718E4818F04EFE012147
:109FD0008C4818F044FE8C498A4818F09BFE3346A2
:109FE0004A22192187481AF013F988498548F6F75B
:109FF000CAFA844818F0A8FE3346BE2219218148C7
:10A000001AF006F982497F48F6F7BDFA3346CB22AB
:10A0100019217C481AAC1AF0FBF87E49794816AD34
:10A02000F6F7B1FA7C4920461FF075F9282798F811
:10A03000001028461FF08FF93C234D22192170484B
:10A0400003960295019400970FF007FB28461FF036
:10A0500022F920461FF01FF9704920461FF05BF9D6
:10A0600098F8011028461FF076F93C234D2269210B
:10A070006B4803960295019400970FF0EEFA28467C
:10A080001FF009F920461FF006F9664920461FF027
:10A0900042F998F8021028461FF05DF93C234D2242
:10A0A000B921614803960295019400970FF0D5FA03
:10A0B00028461FF0F0F820461FF0EDF85B492046D7
:10A0C0001FF029F998F8031028461FF044F93C23A3
:10A0D0007F221921564803960295019400970FF0AC
:10A0E000BCFA28461FF0D7F820461FF0D4F8514993
:10A0F00020461FF010F998F8041028461FF02BF99D
:10A100003C237F2269214C480396029501940097D5
:10A110000FF0A3FA28461FF0BEF820461FF0BBF848
:10A12000464920461FF0F7F898F8051028461FF01A
:10A1300012F903960295019400973C237F22B921DE
:10A140003F4800F008BF0E2840F0EE820026FF29AD
:10A150003C4FDFF80C9101961AAD40F0A2813B888C
:10A1600028480D3B1BB20D223146009323B21AF052
:10A17000FFFE4FF6FF71234818F077FD01212148BB
:10A1800018F06DFD20491F4818F0C4FD3346242205
:10A1900005211C481AF03CF82B491A48F6F7F3F948
:10A1A00016AC184818F0D0FD284920461FF0B3F827
:10A1B000254928461FF0AFF828232D225021039669
:10A1C0000093234802953C2301940FF046FA284659
:10A1D0001FF061F820461FF05EF840F2AB10F6F772
:10A1E0001EFB1C4B1C4E187019781A46002901F0F2
:10A1F00075833378022B41F0C18301F06FBB00BF40
:10A20000A4BAFF1F08C6FF1F6C2603001518030021
:10A2100026180300531803006E1803007418030077
:10A22000B8BAFF1F7A180300CCBAFF1F80180300CA
:10A23000E0BAFF1F86180300F4BAFF1F8C18030052
:10A2400008BBFF1F3E88FF1F67150300531703005D
:10A250006CBBFF1F7990FF1F5BC7FF1FD4D4FF1F8C
:10A2600022C4FF1F1F78FFB2052F41F0A283A84927
:10A2700028461FF050F84FF4FC6302932823009304
:10A2800001953C232D223946A2480FF041F928467A
:10A290001FF001F84FF0000828279F4928461FF0BB
:10A2A0003AF83C235F2205219C48CDF808800195AF
:10A2B00000970FF02DF928461EF0EDFF984928462B
:10A2C0001FF029F83C235F2250219648CDF80880E2
:10A2D000019500970FF01CF928461EF0DCFF92490B
:10A2E00028461FF018F83C23912205218F48CDF80D
:10A2F0000880019500970FF00BF928461EF0CBFF60
:10A300008B4928461FF007F83C23502191228948A9
:10A31000CDF80880019500970FF0FAF828461EF056
:10A32000BAFF337884497D4E022B204641F0F182FA
:10A330001EF0F1FF814928461EF0EDFF4CF2186334
:10A34000C3220521039306F1F0003C2302950194FA
:10A3500000970FF082F928461EF09DFF20461EF060
:10A360009AFF774B1B78002B41F0E9827549204614
:10A370001EF0D1FF744928461EF0CDFF4CF2186341
:10A3800003932823C3225021019400936F48029520
:10A390003C230FF062F928461EF07DFF20466C4CEE
:10A3A0001EF079FF99F800302178092228460FF035
:10A3B0000BFE05237A22009323212B46654810F0DB
:10A3C00069F928461EF067FF227899F800309A4212
:10A3D00019D2F28BB18B60481B32193112B20023B3
:10A3E00009B219F015FF5D4B186821F0FFFF2278C4
:10A3F0005B4BA82707FB023302465B7D0093564860
:10A400000B46F6F772FA99F800306178092228466F
:10A410000FF0DAFD0523AC22009323212B464D4893
:10A4200010F038F928461EF036FF627899F80030AF
:10A430009A421CD2B6F84620B6F8441046481B3261
:10A44000193112B2002309B219F0E2FE434B5868E9
:10A4500021F0CCFF3E4B5A78414BA82404FB023339
:10A4600002465B7D00933C480B46F6F73EFA6420BB
:10A47000FAF7F6FB3B4B3C4801221A700EF0D8FE6F
:10A480003A480EF0D5FE3A480EF0D2FE39480EF0AA
:10A49000CFFE39480EF0CCFE38480EF0C9FE01F070
:10A4A000B0BA28230093C3229A2305212A481AF020
:10A4B0005FFD334B1A78334B1B78511E994215D0F0
:10A4C0000AB9FF2B12D09A4216D099F800108A428E
:10A4D00001D1FF2B10D0501C834212D08A4200D1F0
:10A4E0007BB1884250D1FF2B4ED10AE044F20824C0
:10A4F00026464FF4FC684BE044F208244FF4FC6617
:10A5000045E044F208264FF4FC64B04640E000BF4A
:10A51000A8180300F4BAFF1FC6180300A4BAFF1F4F
:10A52000CF180300B8BAFF1FD7180300CCBAFF1F1B
:10A53000E1180300E0BAFF1F2E170300B21B03004F
:10A540008ABAFF1FEA180300F2180300A8BBFF1F16
:10A550002688FF1FB0BCFF1F08C6FF1F8CC5FF1F4A
:10A560008890FF1F3C88FF1F08BBFF1F1CBBFF1FFD
:10A5700030BBFF1F44BBFF1F58BBFF1F80BBFF1F2B
:10A5800094C5FF1FE08EFF1F44F208242646A04614
:10A59000B7F800A08D492846AAF11A0A1EF0BBFEA2
:10A5A0001FFA8AFACDF808804FF01A085246332372
:10A5B00037210195CDF800808548DFF85CA20EF0C8
:10A5C000A7FF28461EF067FE3A888248113A00230A
:10A5D00012B2392119F01CFE9AF8001099F80030D7
:10A5E000013908222846C9B20FF0EEFC2946794805
:10A5F0001EF00EFD28461EF04EFEB7F800B073495F
:10A60000ABF11A0B1FFA8BFB28461EF084FE5A464C
:10A610000296332370210195CDF800806E480EF02C
:10A6200077FF28461EF037FE3A886A48113A002321
:10A6300012B2732119F0ECFD99F800309AF800106D
:10A64000082228460FF0C0FC294662481EF0E0FCB4
:10A6500028461EF020FE3E885C491A3EB6B22846C7
:10A660001EF059FE324602943323A9210195CDF8FC
:10A6700000805A480EF04CFF28461EF00CFE3A8827
:10A680005448113A002312B2AC2119F0C1FD9AF8D6
:10A69000001099F80030013108222846C9B20FF0A5
:10A6A00093FC29464B481EF0B3FC28461EF0F3FDF0
:10A6B0003C884B491A3C0026A4B228461EF02BFECB
:10A6C00022463323314602960195CDF80080454855
:10A6D0000EF01EFF28461EF0DEFD3C8842491A3C63
:10A6E000A4B228461EF017FE22463323E22102962A
:10A6F0000195CDF800803D480EF00AFF28461EF077
:10A70000CAFD3C883A491A3CA4B228461EF003FE12
:10A7100002960195CDF80080272322464FF48C71D4
:10A7200034480EF0F5FE1BE1102840F0EF81FD29C2
:10A7300040F21981FF2926D100252F4B01951B8856
:10A7400024480D3B1BB20D220093294623B21AF078
:10A750000FFC4FF6FF711F4818F087FA01211D48C2
:10A7600018F07DFA25491B4818F0D4FA2B4624220C
:10A770000521184819F04CFD21491648F5F703FF4B
:10A78000144818F0E1FA40F21B10F6F748F81AAC3A
:10A790000A2843D8DFE800F0060D0F11424242427A
:10A7A00042421300174920461EF0B5FD46F22C33F5
:10A7B0003AE0154904E0154902E0154900E0154961
:10A7C00020461EF0A8FD4FF4FC632DE0A9160300FF
:10A7D00008BBFF1F08C6FF1F1CBBFF1F30BBFF1FAE
:10A7E0001111030044BBFF1F1311030058BBFF1FCF
:10A7F000F013030080BBFF1F3E88FF1F6C26030081
:10A8000037150300E6180300401503004515030043
:10A810004B1503005F15030094C5FF1FA449204694
:10A820001EF079FD4FF6E073029328232D220521B7
:10A830000093A04801943C2316AD0EF069FE20461B
:10A840001EF029FD9C4928461EF065FD002728269C
:10A850009A4920461EF05FFD3C235F22052198485F
:10A8600003970294019500960EF0F7FE20461EF025
:10A8700012FD28461EF00FFD924928461EF04BFDA2
:10A88000914920461EF047FD3C23912205218F4827
:10A8900003970294019500960EF0DFFE20461EF00D
:10A8A000FAFC28461EF0F7FC894928461EF033FDC5
:10A8B000854920461EF02FFD05213C23C3228548F3
:10A8C00003970294019500960EF0C7FE20461EF0F5
:10A8D000E2FC28461EF0DFFC4FF4D770F5F79FFF2F
:10A8E0007D4948B928461EF016FD7C4920461EF0D9
:10A8F00012FD46F22C3308E028461EF00CFD774985
:10A9000020461EF008FD4FF4FC63C322642103932C
:10A91000734802943C23019500960EF09EFE20465B
:10A920001EF0B9FC28461EF0B6FC6E4928461EF003
:10A93000F2FC4FF48A70F5F772FF014620461EF0D4
:10A940000AFD00230393282300936748029401958E
:10A950003C23C3229B210EF080FE20461EF09BFC70
:10A96000284600F0A4BE002944D1604B0A4643F8B3
:10A970002B200BF1010BBBF1080F4FF00004F6D1B7
:10A98000C823272250215A4800930194DC231AF04F
:10A99000EFFAF9F7C1FF234628228C21544819F019
:10A9A00037FC54495248F5F7EEFD234632228C21FC
:10A9B0004F4819F02DFC50494D48F5F7E4FD3E494C
:10A9C00016A81EF0A8FC3D491AA81EF0A4FC1F23DF
:10A9D0001AAA16A93A480EF0F7FC1AA81EF05BFC5A
:10A9E00016A81EF058FC454B14221A70444B1C70DC
:10A9F00001F007B801292DD100233C4A194642F83D
:10AA000023100133082B4FF00004F8D1C82327226C
:10AA10005021374800930194DC231AF0A9FAF9F782
:10AA20007BFF284916A81EF076FC27491AA81EF0BD
:10AA300072FC23461AAA16A924480EF0C5FC1AA8CF
:10AA40001EF029FC16A81EF026FC284B02221A61D3
:10AA500000F0D7BF022940F0D487244B2448196165
:10AA60000024C823272250218DE81800DC231AF087
:10AA70007FFAF9F751FF164916A81EF04CFC12494F
:10AA80001AA81EF048FC23461AAA16A911480EF06F
:10AA90009BFC1AA81EF0FFFB16A81EF0FCFB194B2E
:10AAA0001B681A93184B1A9A1A6000F0AABF00BFCD
:10AAB0000E120300A4BAFF1FF7180300FC180300CE
:10AAC000B8BAFF1F061903000B190300CCBAFF1F09
:10AAD0000F190300E0BAFF1F40150300151903000A
:10AAE000F4BAFF1F1B19030008BBFF1FC8C5FF1FD7
:10AAF00008C6FF1F231903003B19030096C6FF1F5A
:10AB00000988FF1F00D8FF1FDC8EFF1F112840F0AF
:10AB100043824FF00008B54BCDF804801B88B44841
:10AB20000D3B1BB20D220093414623B21AF020FACE
:10AB30004FF6FF71AE4818F098F80121AC4818F0B4
:10AB40008EF8AC49AA4818F0E5F8434624220521BE
:10AB5000A74819F05DFBA849A548F5F714FD16AD07
:10AB6000A34818F0F1F8A54928461EF0D4FB4FF48D
:10AB70008E70F5F754FE1AAC0146282720461EF0C9
:10AB8000EAFB50213C233A469D48CDF80C800294C4
:10AB9000019500970EF061FD20461EF07CFB2846D3
:10ABA0001EF079FB4FF4D670F5F739FE12AE01288E
:10ABB0009449304620D11EF0AEFB934928461EF042
:10ABC000AAFB924920461EF0A6FB4FF4FC633A46CE
:10ABD0009B21049303943C230295019600978C4893
:10ABE0000EF0D6FC20461EF056FB28461EF053FB06
:10ABF00030461EF050FB24E01EF08DFB82492846B3
:10AC00001EF089FB814920461EF085FB46F22C335D
:10AC10009B213A4604937E4803943C230295019677
:10AC200000970EF0B5FC20461EF035FB28461EF0BE
:10AC300032FB30461EF02FFB41464FF4D670F5F73D
:10AC400081FD40F2AD10F5F7EAFD724928B12046CA
:10AC50001EF061FB4FF4FC6304E020461EF05BFB3A
:10AC600046F22C3328220092052102936A4801946F
:10AC70003C230EF04DFC20461EF00DFB674920469C
:10AC80001EF049FB664B282719784CF218682846B5
:10AC90001EF061FB3C233A46EB216248CDF80C8064
:10ACA0000295019400970EF0D8FC28461EF0F3FAA6
:10ACB00020461EF0F0FA5C4920461EF02CFB4FF4B3
:10ACC000D270F5F7ACFD014628461EF044FB3C234C
:10ACD0005F2205215548CDF80C800295019400971C
:10ACE0000EF0BBFC28461EF0D6FA20461EF0D3FA22
:10ACF0004F4920461EF00FFB002350215F22029394
:10AD00004C4801943C2300970EF002FC20461EF0B4
:10AD1000C2FA40F2AF10F5F782FD4749C8B9304694
:10AD20001EF0F9FA454928461EF0F5FA4449204636
:10AD30001EF0F1FA46F22C33049342480394029534
:10AD4000019600973C235F229B210EF021FC2046B8
:10AD50002EE030461EF0DFFA384928461EF0DBFAB6
:10AD600040F2AF10F5F75BFD01460AA81EF0F3FABA
:10AD70000AA90EA81EF039FB33490EA81EF0E6FB07
:10AD8000014620461EF031FB4FF4FC635F229B21FD
:10AD900004932C4803943C230295019600970EF0EF
:10ADA000F7FB20461EF077FA0EA81EF074FA0AA8E8
:10ADB0001EF071FA28461EF06EFA30461EF06BFA4D
:10ADC00040F21D10F5F72BFD01282049304643D1F4
:10ADD0001EF0A1FA1E4928461EF09DFA1D49204684
:10ADE0001EF099FA4FF4FC6342E000BF3E88FF1F5B
:10ADF00008C6FF1F6C2603005419030063190300E3
:10AE0000B8BAFF1FFB1403006C190300E51403001C
:10AE1000E0BAFF1F7519030008BBFF1F7D1903006F
:10AE2000FF87FF1FF4BAFF1F851903001CBBFF1F1C
:10AE30008E19030030BBFF1F941903009B190300F8
:10AE4000E618030044BBFF1F41160300A2190300CC
:10AE5000A7190300D41803001EF05DFA41492846E3
:10AE60001EF059FA404920461EF055FA46F22C339E
:10AE7000049328235F22EB2100933C4803943C2356
:10AE8000029501960EF084FB20461EF004FA284637
:10AE90001EF001FA30461EF0FEF9354B354F1B7897
:10AEA000F3B9354928461EF036FA344920461EF0DB
:10AEB00032FA39880A2230461EF060FA46F22C3304
:10AEC0000493282300930396029401953C23962231
:10AED00005212B480EF05CFB30461EF0DCF91FE02C
:10AEE0003B882549284643B11EF015FA25492046DE
:10AEF0001EF011FA4FF4784307E01EF00CFA2249D5
:10AF000020461EF008FA4FF4FC63039328230093B5
:10AF1000029401953C239622052119480EF09DFBD1
:10AF200020461EF0B8F928461EF0B5F9174920460C
:10AF30001EF0F1F9164B19780A22013128461EF04D
:10AF40001DFA0023039313480295282300930194CC
:10AF50003C23962250210EF080FB28461EF09BF9E0
:10AF6000A4E300BFA7190300E618030058BBFF1FA6
:10AF700064C5FF1FC08EFF1F6E150300AC190300D0
:10AF80006CBBFF1FB2190300B9190300C2190300FB
:10AF90008DC7FF1F80BBFF1F122840F0328500279E
:10AFA000B54B01971B88B5480D3B1BB20D223946A6
:10AFB000009323B219F0DCFF4FF6FF71AF4817F092
:10AFC00054FE0121AD4817F04AFEAD49AB4817F0D9
:10AFD000A1FE3B4624220521A84819F019F9A949E8
:10AFE000A648F5F7D0FAA54817F0AEFE4FF4D97091
:10AFF000F5F751FC16AD82B2A34912A81AAC22F0A3
:10B00000E9FBA249284628261EF085F912A9204608
:10B010001EF081F93C232D22052103979C480294C0
:10B02000019500960EF019FB20461EF034F92846D3
:10B030001EF031F94FF4DA70F5F72DFC924982B227
:10B0400012A822F0C7FB934928461EF064F912A902
:10B0500020461EF060F93C232D22502103978E4894
:10B060000294019500960EF0F8FA20461EF013F9AE
:10B0700028461EF010F94FF4DB70F5F70CFC8249FE
:10B0800082B212A822F0A6FB844928461EF043F99A
:10B0900012A920461EF03FF93C232D229B21039745
:10B0A0007F480294019500960EF0D7FA20461EF0D4
:10B0B000F2F828461EF0EFF84FF4DC70F5F7EBFBE2
:10B0C000714982B212A822F085FB764928461EF00B
:10B0D00022F912A920461EF01EF93C232D22E6215A
:10B0E000039771480294019500960EF0B6FA204637
:10B0F0001EF0D1F828461EF0CEF84FF4DD70F5F7BB
:10B10000CAFB614982B212A822F064FB6749284653
:10B110001EF001F912A920461EF0FDF83C235F2223
:10B120000521039762480294019500960EF095FA66
:10B1300020461EF0B0F828461EF0ADF84FF4DE7041
:10B14000F5F7A9FB504982B212A822F043FB5949F6
:10B1500028461EF0E0F812A920461EF0DCF83C2339
:10B160005F225021039754480294019500960EF0F7
:10B1700074FA20461EF08FF828461EF08CF84FF423
:10B18000DF70F5F788FB404982B212A822F022FB5B
:10B190004A4928461EF0BFF812A920461EF0BBF807
:10B1A0003C235F229B21039745480294019500961A
:10B1B0000EF053FA20461EF06EF828461EF06BF88B
:10B1C0004FF4E070F5F767FB2F4982B212A822F026
:10B1D00001FB3C4928461EF09EF812A920461EF0AD
:10B1E0009AF83C235F22E6210397374802940195A1
:10B1F00000960EF032FA20461EF04DF828461EF05A
:10B200004AF84FF4D870F5F746FBB8424FF4D870BF
:10B21000C8BF4FF4FC67F5F73EFB1B4982B212A88A
:10B2200022F0D8FA294928461EF075F812A92046BE
:10B230001EF071F805213C239122254803970294C2
:10B24000019500960EF009FA20461EF024F82846D3
:10B250001EF021F84FF4E270F5F7E1FA01281D49DC
:10B2600028463BD11EF057F81B4920461EF053F8E4
:10B270004FF4FC633AE000BF3E88FF1F08C6FF1F83
:10B280006C260300CA190300D5190300DC1903005A
:10B29000A4BAFF1FE4190300B8BAFF1FEC1903009A
:10B2A000CCBAFF1FF4190300E0BAFF1FFC1903001A
:10B2B000F4BAFF1F041A030008BBFF1F0C1A030097
:10B2C0001CBBFF1F141A030030BBFF1F1C1A030016
:10B2D00044BBFF1F211A0300AB1E03001EF01BF826
:10B2E000684920461EF017F846F22C33912250216F
:10B2F000039300963C230294019563480EF0ADF948
:10B3000020461DF0C8FF28461DF0C5FF5F492846AE
:10B310001EF001F8002628275D4920461DF0FBFF9E
:10B320003C23BE22052103960294019500975948BB
:10B330000EF093F920461DF0AEFF28461DF0ABFF3E
:10B34000554920461DF0E7FF3C23BE2250210296BE
:10B350000194009751480EF0DBF820461DF09BFF4A
:10B360004F4920461DF0D7FF3C23BE229B21029669
:10B37000019400974B480EF0CBF820461DF08BFF50
:10B38000494928461DF0C7FF484920461DF0C3FF24
:10B390003C23BE22E621039602940195009744487F
:10B3A0000EF05BF920461DF076FF28461DF073FF76
:10B3B0004CF218613F4817F058FC3346E7220A2147
:10B3C0003C4818F025FF3C493A48F5F7DCF818E30B
:10B3D0002B78052B07D1394B002019780EF0CCFDC6
:10B3E000002840F056812B78062B04D02B78072BB1
:10B3F00040F0518108E0314B012019780EF0BCFD7E
:10B40000002840F04681F1E72C4B032019780EF01C
:10B41000B3FD002840F03D813DE11A780A2A59D158
:10B42000274920461DF077FF002221461D480DF0D8
:10B4300095FF20461DF02FFF224920461DF06BFF8F
:10B4400046F22C3302931A23494601940093832237
:10B45000642317480EF05CF820461DF01CFF1A4AC2
:10B4600000231370194A1370194B14201C681EF026
:10B470002AF90546F5F7C6FA2946204616F072FC69
:10B48000BFE200BF8116030080BBFF1F2A1A030022
:10B49000311A030094BBFF1F351A0300A8BBFF1F1E
:10B4A0003B1A030058BBFF1F0F190300461A030085
:10B4B0006CBBFF1F08C6FF1F4A1A030094C5FF1F7D
:10B4C000F01503008F110300C4C5FF1FBCC5FF1F8B
:10B4D0004CD7FF1F1E78F6B2082E40F0D4808F4D57
:10B4E0008F49B5F80080DFF87CB2DFF88492A8F1CC
:10B4F0001A0820461DF00FFF1A271FFA88F844F299
:10B500000823424619210293864801943323009769
:10B510000DF0FEFF20461DF0BEFE2A888248DFF8AF
:10B520005482113A002312B21B2118F071FE9BF8CD
:10B5300000304FF0A80A0AFB0393324693F89110AB
:10B5400098F800300139C9B220460EF03DFD214681
:10B5500075481DF05DFD20461DF09DFE2A8870494E
:10B560001A3A92B2204607921DF0D5FE4FF4FC63C2
:10B57000079A0293522133236C48019400970DF0EF
:10B58000C7FF20461DF087FE2A886748113A00232E
:10B5900012B2552118F03CFE9BF8001098F80030CC
:10B5A0000AFB0191324691F8911020460EF00CFDF5
:10B5B00021465D481DF02CFD20461DF06CFE2A88BA
:10B5C00057491A3A92B2204607921DF0A4FE44F25F
:10B5D0000823079A02938B2133235548019400973F
:10B5E0000DF096FF20461DF056FE2A884E48113A6F
:10B5F000002312B28E2118F00BFE9BF800300AFBDC
:10B600000399324699F8911098F800300131C9B287
:10B6100020460EF0D9FC214643481DF0F9FC204697
:10B620001DF039FE2E8843491A3E4FF00008B6B28D
:10B6300020461DF070FE3246132341463E48CDF8A9
:10B640000880019400970DF063FF20461DF023FE53
:10B650003A4B2D881E883A497D3E1A3DB6B2ADB2AE
:10B6600020461DF058FE13232A4631463548CDF8B2
:10B670000880019400970DF04BFF20461DF00BFE53
:10B680003148FCF76EB81A783AB11B78022B11D109
:10B6900003E02E4902E02E4900E02E4920461DF02D
:10B6A0003AFE0022214628480DF058FE20461DF0A3
:10B6B000F2FDA6E1284920461DF02DFE002221467C
:10B6C00021480DF04BFE20461DF0E5FD2348F5F71F
:10B6D00043F9234B01221A7093E1237808FB03738B
:10B6E000002103F80A10FDF778BD1E4B93F8009077
:10B6F0002378F35C09F1FF329A4208D0B9F1000FC8
:10B700003AD1194B194A1B78D35CFF2B34D144F240
:10B71000082427464FF4FC6A48E000BF3E88FF1F1C
:10B72000A91603001CBBFF1F08C6FF1FE0BAFF1FBE
:10B7300030BBFF1F11110300F4BAFF1F0488FF1F65
:10B740001311030008BBFF1F58BBFF1F3B1A030068
:10B75000771A030088190300E91503006CBBFF1F6B
:10B76000C4C5FF1F94C5FF1F96C6FF1FC88EFF1FCD
:10B770008890FF1F22C4FF1F2378F35C4B4500F025
:10B7800097802A78914500F08C802178715C09F1CE
:10B7900001038B4200F09C80914500F08E80934223
:10B7A00000F0918044F208242746A246B8F800B081
:10B7B0002B781AAE09F1FF3130460822C9B2ABF13D
:10B7C000180B0EF001FC1FFA8BFBCDF808A04FF010
:10B7D000150A5A4633234A210196CDF800A08A481B
:10B7E0000DF096FE30461DF056FDB8F800B02B78EF
:10B7F000ABF1180B494630461FFA8BFB08220EF0BE
:10B80000E3FB5A460297332382210196CDF800A02C
:10B810007E480DF07DFE30461DF03DFDB8F800700D
:10B820002B7809F10101183F3046BFB20822C9B296
:10B830000EF0CAFB3A4633230294BA210196CDF8A2
:10B8400000A073480DF064FE30461DF024FDB8F8EA
:10B8500000407049183C0025A4B230461DF05BFD45
:10B8600022463323112102950196CDF800A06A48A3
:10B870000DF04EFE30461DF00EFDB8F80040674951
:10B88000183CA4B230461DF046FD02950196CDF855
:10B8900000A033232246F22161480DF039FEFCF767
:10B8A00026BD604B60491B78CB5CFF2B7FF46DAFEE
:10B8B00044F208244FF4FC6777E75A495A4809785C
:10B8C000415C29B16BE72378F35CFF2B7FF46AAF0F
:10B8D00044F208274FF4FC64BA4667E75349204610
:10B8E0001DF019FD524928461DF015FD4CF2186354
:10B8F0000393282300932D223C2305214D480295D4
:10B9000001940DF0AAFE28461DF0C5FC2046FEF766
:10B91000BFBC032B09D11DF0FEFC474928461DF092
:10B92000FAFC40F2FF73FEF70BBD1DF0F4FC434937
:10B9300028461DF0F0FC4FF4FC63FEF701BD022B1E
:10B940000BD13F4920461DF0E6FC3E4928461DF03C
:10B95000E2FC4FF6E073FEF713BD01214FF4D57002
:10B96000F4F7F0FE384920461DF0D5FC334928464F
:10B970001DF0D1FC4FF4FC63FEF702BD1278334B8F
:10B98000012A06D1324928461DF0C5FC4FF6E07366
:10B990002EE01A78022A01D12E491DE01A78032AD6
:10B9A00001D12D4918E01A78042A7EF45BAC2B49AA
:10B9B00012E01A78062A01D129490DE01A78072ADF
:10B9C00001D1284908E01A78082A01D1264903E064
:10B9D0001B78092B06D1254928461DF09CFC4FF405
:10B9E000FC6305E0224928461DF095FC4FF478439E
:10B9F00002932823009301953C232D220521FEF775
:10BA000043BC1FB0BDE8F08F6CBBFF1F80BBFF1FA6
:10BA100094BBFF1F11110300A8BBFF1F13110300EC
:10BA2000BCBBFF1F96C6FF1FC88EFF1FE618030092
:10BA3000AF170300F4BAFF1FF21103009E1B0300AF
:10BA4000F2180300AB1E0300EA1803007990FF1FF1
:10BA500092180300971803009C180300A318030012
:10BA6000AC180300B0180300B4180300B8180300A2
:10BA7000C01803002DE9F04F8BB004ABB84E83E83B
:10BA800003003778BDF91040BDF91250AFB90DF180
:10BA90001808B44940461DF03EFC23220F230093B2
:10BAA00011468223B0480297CDF804800DF030FD96
:10BAB00040461DF0F0FBAD4B1F700021AC4817F065
:10BAC000D4F80121AA4817F0CAF83178A84801EB48
:10BAD0004101490000232722323118F099FBA54B80
:10BAE0001F7899462FB17B1C89F800304FF0010870
:10BAF00001E04FF00A08A4B2ADB201232A46214664
:10BB00009D480DF09DFB38B33378DFF854B2062B17
:10BB100022D8DFF8B4A29949DAF8000021F0AEFA91
:10BB2000D0B197499248F4F72EFD404621F0B4F881
:10BB3000DAF8001021F004F9CAF80000384620F0C5
:10BB400033FC02460B4600208E491DF09FFF024643
:10BB50000B4600208C490AE201232A4621468B48E5
:10BB60000DF06EFB40B33378DFF8F4B1062B23D829
:10BB7000DFF854A28149DAF8000021F07FFAD8B149
:10BB800083497B48F4F7FFFC404621F085F8DAF85A
:10BB9000001021F0D5F8CAF80000384620F004FC67
:10BBA00002460B46002077491DF070FF02460B4607
:10BBB00000204FF08041DAE101232A4621467548F2
:10BBC0000DF03EFB38B33378DFF894B1062B22D862
:10BBD000DFF8F4A16949DAF8000021F04FFAD0B19A
:10BBE0006D496348F4F7CFFC404621F055F8DAF888
:10BBF000001021F0A5F8CAF80000384620F0D4FB68
:10BC000002460B4600205F491DF040FF02460B46EE
:10BC100000206249ABE101232A46214660480DF02D
:10BC20000FFB38B33378DFF838B1062B22D8DFF8B2
:10BC300098A15249DAF8000021F020FAD0B1594910
:10BC40004B48F4F7A0FC404621F026F8DAF8001043
:10BC500021F076F8CAF80000384620F0A5FB02462D
:10BC60000B46002047491DF011FF02460B460020FD
:10BC70004D497CE101232A4621464C480DF0E0FA6B
:10BC800038B33378DFF8D8B0062B22D8DFF838A1E4
:10BC90003A49DAF8000021F0F1F9D0B144493448CA
:10BCA000F4F771FC404620F0F7FFDAF8001021F0BD
:10BCB00047F8CAF80000384620F076FB02460B46EB
:10BCC000002030491DF0E2FE02460B4600203949B3
:10BCD0004DE101232A46214637480DF0B1FA68B1FB
:10BCE0003378DFF87CB0062B08D8DFF8DCA02349D6
:10BCF000DAF8000021F0C2F9002867D101232A46B2
:10BD000021462E480DF09CFA00287AD03378DFF8CF
:10BD100050B0062B75D8DFF8B0A01849DAF800004B
:10BD200021F0ACF900286CD025491148F4F72BFC20
:10BD3000404620F0B1FFDAF8001021F001F8CAF80F
:10BD40000000384620F030FB02460B4600200D492B
:10BD50001DF09CFE02460B4600201A4907E100BF79
:10BD60000088FF1F8F110300E0BAFF1FD98EFF1F4D
:10BD700008C6FF1F0988FF1F6CBBFF1F003C1C4645
:10BD8000CC160300000024400000F03F80BBFF1FE2
:10BD90008713030094BBFF1FD41603000000084064
:10BDA000A8BBFF1FD816030000001040BCBBFF1F3C
:10BDB000BF1A030000001440D0BBFF1FE4BBFF1FED
:10BDC0005D15030000001C40C0C5FF1FB949BA48FB
:10BDD000F4F7D9FB404620F05FFFDAF8001020F0BE
:10BDE000AFFFCAF80000384620F0DEFA02460B46E4
:10BDF0000020B2491DF04AFE02460B460020B04921
:10BE0000B5E001232A462146AE480DF019FA38B3B1
:10BE10003378DFF8FCB2062B22D8DFF8D8A2AA4983
:10BE2000DAF8000021F02AF9D0B1A849A248F4F7C5
:10BE3000AAFB404620F030FFDAF8001020F080FF27
:10BE4000CAF80000384620F0AFFA02460B46002040
:10BE50009A491DF01BFE02460B4600209C4986E0D5
:10BE600001232A4621469B480DF0EAF938B333787E
:10BE7000DFF89CB2062B22D8DFF878A29249DAF8D4
:10BE8000000021F0FBF8D0B193498B48F4F77BFB1D
:10BE9000404620F001FFDAF8001020F051FFCAF808
:10BEA0000000384620F080FA02460B460020834905
:10BEB0001DF0ECFD02460B460020884957E00123A7
:10BEC0002A46214686480DF0BBF978B199F8003032
:10BED000844C43B984497848F4F755FB33780133EF
:10BEE0003370012300E0013B237028E37F480123E6
:10BEF0002A46214600F5C8700DF0A2F960B13378EA
:10BF0000DFF80CB2062B07D8DFF8E8A16E49DAF8A3
:10BF1000000021F0B3F880B901232A462146744875
:10BF20000DF08EF900283AD0724B0021186821F0EC
:10BF30009BF8074600283FD031E06F495E48F4F790
:10BF400022FB404620F0A8FEDAF8001020F0F8FEB0
:10BF5000CAF80000384620F027FA02460B460020B7
:10BF600056491DF093FD02460B460020002120F0AB
:10BF7000BBFB0446DAF800000D4620F037FA0B460A
:10BF800002462946204620F0D3F820F07BFD9BF89E
:10BF90000030CAF8000001338BF80030CFE20123F3
:10BFA0002A46214655480DF04BF9002841D0544F00
:10BFB0003B780C2B4CD93CE0524C237883F00103A6
:10BFC00023702722034628213B4818F021F92578C1
:10BFD00006AC4DB14C493848F4F7D5FA4A492046E9
:10BFE0001DF099F902970FE008224CF218638DE8D2
:10BFF0000C002821052327222F4818F0B9FF4249B9
:10C0000020461DF088F902951923009391222823D8
:10C010007D21374801940DF07BFA20461DF03BF955
:10C0200099F80030002B00F08A822E4A013B1370F1
:10C0300085E201232A46214630480DF001F9A8B1D6
:10C040002F4B1A780D2A0FD01A780E2A0ED10BE03A
:10C0500000210520FAF718F839780620FAF714F8C5
:10C060002A4B06221A706AE20E2070E001232A464B
:10C07000214622480DF0E4F840B1214B1A780E2AEF
:10C0800004D91A78112A01D8142060E001232A4625
:10C0900021461A480DF0D4F800283BD0184B1A78E6
:10C0A000122A37D1194A1420107000221A70FF2169
:10C0B00052E000BF9018030008C6FF1F0000244094
:10C0C00000001840F8BBFF1F003C1C46F71203009D
:10C0D000000020400CBCFF1F73130300000022402F
:10C0E00020BCFF1F0988FF1F89130300A4BAFF1F8C
:10C0F00048BCFF1FC0C5FF1F4915030008BBFF1F39
:10C1000096C6FF1FD98EFF1F8B130300FD87FF1FED
:10C110000088FF1F01232A4621469B480DF090F816
:10C1200030B19A4B1A78122A02D91A78182A0DD9E6
:10C1300001232A46214694480DF082F878B1934BAA
:10C140001A781C2A0BD91A781E2A08D81120904A6E
:10C150001070FF221A701978F9F796FFEFE10123AA
:10C160002A4621468B480DF06BF808B133787BB92D
:10C17000002327225921884818F04AF84FF47841C3
:10C18000854816F072FD85498348F4F7FCF9D6E13D
:10C19000834B1B7823B1834A136803F10043136078
:10C1A0007A4C2378012B14D17F4B804A1B78A82529
:10C1B00005FB03257B4B186820F018F9C5E912012F
:10C1C00000210520F9F760FF714B06221A70002547
:10C1D00002E12378032B0CD1734B744A1B78A825FA
:10C1E00005FB03256F4B186820F000F9C5E916011F
:10C1F000E6E723780B2B0CD16B4B6C4A1B78A825F8
:10C2000005FB0325674B186820F0F0F8C5E920010D
:10C21000D6E723780C2B0CD1634B644A1B78A825F6
:10C2200005FB03255F4B186820F0E0F8C5E9220103
:10C23000C6E72378092B0CD15B4B5C4A1B78A825F9
:10C2400005FB0325574B186820F0D0F8C5E92601F7
:10C25000B6E723780D2B08D1524B55491B680B606C
:10C260001520F4F7B0FA0E2289E02578EDB20E2DF4
:10C270000AD14C4B4E491B6841F8043F1A20F4F791
:10C28000A2FA434B1D707CE023780F2B22D1454D41
:10C2900048492E68304620F00FFF20B90021304673
:10C2A00020F0E2FE08B1434B2B602868424E20F09C
:10C2B00049FF308041481CF04DFE338840493F48DB
:10C2C0004FF47A7292FBF3F2F4F732FB317840F2DA
:10C2D000CD1051E02378102B10D1324D3949286808
:10C2E00020F0EAFE08B1374B2B60286820F02AFFC7
:10C2F000354BC1B2197040F2CB103DE02378112BC1
:10C3000010D1284D2F4E2868314620F0D5FE00B1BF
:10C310002E60286820F016FF2C4BC1B219704FF424
:10C32000E67029E02378194D122B09D11D4B2849BD
:10C330001B680B6040F2D310F4F745FA1422F9E0C1
:10C340002B78122B03D92B78182B40F2E28023781C
:10C350000E4D192B4CD1134D164E2868314620F046
:10C36000ABFE00B12E60286820F0ECFE194B81B2C4
:10C37000198040F22710C9B2F4F7E4F91422044BF3
:10C380001A70FF23237022E708BBFF1F96C6FF1F0A
:10C39000FD87FF1FF4BAFF1F08C6FF1FC018030068
:10C3A000D98EFF1FC0C5FF1F94C5FF1F8890FF1FB8
:10C3B0008CC5FF1F00007F43E6C4FF1F84C7FF1F1B
:10C3C000CD0500000000C84288BAFF1F96C9FF1FB4
:10C3D00064C7FF1F62C5FF1F5A4B581914350CF074
:10C3E00027FFB5F5DC7FF7D1574B21781878B3E6F6
:10C3F0002B781A2B11D1554D554E2868314620F017
:10C400005BFE00B12E60286820F09CFE514B81B28B
:10C4100019804FF49470C9B2AEE72B781B2B11D161
:10C420004A4D4B4E2868314620F046FE00B12E6042
:10C43000286820F087FE484B81B2198040F229100D
:10C44000C9B299E72B781C2B11D1404D404E28687A
:10C45000314620F031FE00B12E60286820F072FED7
:10C460003E4B81B219804FF49570C9B284E72B78A6
:10C470001D2B0AD1354B186820F064FE384B1A8802
:10C4800080B2904213D100200EE02B781E2B16D1E3
:10C490002E4B34491D68284620F0F0FD38B128465F
:10C4A00020F050FE2E4B80B21880F4F795F9264B01
:10C4B00011221A702C4AFF232370137087E62B7801
:10C4C0001F2B7FF484AE214B274F1868DFF878804C
:10C4D00020F038FE224B1A8880B290424FF00006BE
:10C4E0000ED130461E80F4F777F9204B1E701423CE
:10C4F00088F800301E4B1E70FF232B703B7066E6E1
:10C50000032388F800302E70FF233B7029783046D3
:10C5100022E60E4B2E78186820F014FE154BC1B29F
:10C52000F6B228781E4400F5877006F8131CF4F75D
:10C5300009F91722044B1A70FF232B7047E60BB042
:10C54000BDE8F08FA4BAFF1FFD87FF1FC0C5FF1F06
:10C5500000007F43368DFF1FDCD4FF1F54C6FF1F32
:10C56000C08EFF1F00401C460988FF1F94C5FF1F97
:10C57000E08EFF1FD4D4FF1F2DE9F04F012085B0BE
:10C58000F4F74DF9304A314EA82303FB0020D0E9DF
:10C590000E8900222E4BD0E9160120F0A5F80246A4
:10C5A0000B4604460D464046494620F09DF820F0D3
:10C5B00049FA5FFA80FABAF1090F40D829462046B5
:10C5C00020F040FA87B207FB0AFB58461FF0FCFE3A
:10C5D000CDE9000116F80A001FF0E6FEB244044659
:10C5E0000D469AF801001FF0DFFE22462B461FF091
:10C5F0009DFDDDE90023CDE90201404649461FF0DB
:10C6000095FD02460B46DDE902011FF043FF80461F
:10C6100007EB0B0089461FF0D7FEDDE900231FF072
:10C6200085FD02460B464046494620F05DF822460D
:10C630002B461FF07DFD20F005FAC0B200E0B07A75
:10C6400005B0BDE8F08F00BF8890FF1FB9C4FF1F81
:10C650000000244037B500244FF4D8708DF8004016
:10C660008DF801400194F4F716F900283CD02349D5
:10C670002348F3F788FF4FF4E270F4F7D0F801286D
:10C68000054609D01F491E48F3F77DFF21464FF4A8
:10C69000E270F4F757F825461B491948F3F773FF82
:10C6A000002404F1D900400080B28DF80150F4F765
:10C6B000F2F8E2B201906946144815F053FC0134D7
:10C6C000019A13490E481CF0DAFC082CE9D14FF40A
:10C6D000D8708DF80050F4F7DEF80E49019002464C
:10C6E00007481CF0CCFC03E00B490548F4F702F9BD
:10C6F0006946064815F0FAFB03B030BD801A030006
:10C70000848AFF1F8C1A0300911A030034C5FF1F8F
:10C710009B1A0300A11A0300AD1A030038B10023CD
:10C720004210D9B290B20133002AF9D108467047BD
:10C730002DE9F04FB44DDFF8D8A2002687B00C46A3
:10C7400000F1FF3900F1BF083746AB4619F8013F49
:10C750003B2B40F07681092F04D10F2E40F29C80B4
:10C760000F269BE02EB37B1E172B22D8DFE813F099
:10C77000180024004F005900630070007A008A00FE
:10C780002100A500AF00B900C400CE00D800E2002F
:10C79000EC00FA0004010E011901230131015201DC
:10C7A0001022002102A821F061FFA82303FB0453FB
:10C7B0005860002320223BE11022002102A821F032
:10C7C00055FFA823C0B203FB04530228187201D1FD
:10C7D000012208E003280BD0042801D1022202E044
:10C7E000072803D10522894B1A70E2E7082802D1F5
:10C7F000864B1870DDE7092801D10622F3E70A28E5
:10C8000001D10722EFE70B28D3D10922EBE70A2257
:10C81000002102A821F02AFFA82303FB0453587229
:10C82000C7E70A22002102A821F020FFA82303FB6A
:10C8300004539872BDE70A22002102A821F016FFD6
:10C84000A823003003FB045318BF0120D872B0E7BF
:10C850001022002102A821F009FFA82303FB0453A2
:10C860001873A6E7A82606FB04561022002102A88A
:10C8700021F0FCFE337B3061D84080B2FFF74EFFE1
:10C88000307596E70A22002102A821F0EFFEA823C6
:10C8900003FB045358758CE7002E8AD0A82363430A
:10C8A000E818324602A91630019321F003F8019BE3
:10C8B0002B441E440023B3757BE7002102A821F01E
:10C8C0003BFEA82303FB0453C3E90A0171E70021DF
:10C8D00002A821F031FEA82303FB0453C3E90C0195
:10C8E00067E70A22002102A821F0C0FEA82303FB6B
:10C8F000045383F868005CE7002102A821F01CFEC5
:10C90000A82303FB0453C3E91C0152E7002102A83A
:10C9100021F012FEA82303FB0453C3E91E0148E7DC
:10C92000002102A821F008FEA82303FB0453C3E959
:10C9300020013EE7002102A821F0FEFDA82303FB11
:10C940000453C3E9220134E70A22002102A821F09E
:10C950008DFEA823003003FB045318BF012083F889
:10C96000900026E7002102A821F0E6FDA82303FBA2
:10C970000453C3E912011CE7002102A821F0DCFDE9
:10C98000A82303FB0453C3E9160112E70A2200217E
:10C9900002A821F06BFEA82303FB045383F8910047
:10C9A00007E7002102A821F0C7FDA82303FB0453D9
:10C9B000C3E92601FDE60A22002102A821F056FE65
:10C9C000A823003003FB045318BF012083F8A00004
:10C9D000EFE60A22002102A821F048FEA82303FB6B
:10C9E0000453002814BF0122002283F8A1201EBF97
:10C9F0009AF8003001338AF80030A82303FB04B30F
:10CA0000002283F8A220D4E68890FF1F8DBAFF1F72
:10CA10006BC7FF1F0A22002102A821F027FEA823CE
:10CA2000003003FB045318BF012083F8A300C0E6C5
:10CA300002A9CA5401330F2BFAD10137FFB20026E5
:10CA40002FE10A2B04D00D2B02D0192F40F01F81AB
:10CA5000A348A82303FB040240F6FF755168A942CE
:10CA600041D1537A0BB99F4B15E0012B01D19D4B5E
:10CA70002EE0022B02D19B4B9C7004E1032B02D1D0
:10CA8000984BDC70FFE0042B02D1964B1C71FAE04E
:10CA9000052B02D1944B1C70F5E0062B01D1934B72
:10CAA000F9E7072B01D1924BF5E7082B01D1914B08
:10CAB000F1E7092B01D1904BEDE70A2B01D18F4B08
:10CAC000E9E70B2B01D18E4BE5E70C2B02D18C4B08
:10CAD0005C70D8E00D2B01D18A4BDCE70E2B40F0C7
:10CAE000D280894BD7E740F6FE75A94240F0B88066
:10CAF000117A062940F0C780517A41B94FF420736A
:10CB000053600223537293720026804F0AE001297A
:10CB10000DD14FF4207368A7D7E900675360052350
:10CB200053729172C2E90A6700260027A9E0022920
:10CB300002D14FF4227313E003290DD14FF4307367
:10CB4000734F536000260123C2E90A675372937240
:10CB50005BA7D7E9006794E004290CD14FF4607318
:10CB60006C4F536000260123C2E90A675372937227
:10CB70000026694F85E005290FD14FF4727352A743
:10CB8000D7E900675360002353720123C2E90A67A3
:10CB900093724FA7D7E9006773E0062903FB0403EC
:10CBA0000DD14FF484625D4F5A60022200265A7202
:10CBB0000122C3E90A679A720026594F4DE05A7A5A
:10CBC000072A04D14FF484625A6003222BE0082A1A
:10CBD0000DD14FF484624F4F5A60042200265A72DE
:10CBE0000122C3E90A679A7200264B4F35E0092AF1
:10CBF0000AD14FF490625A6004225A7201229A724A
:10CC00002DA7D7E9006724E00A2A06D14FF4B162C4
:10CC10005A6004225A72012217E00B2A0DD14FF4F8
:10CC2000B1625A6007223F4F5A7200260122C3E9BF
:10CC30000A679A7200263C4F0FE00C2A23D14FF46A
:10CC400094625A6006225A72022223A7D7E900672B
:10CC50009A72C3E90A6700260027C3E90C6712E04D
:10CC600040F6FD7399420ED14FF4B1632D4F5360DE
:10CC700000260723C2E90A6753722B4F01239372E0
:10CC80000026C2E90C67A82303FB040410E0A3F10B
:10CC90002102592A05D806AA3244013602F8103C6E
:10CCA000F6B2C1457FF452AD0D4AA82303FB04241C
:10CCB000606807B0BDE8F08F000000A09999D93FE7
:10CCC0000000000000F08BC0000000C07268E93F67
:10CCD00000000040DF6759C000000040E17A843F57
:10CCE0008890FF1F8EBAFF1F4388FF1F4088FF1FD9
:10CCF0000288FF1F0788FF1F0A88FF1F4288FF1F47
:10CD00003988FF1F0188FF1F0B88FF1F0000D03FDD
:10CD100000001C400000E83F000048C00000E03F69
:10CD2000000049C00000F03F00004EC02DE9F04F68
:10CD3000CBB00646AD491AA81CF0EDFA1AA9304648
:10CD40001CF07DFC04461AA81CF0A5FA74BB08234D
:10CD50000A22A7491AA8F3F7C5FB1AA930461CF006
:10CD60004FFB1AA81CF097FA062231461AA81CF0AD
:10CD700089FCA04912A81CF0CEFA12A91AA81CF02E
:10CD80005EFC044612A81CF086FA1AA81CF083FA6E
:10CD900064B90623224631461AA81CF053FC1AA98E
:10CDA00030461CF02DFB1AA81CF075FA92491AA8FF
:10CDB0001CF0B1FA31461AA81CF0C0FB8F491CF0D8
:10CDC000C5FB014602A81CF010FB1AA81CF063FA70
:10CDD000029C8B4912A80123224613F069FD12A878
:10CDE00013F025FC00286AD112A813F014FC224687
:10CDF000844985481CF043F91BF060FF7E491AA85E
:10CE00001CF089FA31461AA81CF098FB7F491CF0E7
:10CE10009DFB014602A81CF0E1FA1AA81CF03BFA9F
:10CE2000224601237649029D1AA813F041FD1AA952
:10CE300012A8F4F7C7FB1AA813F0B6FB12A813F058
:10CE4000F6FB044600283AD12A46714D71496E48D6
:10CE50001CF015F91BF032FF2A886F480A3A234666
:10CE600012B20A2117F0D4F96C4B2A881B886A4841
:10CE70000B21693B0B3A4FF6E0751BB212B28DE8FD
:10CE80002200214618F074F84FF47841624815F0FA
:10CE9000ECFE63491AA81CF03EFA31461AA81CF0B1
:10CEA0004DFB01465C481CF0B3F81AA81CF0F3F9DE
:10CEB00012A813F0B0FB4FF4FA601AF019FB4FF40C
:10CEC0008C70F3F7ACFCFF284FF0000405D121462D
:10CED0004FF48C70F3F736FC63E1524B524A1C70EE
:10CEE000524B534D1C70FF23137053709370D370CB
:10CEF0001371504A2B7013704F4A6B7013704F4A66
:10CF000013704F4A13704F4A13704F4A13704F4AB1
:10CF100013704F4A12A8137013F089FBA94660B131
:10CF2000DFF834B127462546A046A24612A813F0E2
:10CF30005FFB002840D077B12CE146491AA81CF0CD
:10CF4000EAF91AAA0A212A48F3F7F6FA1AA81CF0F5
:10CF5000A2F9052787E012A813F0D3FA4AABC0B2B2
:10CF60002B440A2803F8C00C1AD1402C1DD80A2DD6
:10CF70001ED921461AA8FFF7DBFB50450CD0DBF881
:10CF800000300FFA88F203EBC20108F1010843F800
:10CF900032005FFA88F80C710134E4B2824605E091
:10CFA000C02D34BF0027032703E00227002500E03F
:10CFB0003D460135EDB2B9E70A2D11D9002F40F0F9
:10CFC000EC8021461AA8FFF7B3FB824546D0224BDE
:10CFD0001B680FFA88F803EBC80243F83800147195
:10CFE00012A813F018FB002F3BD03CE0BD1A030041
:10CFF00030C5FF1FA916030090110300961103000E
:10D00000E0D4FF1FC11A0300848AFF1FDF1A030048
:10D010003E88FF1FE41A030008C6FF1F0488FF1F95
:10D02000F31A03005AC7FF1F8EBAFF1F6BC7FF1FFB
:10D030003988FF1F4388FF1F4088FF1F0288FF1F9A
:10D040000788FF1F0A88FF1F0188FF1F0B88FF1F2B
:10D050004288FF1F081B0300A0C9FF1F12A813F07E
:10D06000DAFA34BB0427544C544822880A3A002385
:10D0700012B20A2117F0CCF8514B22881B880B20E2
:10D080004FF6E071693B0B3A8DE803001BB212B218
:10D0900000214A4817F06CFF4FF47841474815F0DB
:10D0A000E4FD3B463246474944481BF0E8FF002474
:10D0B00077E099F80030FF2B07D0434AA82101FB05
:10D0C00003239A7A0AB902229A7299F80120FF2A58
:10D0D00007D03D4BA82101FB02339A7A0AB90222FC
:10D0E0009A7230461CF0D5FA014606A81CF07DF96C
:10D0F00036490AA81CF00FF90AA930461CF09FFA1D
:10D100000022034606A90EA81CF09CFA0EA906A848
:10D110001CF076F90EA81CF0BEF80AA81CF0BBF8AB
:10D12000089B062B03D82A4906A8F3F7C4FB08235B
:10D130000A2228490EA8F3F7D5F90EA906A81CF073
:10D140007EFA05460EA81CF0A6F8BDB12249234878
:10D15000F3F719FA06A921481BF05AFF06A90EA8F1
:10D160001CF043F90A210EAA1A48F3F7E5F90EA8B4
:10D170001CF091F81A491948F3F7BCFB194B1978C0
:10D1800001B101214FF48C70F3F7DCFA06A81CF012
:10D1900082F806E00A2D7FF623AF12A813F03BFABF
:10D1A00061E712A813F000FA02A81CF074F82046F8
:10D1B0004BB0BDE8F08F00BF3E88FF1F08C6FF1FC1
:10D1C0000488FF1F2A1B03008890FF1F101B030009
:10D1D000A916030030C5FF1F141B0300848AFF1F1C
:10D1E000211B03008DBAFF1F034B1B780BB1FFF708
:10D1F0009DBD1846704700BFDBD4FF1F2DE9F04FDF
:10D20000A7B006AF07F1200381464FF4CC7083E846
:10D210000600F3F704FBB34CB7F92050B7F922A08E
:10D22000212888BFFF2019F01BFF01232370AE4B7C
:10D230007B61187808B9F5F7F3FFABB2AB4D3B61F2
:10D240002B68BB62AA4BBA6A1A604FF4E170F3F71D
:10D25000E6FABD6140B10021F02300911A46386919
:10D26000F3F7A1FA03B210E04FF6C1661AFB06F617
:10D2700040F2411396FBF3F63B6906F5A07603F105
:10D2800001080FFA86FA0FFA88F39A48FB6115F045
:10D290005BFD994A1578FF2D934611D1974909886E
:10D2A000183900235145237006DCF969182903DC7D
:10D2B0000123137002F099BC8BF8003002F095BC8A
:10D2C000012D40F2A980162D04D88D4BEB40DA07D2
:10D2D00000F14581894B1B88313B534578DCFA6965
:10D2E000132A75DC874E96F80080B8F1FF0F40F0E6
:10D2F0003381854C2078F4F77BF986F80080F4F7C9
:10D3000015FC9BF800300B2B09D1804B40F2A71085
:10D310001978F3F717FA7E4B1A787E4B1A709BF840
:10D320000030022B06D17B4B18780138C0B2F8F7D9
:10D330005BF807E006D9774B187801380021C0B2B6
:10D34000F8F7BCFC744B10225A72744B1B78042BF8
:10D3500003D101210846F5F735F8714BDFF8EC8170
:10D36000DFF8EC916F4E01221A704FF0000A6E4BFD
:10D37000504683F800A0F5F713FB0A201AF0B8F81E
:10D3800020786A4CF4F734F9554694F82730052B89
:10D390005FFA8AF202D00E2B42F0498494F85810BA
:10D3A000002902F06284618A208AF8F73BFB0AF1C7
:10D3B000010ABAF1110F04F17004E6D15C4BFF20B1
:10D3C000187000238BF80030F7F74AFC02F00DBC10
:10D3D000022D40F0C480534500F3C380FB69132B3A
:10D3E00000F3BF80474E3378FF2B00F0BA804F48E0
:10D3F000702404FB03000122FF210DF08DF9F4F7E6
:10D4000095FB0120F7F702FDF8F70EFC484AFF23D1
:10D410003370137002F0E9BB002D40F0A0800123AF
:10D420001370444A33481370434A404CDFF8249148
:10D43000137015F089FC7D6194F8583097F81480CA
:10D4400033B31FFA8AF60123BA8B314620460CF01B
:10D450000FFE18B12C4B1B78032B0DD03B69C3F189
:10D46000F0013246012389B220460CF001FE78B16A
:10D47000254B1B78032B0BD094F82730092B42F057
:10D4800087842E4B1B7803F0FD03012B02F0C2842E
:10D490007B690133112B7B6104F17004CCD1002D29
:10D4A00042F0A383264A274B107819788842154604
:10D4B0001C4606D2244B1878222828BFFF2019F0DA
:10D4C000CFFD6A7823789A4206D21F4B58782228DB
:10D4D00028BFFF2019F0C4FD0020F7F797FC02F0E9
:10D4E00084BB00BFBCC5FF1FD98EFF1F00D8FF1F24
:10D4F00024C5FF1F08C6FF1FFD87FF1F0488FF1FED
:10D50000004561004488FF1F2888FF1F65C5FF1F75
:10D510000888FF1F0688FF1F4CC4FF1F8CBAFF1F1F
:10D520003C88FF1F95BAFF1F8BBAFF1FB0BCFF1FBF
:10D530000988FF1FC4C5FF1F95C6FF1F5BC7FF1FDC
:10D540003988FF1F22C4FF1F69C7FF1F89BAFF1F49
:10D55000A4C5FF1FD58EFF1F022D3FF443AF142D2E
:10D5600033D8C24BEB40DE0708D5C14B1B78FF2BED
:10D5700004D1AAF138039BB22B2B09D90A2D24D14F
:10D58000BC4B1B88313B534547F3C98602F02DBB8A
:10D59000FB69132B19DCB84B00251D70B44BFF221F
:10D5A0001A70B64A01231370B54A23700220137013
:10D5B000F7F72CFC03238BF80030F4F7B7FA294671
:10D5C0002846F8F761FD02F010BB022D7DD1DFF88F
:10D5D000A08298F80030FF2B41F0DE81AAF16E03A3
:10D5E0009BB2362B0CD8FB69132B09DCF4F78CFAB1
:10D5F000FF28834604D0A34B1B78012B42F0CD8536
:10D60000AAF1A7039BB22C2B14D8FB69132B11DCB6
:10D610009C4B1A78012A14BF0122002201201A70A3
:10D62000F7F7F4FB984B18780138C0B2F7F7DCFE37
:10D6300002F0DBBAAAF1D6039BB22D2B01F2AC812A
:10D64000FB69132B01F3A8818E4B1B78012B01F092
:10D65000A3810320F3F7CCFF01218C4815F0FFFADA
:10D6600000218A4815F001FB894B1A78032A05D15D
:10D6700002221A704CF21863019308E0022A08BFD4
:10D6800004214CF2186218BF0321197001920B2378
:10D69000009301222B23D7217C4817F069FC7D4998
:10D6A00007F170001BF037FE05230093032207F1FA
:10D6B0007003ED2178480CF0EDFF07F170001BF0CE
:10D6C000EAFDF8F7B1FA02F090BA012D06F0A98749
:10D6D000032D06F04984042D06F09787052D12D0FE
:10D6E000072D06F086870C2D06F095870D2D06F088
:10D6F0008687112D06F07787122D07F03381142DC0
:10D7000016D105F0BBBFBAF1310F00F3AA85BAF10B
:10D71000000F40F3A685FB69272B47F30686012DF2
:10D7200006F08387032D06F02384142D05F0AA87C5
:10D73000182D30D1FB69322B10DD584BFA691B884C
:10D74000323B9A420ADA564B1A78FF2A06D1002158
:10D7500028461970F8F798FC02F047BABC8B51487C
:10D760001FFA8AF60123224631460BF069FD002894
:10D7700002F054854A4B1978FF2902F04F854A4A36
:10D78000535C632B02F24A85013318205354F8F797
:10D790007BFC02F02ABA162D3CD1FB69692B13DD04
:10D7A0003E4BFA691B881E3B9A420DDA3F4B1A78B2
:10D7B000FE2A09D03A4A002111702846FE221A702A
:10D7C000F8F762FC02F011BABC8B36481FFA8AF6F1
:10D7D0000123224631460BF033FD002802F0648617
:10D7E0002F4B1978FF2902F05F86314D314B2A7893
:10D7F0000B2000FB02325256632A02F355862A7828
:10D8000000FB023316205A5C01325A54F8F73CFCF4
:10D8100002F0EBB9152D51D1FB69214C322B09DDFA
:10D820002378FF2B06D1002128462170F8F72CFC25
:10D8300002F0DBB9BE8B1B481FFA8AF50123324682
:10D8400029460BF0FDFC002802F0D6872178FF293D
:10D8500002F0D287184A535C632B02F2CD87013362
:10D8600015205354F8F710FC02F0BFB9B6F21700B8
:10D870000988FF1F0488FF1FB8C4FF1FC4C5FF1F0E
:10D8800095C6FF1F0F88FF1F0688FF1F08C6FF1FD2
:10D890002888FF1FC7130300B0BCFF1F3E88FF1F6F
:10D8A00094C5FF1FA4BAFF1F78C5FF1FE08EFF1F9E
:10D8B00096C6FF1F57C6FF1FB9C4FF1F112D73D196
:10D8C000B7F81C80C4481FFA8AF601234246314645
:10D8D0000BF0B6FC50B34FF48E70F2F7A0FF01309E
:10D8E000C4B2292C28BF022421464FF48E70F2F7CF
:10D8F00029FFBA4907F160001BF00DFD214607F131
:10D9000070001BF028FD4CF2186307F1700207F15C
:10D910006001B1480BF058FD07F170001BF0BBFC33
:10D9200007F160001BF0B7FC02F05FB9012342462B
:10D930003146AB480BF084FC002803F007804FF41D
:10D94000D670F2F76CFF002843F00080A54907F17C
:10D9500050001BF0E0FCA44907F160001BF0DBFC69
:10D96000A24907F170001BF0D6FC4FF4FC6307F1ED
:10D97000500107F160020093994807F170030BF022
:10D980006BFD07F170001BF086FC07F160001BF0D7
:10D9900082FC07F150001BF07EFC01214FF4D67091
:10D9A000F2F7D0FE02F021B9172D40F09F80FB69FD
:10D9B0002C2B0EDC8E4A002313708E4A13708E4A75
:10D9C0001120FF2113708BF80000F8F75DFB02F0C7
:10D9D0000CB9B7F81C8089481FFA8AF6032342461F
:10D9E00031460BF02DFC054670B1834B13221A70A3
:10D9F00009238BF80030824B18781EF0D5FC0022EA
:10DA0000F6F7FEFD02F0F1B80323424631467248B4
:10DA10000BF016FC044670B1774B14221A700923E0
:10DA20008BF80030764B58781EF0BEFC2A46F6F78D
:10DA3000E7FD02F0DAB803234246314671480BF0A5
:10DA4000FFFB70B16C4B15221A7009238BF8003064
:10DA50006B4B98781EF0A8FC2246F6F7D1FD02F039
:10DA6000C4B80323424631465D480BF0E9FB70B170
:10DA7000614B16221A7009238BF80030604BD8785E
:10DA80001EF092FC0022F6F7BBFD02F0AEB80323B5
:10DA9000424631465C480BF0D3FB044670B1564B0E
:10DAA00017221A7009238BF80030554B18791EF095
:10DAB0007BFC0022F6F7A4FD02F097B80323424650
:10DAC000314652480BF0BCFB002802F08E804A4BD6
:10DAD00018221A7009238BF80030494B58791EF030
:10DAE00063FC2246F6F78CFD02F07FB8122D40F061
:10DAF00041810021464815F0B8F8B7F81C803F482E
:10DB00001FFA8AF60123424631460BF099FB05467F
:10DB100068B1404B00221A80364B022201201A7055
:10DB2000F6F752FB13238BF8003002F05EB80123A6
:10DB30004246314628480BF083FB044660B1354B22
:10DB40001D802C4B042201201A70F6F73DFB132395
:10DB50008BF8003002F049B801234246314629488B
:10DB60000BF06EFB054660B12A4B1C80214B062250
:10DB700001201A70F6F728FB13238BF8003002F00F
:10DB800034B801234246314615480BF059FB044690
:10DB900060B1204B1D80174B082201201A70F6F748
:10DBA00013FB13238BF8003002F01FB80123424609
:10DBB000314615480BF044FB054668B3154B1C80F5
:10DBC0000C4B0A2201201A70F6F7FEFA13238BF889
:10DBD000003002F00AB800BFB8BAFF1F6319030093
:10DBE000E0BAFF1FFB1403006C190300E5140300E7
:10DBF00094C5FF1FE08EFF1F96C6FF1FA4BAFF1F2C
:10DC0000D4D4FF1FCCBAFF1FF4BAFF1F08BBFF1FFD
:10DC100008C6FF1F58C7FF1F012342463146C548AB
:10DC20000BF00EFB044660B1C34B1D80C34B0C22AE
:10DC300001201A70F6F7C8FA13238BF8003001F0B0
:10DC4000D4BF012342463146BD480BF0F9FA0546E0
:10DC500060B1B94B1C80B94B0E2201201A70F6F747
:10DC6000B3FA13238BF8003001F0BFBF0123424603
:10DC70003146B4480BF0E4FA044660B1AE4B1D8067
:10DC8000AE4B102201201A70F6F79EFA13238BF880
:10DC9000003001F0AABF012342463146AA480BF0EA
:10DCA000CFFA58B1A44B1C80A44B01201C70F6F78E
:10DCB0008BFA13238BF8003001F097BF0123424603
:10DCC0003146A2480BF0BCFA50B100214FF4D87095
:10DCD000F2F746FD00211220F8F7D6F901F085BFD2
:10DCE0000123424631469A480BF0AAFA044678B11D
:10DCF0004FF4D874204600210134F2F723FDB4F527
:10DD0000E17FF7D100211220F8F7BEF901F06DBFD5
:10DD10000123424631468F480BF092FA002803F067
:10DD2000B2804FF4E270F2F77AFD012843F0AB8045
:10DD3000894907F160001BF0EEFA884907F170008D
:10DD40001BF0E9FA07F1600146F22C3307F170028B
:10DD500080480BF039FB07F170001BF09CFA07F1CB
:10DD600060001BF098FA21464FF4E270F2F7E8FCED
:10DD700001F03BBF132D5AD1794C267896B907F1A3
:10DD80007005784928461BF0C6FA0F2300937648A1
:10DD900002960195DC2323222D210BF0B9FB2846A6
:10DDA0001BF079FA002171486D4D14F05EFF0121DE
:10DDB0006E4814F054FF21786C4801EB4101490092
:10DDC00000232722323116F023FAB7F81C8060486E
:10DDD0001FFA8AF60123424631460BF031FA002839
:10DDE00003F0FF802B78032B03F2FB8060495F4830
:10DDF000F2F7C9FB504A2978138801311B0101331E
:10DE0000C9B2138029700A22C1F1040107F1700020
:10DE10001BF0B4FA4FF6E07207F1700148480BF0BE
:10DE20009DFA07F170001BF036FA01F0DEBE082DF6
:10DE30004FD1504B504C1B88313B534519DCFB698B
:10DE4000132B16DC4D4BFF221A704D4B01251D7014
:10DE50004C4B02201D70F6F7D9FF03238BF80030DE
:10DE6000F3F764FE002108462570F8F70DF901F07C
:10DE7000BCBEBAF1330F10DCFB69132B0DDC3F4B3A
:10DE8000002201210A201A70F8F7FEF8012364200D
:10DE90002370F6F7E5FE01F0A8BEAAF13606B6B289
:10DEA000322E4FF001050ED8FB69132B0BDC334BE0
:10DEB00000210A201D70F8F7E7F864202570F6F7B6
:10DEC000CFFE01F092BE64202570F6F7C9FE01F086
:10DED0008CBE072D40F0C2817A69BD8B2A48002391
:10DEE0001FFA8AF41370214601232A460BF0A8F981
:10DEF000064660B1254A1378591EC9B2FF29117030
:10DF000001D10C2149E0082948D1072145E001232E
:10DF10002A4621461E480BF093F98046002844D03B
:10DF20001A4A1378591CC9B20C29117032D91670CB
:10DF300034E000BF08BBFF1F58C7FF1FE08EFF1F64
:10DF40001CBBFF1F30BBFF1F44BBFF1F58BBFF1F85
:10DF50006CBBFF1F80BBFF1F211A0300811603004B
:10DF60000088FF1F8F110300E0BAFF1F08C6FF1FC4
:10DF7000CC1603000488FF1F3C88FF1F0988FF1F81
:10DF8000C4C5FF1F95C6FF1FA4BAFF1F94C5FF1F7E
:10DF9000B8BAFF1F082901D10921117012782D216B
:10DFA0000220F3F7FBFE03F00BBC01232A462146B7
:10DFB000BF480BF045F9002857D0BE4DBE48298810
:10DFC000DFF814935F393722434609B216F020F97F
:10DFD000F6F7A2FCB949B848F2F7D5FAB84B4FF4B6
:10DFE000B3701978F2F7AEFBB64B40F265101978B2
:10DFF000F2F7A8FB40F2671440F26F1663006FF46B
:10E00000337B5B44204619F80310DFF8CC820134DF
:10E01000F2F798FBB442F1D140F277166300A3F215
:10E02000DE23204618F803100134F2F78BFBB442CC
:10E03000F4D1322019F05CFA29889F480A234FF066
:10E04000000A5F398DE8080437225E2309B216F012
:10E050008FFF9D4B20461978F2F774FB9B4B40F2E3
:10E06000A9101978F2F76EFB82E001232A462146B7
:10E0700097480BF0E5F850B1964B1A78082A06D865
:10E08000954911F8123013B1013B03F0ECBA0123AA
:10E090002A46214691480BF0D3F820B18D4B1A78CF
:10E0A000082A43F2D982BAF1190F08DDDFF8048299
:10E0B000B8F80030A3F17D029245C3F2D782012364
:10E0C0002A46214682480BF0BBF8002843F0EE8236
:10E0D00001232A46214681480BF0B2F8002843F07C
:10E0E000F682BAF1190F08DDDFF8C881B8F8003000
:10E0F000A3F17D029245C3F22D8301232A462146D6
:10E1000073480BF09DF8002843F0458301232A460D
:10E11000214672480BF094F8002843F04883BAF186
:10E12000190F06DD634E3388A3F17D029245C3F2D9
:10E130004D8301232A46214665480BF081F80028CB
:10E1400003F06583634B1B780B2B43F06083644AB9
:10E150001378002B03F05B83012B43F25583023BC2
:10E16000137001210920F7F78FFF7A6901231370DB
:10E170007B691B78002B01F03885594B504A197880
:10E1800012789142984610D9564C207838B1524BAB
:10E19000D87BF5F745F80023237001F026BDF5F78D
:10E1A0003FF80123237001F020BD4FF4D470F2F743
:10E1B00036FB494C012894F80F902AD14FF0000A01
:10E1C0000546A27B98F800309A421FFA8AF60CD8CE
:10E1D0000DB194F80F904846F4F7D6FF3146024649
:10E1E000414818F0DAF9002507E00020F4F7CCFFE9
:10E1F000314602463C4818F0D0F90AF1010ABAF15A
:10E20000080FA4F10204DCD1374818F0F9F801F046
:10E21000ECBC072501264FF6FF7AA27B98F8003068
:10E220009A420CD80EB194F80F904846F4F7ACFF20
:10E23000294602462C4818F0B0F9002607E00020D5
:10E24000F4F7A2FF29460246274818F0A6F9013D37
:10E25000ADB25545A4F10204DFD1D5E7052D40F05C
:10E26000C880B7F81C90214D1FFA8AF801234A464E
:10E27000414628460AF0E4FF2C460646002855D0C1
:10E28000144E1B4D33782A78C2EB0308013BDBB2F6
:10E29000FF2B5FFA88F833702ED1164B1B785A1E6D
:10E2A000D2B20C2A32702FD90D3B2B7028E000BF60
:10E2B000CCBAFF1F0488FF1F08C6FF1F5B1B0300AB
:10E2C0003B88FF1FFC87FF1FE88EFF1F23C4FF1F33
:10E2D000E0BAFF1F94C5FF1F2988FF1FF4BAFF1F74
:10E2E000368EFF1FB8C5FF1F10C5FF1FA4BAFF1F42
:10E2F000E08EFF1F22C4FF1F9A4205D9013A2A70FF
:10E3000000210420F7F7C0FE33782A78618920893C
:10E310009A1AE3891944D2B2434689B2F3F73EFD13
:10E3200000210520F7F7B0FE01F05FBC4146012354
:10E330004A4605F114000AF083FF8046002838D0D1
:10E34000BE4ABF48137890F800E0CEEB03050133D6
:10E35000DBB2CEEB03010C29EDB21370B949904644
:10E36000814607DD0A789A4204D90EF10103037051
:10E37000314607E00A789A4207D8002188F8001051
:10E3800089F800100420F7F77FFE98F8003099F81C
:10E390000020618920899A1AE3891944D2B22B4658
:10E3A00089B2F3F7FBFC00210520F7F76DFE01F0C1
:10E3B0001CBCA54B1B88643B9A4581F21684FB6903
:10E3C000142B41F312849D4B9D4A1B781278698966
:10E3D00028899B1AEA891144DBB2FF2289B2F3F73C
:10E3E000DDFC062041468BF80000F7F74DFE01F0FA
:10E3F000FCBB062D40F0AD82B7F81C80934C1FFA91
:10E400008AF601234246314620460AF019FF81462A
:10E4100058B18F4C00212078F3F7EAFC00212070DE
:10E420000720F7F731FE01F0E0BB012342463146F9
:10E4300004F114000AF004FF824658B1844C012113
:10E440002078F3F7D5FC494620700720F7F71CFE2B
:10E4500001F0CBBB01234246314604F128000AF00B
:10E46000EFFE814668B37A4D05238BF80030794B77
:10E470002878FF2202211A70F3F7BAFC724B287039
:10E48000198875485F395346372209B215F0C0FE26
:10E49000F6F742FA714B2978012203201A70F7F738
:10E4A000F3FD664B664A1B781278618920899B1AB6
:10E4B000E289DBB2114489B21A46F3F76FFC01F02E
:10E4C00094BB01234246314604F1B4000AF0B8FE81
:10E4D0008246002800F028825D4C2378082B2646CF
:10E4E0004CD1DFF858A15E4E9AF8003021784FF0F9
:10E4F000A80808FB0363FF2283F891202846F7F75A
:10E50000C3FD01210720F7F7BFFD4FF6FF71524809
:10E5100014F0ABFB23785048CDF8049003EB430292
:10E5200003EB82022D320923009312B25A23642195
:10E5300016F01EFD2378484803EB430203EB8202EA
:10E540002D324B4612B2672115F062FE9AF8003068
:10E5500008FB03663B4B96F891101B784A4607F17F
:10E5600070000BF031FD07F170013B481AF050FDCF
:10E5700007F170001AF08FFE01F037BB23780B2BE8
:10E580000FD12E4B1A78364BA82101FB0233D3E969
:10E5900020010122F6F734F809238BF8003001F04E
:10E5A00024BB23780C2B0FD1244B1A782C4BA82199
:10E5B00001FB0233D3E922010122F6F721F80923F6
:10E5C0008BF8003001F011BB2478E4B2092C0ED195
:10E5D0001A4B1A78224BA82101FB0233D3E92601FA
:10E5E0000122F6F70DF88BF8004001F0FEBA3378FF
:10E5F000012B0FD1114B1A78194BA82101FB0233C3
:10E60000D3E912010122F5F7FBFF09238BF8003053
:10E6100001F0EBBA33780E4C032B23D1074B1A7859
:10E620000F4BA82101FB0233D3E916010122F5F7B4
:10E63000E7FF09238BF8003001F0D7BA94C5FF1F1C
:10E64000E08EFF1F22C4FF1F0488FF1FA4BAFF1F14
:10E6500096C6FF1F0988FF1F08C6FF1F68C7FF1F58
:10E660008890FF1F2378052B35D1C14D2C780020D1
:10E6700021460BF081FC80F00101C9B220460BF06D
:10E6800053FC00210720F7F7FFFC4FF6FF71B94854
:10E6900014F0EBFA002409238DE818006E223C23C5
:10E6A0006421B44816F064FC23466E226721B14809
:10E6B00015F0AEFD297820460BF05EFCF4F726F944
:10E6C000297820460BF058FC6D2102465120F3F7C3
:10E6D000E1FF01F08ABA2378062B51D1A44DA64E52
:10E6E0002C78012021460BF047FC80F00101C9B2D3
:10E6F00020460BF023FC337808B1013300E0013BE6
:10E7000000210720002433704FF00908F7F7BCFC04
:10E710004FF6FF71974814F0A8FA0194CDF80080E5
:10E720003C237B226421934816F022FC23467B2263
:10E730006721904815F06CFD297801200BF01CFC36
:10E74000F4F7E4F80194CDF8008008237B223D2102
:10E75000884816F00DFC23467B223D21854815F0A4
:10E7600057FD31788348F2F7B6F8297801200BF08D
:10E7700003FC7A2102465120F3F7C6FF01F035BAB7
:10E78000237803F0FF057BBB794B1A787B4BA821DC
:10E7900001FB023300200021C3E910014CF2186193
:10E7A000744814F062FA23787248019503EB43022F
:10E7B00003EB82022D320923009312B23C23642121
:10E7C00016F0D6FB23786B4803EB430203EB82027F
:10E7D0002D322B4612B2672115F01AFD68496548A3
:10E7E000F1F7D1FE01F001BA2378022B30D1604B52
:10E7F0001A78624BA82101FB023300200021C3E9F3
:10E8000014014CF218615B4814F02FFA2378594830
:10E8100003EB430203EB8202002509232D328DE82E
:10E82000280012B23C23642116F0A2FB2378514841
:10E8300003EB430203EB82022D322B4612B2672117
:10E8400015F0E6FC4E494B48F1F79DFE01F0CDB9BD
:10E850002578EDB2072D35D1454C26780320314679
:10E860000BF08AFB80F00101C9B230460BF07AFB55
:10E8700028460021F7F708FC4FF6FF713D4814F0D9
:10E88000F4F9002509238DE8280088224623642115
:10E89000384816F06DFB2B4689226721354815F064
:10E8A000B7FC217803200BF067FBF4F72FF82178F1
:10E8B00003200BF061FB892102465120F4F710F888
:10E8C00001F093B923780A2B41F08F812D4B2B480F
:10E8D00001221A70264B1978A82202FB010292F835
:10E8E00068300133DBB2022B82F8683006D85468F6
:10E8F00040F6FF72944207D0022B05D1A82303FBF8
:10E900000101002381F8683000210520F7F7BCFBE6
:10E91000307801300021C0B2F3F76AFA00210720F5
:10E92000F7F7B2FB01F061B901234246314604F129
:10E9300050000AF085FC002803F0C380124B1B78BE
:10E94000082B03F0BE8051460820F7F79DFB01F02D
:10E950004CB9092D1AD1BB8B7B84A7F820A007F1F5
:10E96000200393E80300FDF785F801F03EB900BFEE
:10E9700094C5FF1F08C6FF1F6BC7FF1F8890FF1FAE
:10E98000661B0300BCC5FF1F96C6FF1F042D01F0C8
:10E990002C81022D40F08D80112300257B61BD610B
:10E9A000BA4B1B78AB4201D0FF2B68D1BB69B84E84
:10E9B000B84AB7F81C900133DBB27024BB6104FB8A
:10E9C000056400231FFA8AF81370414601234A4662
:10E9D00020460BF04DFB48B1AF4B1B78032B05D104
:10E9E000AE4B1B78012B2BD103F04BB93B69C3F124
:10E9F000F0014246012389B220460BF039FB48B1B1
:10EA0000A54B1B78032B05D04FF4E170F1F707FFFE
:10EA10000028E5D001234246396920460BF028FB47
:10EA2000002803F02E819C4B1B78032B03F02981D7
:10EA30004FF4E170F1F7F3FE0028D1D103F021B9D2
:10EA400094F85830002B03F01C8194F825B0BBF1EA
:10EA5000000F43F016810320F6F7D8F98E4B187893
:10EA6000F2F7C6FD8D4B5A460121204683F800B0CF
:10EA700011F078F9854B1D70894B01221A707B6962
:10EA8000013B013513F0FF03EDB27B6188D1BB6917
:10EA900053B9824C2378FF2B06D00120F6F7B6F944
:10EAA000F7F7C2F8FF2323700320F2F7A1FD01F06E
:10EAB0009CB80B2D7B4E30D1B7F81C807A481FFADA
:10EAC0008AF50123424629460AF0BAFB002803F0E2
:10EAD000C384DFF8FC9199F80040EF2C03F2BC846A
:10EAE0000A34E4B240F2951089F80040F1F797FE3D
:10EAF000214618F009FC348899F800003E3C009447
:10EB000032231422FA21F1F73EFEA3B281B232225F
:10EB100066480AF0F3FD01F068B80C2D40F08581DD
:10EB200000216348634C644D14F09FF8B7F81C80D3
:10EB30002378BB611FFA8AF60123424631465E48BC
:10EB40000AF07EFB814658B32378013BDBB2FF2BF2
:10EB500023701AD159490A788AB9594B1B780B2B63
:10EB600002D8013B237010E00C2020700C2BA3F185
:10EB70000D00087007D8013B23700A7003E0013ACA
:10EB800000230A702370F6F777FAEB8969892278F7
:10EB90002889194489B2BB69F3F700F901F025B857
:10EBA00001234246314605F114000AF049FB824632
:10EBB00020B32378424A414910780A780133DBB206
:10EBC0009E18B042237006DC0B2881F8009084F870
:10EBD000009008D905E00C2B05D901320C230A70EE
:10EBE0002370F6F749FAEB89698922782889194454
:10EBF00089B2BB69F3F7D2F800F0F7BF01234246B0
:10EC0000314605F128000AF01BFB8146002861D03F
:10EC100040F29F10F1F703FE022896BF411C5146B7
:10EC2000C9B240F29F10F1F78DFD264907F160004F
:10EC30001AF071FB40F29F10F1F7F1FD1DF0B4FBEB
:10EC400002460B4600204FF080411AF01FFF1E4B7A
:10EC500000221DF01FFC1DF015FF0222014607F1E6
:10EC600070001AF0DEFB002307F1700207F160016B
:10EC700016480AF0A9FB07F170001AF00CFB07F127
:10EC800060001AF008FB00F0B0BF00BF4488FF1F0F
:10EC9000B0BCFF1FBCC5FF1F2888FF1F0988FF1FCE
:10ECA0003C88FF1F0488FF1FE0BAFF1F08BBFF1F3F
:10ECB00008C6FF1F94C5FF1FA4BAFF1FE08EFF1FE9
:10ECC00093BAFF1F6216030000405F40CCBAFF1FDB
:10ECD00065C5FF1F01234246314605F13C000AF09D
:10ECE000AFFA002800F08E80BC4CDFF83083BC48BF
:10ECF000DFF804A34FF6FF7113F0B7FFB8F8003048
:10ED00002288B748CDF80490693B0B3A0B261BB21A
:10ED100012B24946009616F02BF92288B048CDF879
:10ED20000490213A0A25C82312B20F21009516F04B
:10ED30001FF92288AA480A3A4B4612B2052115F05B
:10ED400067FAA849A648F1F71EFC49464FF48C70B3
:10ED5000F1F7F8FC07F17000F6F7A8FA07F1700078
:10ED6000FEF742FA8AF8000007F170001AF093FAF1
:10ED70009AF80030002B00F03887B8F8003022886D
:10ED80009748693B0B3A49468DE840021BB212B2E4
:10ED900016F0EEF82288924800954FF4E3530B3AB0
:10EDA00001934946782312B216F0E2F822888C4883
:10EDB0000A3A4B4612B2052115F02AFA8A498848C8
:10EDC000F1F7E1FB2A46082307F170008749F1F7C4
:10EDD00089FB07F1700182481AF01AF907F17000F7
:10EDE0001AF059FA22887E4800954FF478430B3A7E
:10EDF000019312B27823494614F004FAF6F73CF96D
:10EE000000F0F3BE01234246314605F164000AF0EA
:10EE100017FA002803F0C2834FF4E570F1F7FFFC06
:10EE2000002803F0EB8303F0B9BB0D2D40F0C18443
:10EE3000B7F81C806E481FFA8AF601234246314615
:10EE40000AF0FEF9B8B16B4C002323702078013032
:10EE5000F1F7E5FC684A694B1278187082429CBF52
:10EE6000FF221A701A78664B21781A700D20F7F776
:10EE70000BF900F0BABE01234246314661480AF060
:10EE8000DFF9B8B15B4C0223237020780130F1F731
:10EE9000C6FC594A594B1278187082429CBFFF2217
:10EEA0001A701A78564B21781A700D20F7F7ECF883
:10EEB00000F09BBE01234246314653480AF0C0F998
:10EEC000B8B14C4C0323237020780130F1F7A7FC34
:10EED000494A4A4B1278187082429CBFFF221A702E
:10EEE0001A78474B21781A700D20F7F7CDF800F00B
:10EEF0007CBE01234246314644480AF0A1F9B8B12C
:10EF00003C4C0423237020780130F1F788FC3A4A06
:10EF10003A4B1278187082429CBFFF221A701A78FE
:10EF2000374B21781A700D20F7F7AEF800F05DBE70
:10EF300001234246314636480AF082F9B8B12D4CD9
:10EF40000523237020780130F1F769FC2A4A2B4B06
:10EF50001278187082429CBFFF221A701A78284BD0
:10EF600021781A700D20F7F78FF800F03EBE0123CC
:10EF70004246314627480AF063F9A0B11F4B1D4CA9
:10EF8000197820781E4B0139C9B201301970F1F798
:10EF9000D9FBFF210D20F7F777F821780D20F7F73F
:10EFA00073F800F022BE0123424631461A480AF0A7
:10EFB00047F9A8B30F4C114B20781978104B01304A
:10EFC0001970F1F7BFFBFF210D20F7F75DF82178ED
:10EFD0000D20F7F759F800F008BE00BF3E88FF1F6C
:10EFE00008C6FF1F721B03004F16030030C5FF1F2A
:10EFF000A4BAFF1F96C6FF1F22C4FF1F94C5FF1FA0
:10F00000E08EFF1FCCBAFF1FE0BAFF1FF4BAFF1F4C
:10F01000D0BBFF1F08BBFF1F1CBBFF1F0488FF1FC7
:10F02000012342463146A9480AF00AF9A0B1A84B8B
:10F03000A84C19782078A84B0131C9B20130197059
:10F04000F1F780FBFF210D20F7F71EF821780D2046
:10F05000F7F71AF800F0C9BD0123424631469F4830
:10F060000AF0EEF880B19A4A1378013BDBB2FF2B2D
:10F07000137002BF9A4B1B781370964B0D201978B2
:10F08000F7F702F800F0B1BD01234246314695483A
:10F090000AF0D6F888B18E4A91491378097801337D
:10F0A000DBB2994213703CBF00231370894B0D20D3
:10F0B0001978F6F7E9FF00F098BD01234246314682
:10F0C00089480AF0BDF8044628B1FF210D20F6F763
:10F0D000DBFF00F08ABD01234246314683480AF037
:10F0E000AFF800285ED0824A13780133DBB2137088
:10F0F000062B15467F4B88BF14701A782B789342E5
:10F1000003D113B17A4A013313702B787A49012B5A
:10F1100007F1600003D11AF0FEF878491CE0022BD9
:10F1200003D11AF0F8F8764916E0032B03D11AF050
:10F13000F2F8744910E0042B03D11AF0ECF872498C
:10F140000AE0052B03D11AF0E6F8704904E0062B1B
:10F1500009D11AF0E0F86E4907F170001AF0DBF8F7
:10F160004FF4FC6308E01AF0D6F86A4907F1700022
:10F170001AF0D1F846F22C3307F1600107F1700262
:10F180005A480AF021F907F170001AF084F807F1E3
:10F1900060001AF080F8297840F21710F1F7D2FADF
:10F1A00000F023BD0123424631465B480AF048F88F
:10F1B0008146002800F0B6804E494D480B78007813
:10F1C0005A1CD2B290420A700C4602D108B10233E6
:10F1D0000B7023785149062B82BF464B00221A70D0
:10F1E0002378012B07F1500008D11AF094F84C490C
:10F1F00007F160001AF08FF8404935E0022B08D182
:10F200001AF089F8464907F160001AF084F83C4981
:10F210002AE0032B08D11AF07EF8414907F160007B
:10F220001AF079F837491FE0042B08D11AF073F867
:10F230003B4907F160001AF06EF8334914E0052BE2
:10F2400008D11AF068F8364907F160001AF063F83F
:10F250002E4909E0062B0ED11AF05DF8304907F16E
:10F2600060001AF058F82A4907F170001AF053F8B4
:10F270004FF4FC630DE01AF04EF8294907F16000E5
:10F280001AF049F8234907F170001AF044F846F2E1
:10F290002C3307F1500107F1600200931E4807F17B
:10F2A00070030AF0D9F807F1700019F0F4FF07F1C4
:10F2B000600019F0F0FF07F1500019F0ECFF217821
:10F2C00040F21510F1F73EFA00F08FBC30BBFF1F83
:10F2D00094C5FF1F96C6FF1FE08EFF1F44BBFF1F94
:10F2E00022C4FF1F58BBFF1F80BBFF1FB8BAFF1F00
:10F2F000348DFF1FE4C4FF1FBE160300CA160300AF
:10F30000CE160300D2160300D61603001A1203000D
:10F3100016120300E61803006CBBFF1FDA16030089
:10F32000C3160300012342463146C34809F088FF53
:10F33000002800F0AB80C14BDFF834831D78C04B50
:10F3400098F800401A784FF6E07395422CBF1D469E
:10F350004FF4FC65FF2C4FF4CD7046460AD1F1F70F
:10F360005EFAB84988F8000007F1600019F0D3FF91
:10F37000B54961E0F1F753FA844240F29B100AD19B
:10F38000F1F74DFAAF4988F8000007F1600019F075
:10F39000C2FFAE4950E0F1F742FA84424FF4CE701A
:10F3A0000AD1F1F73CFAA74988F8000007F160009C
:10F3B00019F0B1FFA6493FE0F1F731FA844240F27B
:10F3C0009D100AD1F1F72BFA9E4988F8000007F149
:10F3D000600019F0A0FF9F492EE0F1F720FA844267
:10F3E00008D1984988F8009007F1600019F093FF60
:10F3F000994921E04CB90123924988F8003007F17E
:10F40000600019F088FF954916E0012C09D1092305
:10F410008C4988F8003007F1600019F07CFF9049B2
:10F420000AE0092C0ED10A23864988F8003007F13A
:10F43000600019F070FF8B4907F1700019F06BFF45
:10F440002B460EE0FF237F4988F8003007F160006B
:10F4500019F061FF844907F1700019F05CFF46F272
:10F460002C3307F1600107F17002734809F0ACFF1B
:10F4700007F1700019F00FFF07F1600019F00BFFA2
:10F4800031784FF49070F1F75DF9AEE30123424615
:10F490003146764809F0D4FE002800F0A280674B80
:10F4A000734D5E78664B6C781A784FF6E07396422F
:10F4B0002CBF1E464FF4FC66FF2C4FF4CD70A846BF
:10F4C00009D1F1F7ACF96B49687007F1600019F0E8
:10F4D00022FF5D495BE0F1F7A2F9844240F29B1004
:10F4E00009D1F1F79CF96349687007F1600019F0E0
:10F4F00012FF56494BE0F1F792F984424FF4CE7077
:10F5000009D1F1F78CF95B49687007F1600019F0D7
:10F5100002FF4F493BE0F1F782F9844240F29D102F
:10F5200009D1F1F77CF95349687007F1600019F0CF
:10F53000F2FE48492BE0F1F772F9844208D100232A
:10F540004C496B7007F1600019F0E5FE42491EE07E
:10F5500044B9012347496B7007F1600019F0DBFEE5
:10F560003E4914E0012C08D1092342496B7007F190
:10F57000600019F0D0FE3A4909E0092C0DD10A23A8
:10F580003C496B7007F1600019F0C5FE354907F181
:10F59000700019F0C0FE33460DE0FF2335496B7053
:10F5A00007F1600019F0B7FE2F4907F1700019F05C
:10F5B000B2FE46F22C3307F1600107F170022B48CE
:10F5C00009F002FF07F1700019F065FE07F1600015
:10F5D00019F061FE98F8011040F21F10F1F7B2F82F
:10F5E00003E3012342463146234809F029FE00285F
:10F5F00000F0FB82214C23786BB901232049237052
:10F6000007F1500019F087FE1E4907F1600019F05C
:10F6100082FE0D4997E0012B36D102231849237051
:10F6200007F1500019F077FE164907F1600019F054
:10F6300072FE064987E000BF94BBFF1F3988FF1F99
:10F6400022C4FF1FE5160300CA160300CE160300EE
:10F65000D2160300D61603001A1203001612030076
:10F660001E12030022120300E6180300A8BBFF1FAE
:10F6700069C7FF1FED160300BCBBFF1F94C6FF1F29
:10F68000F516030058120300022B0DD10323C449C1
:10F69000237007F1500019F03EFEC24907F16000E7
:10F6A00019F039FEC0494EE0032B0DD10423BC49AB
:10F6B000237007F1500019F02EFEBA4907F16000DF
:10F6C00019F029FEB9493EE0042B0DD10523B449B8
:10F6D000237007F1500019F01EFEB24907F16000D7
:10F6E00019F019FEB2492EE0052B0DD10623AC49C5
:10F6F000237007F1500019F00EFEAA4907F16000CF
:10F7000019F009FEAB491EE0062B0DD10723A449D1
:10F71000237007F1500019F0FEFDA24907F16000C7
:10F7200019F0F9FDA4490EE0072B13D108239C49D9
:10F73000237007F1500019F0EEFD9A4907F16000BF
:10F7400019F0E9FD9D4907F1700019F0E4FD4FF44F
:10F75000FC6312E000239249237007F1500019F076
:10F76000DAFD904907F1600019F0D5FD944907F1E1
:10F77000700019F0D0FD46F22C3307F1500107F16B
:10F78000600200938F4807F1700309F065FE07F1EE
:10F79000700019F080FD07F1600019F07CFD07F1A1
:10F7A000500019F078FD217840F2FB10F0F7CAFF05
:10F7B0001BE2102D40F08181002323703388313B00
:10F7C000534519DCFB69132B16DC7F4BFF221A70A3
:10F7D0007E4B01241C707E4B02201C70F5F716FB3B
:10F7E00003238BF80030F2F7A1F97A4B0021084689
:10F7F0001C70F6F749FCF8E1B7F81C8076481FFA50
:10F800008AF601234246314609F01AFD054698B1B1
:10F8100040F21B10F1F703F820B1012814BF0021BA
:10F82000032100E0012140F21B10F0F78BFFFE21C5
:10F830001020F6F729FCD8E10123424631466748FB
:10F8400009F0FEFC044688B1654B33221A70654B03
:10F8500020225A726420F5F703FABB691B683B65E6
:10F86000614B3A6D1A60614B1D70BEE10123424647
:10F8700031465F4809F0E4FC054660B3584B5D49EA
:10F8800034221A70574B18225A7207F1600019F08F
:10F8900042FD594907F1700019F03DFD4FF6E07344
:10F8A00007F1700207F16001514809F08DFD07F181
:10F8B000700019F0F0FC07F1600019F0ECFC642016
:10F8C000F5F7CEF9BB691B683B66474B3A6E1A6089
:10F8D000464B1C7089E1012342463146474809F0F6
:10F8E000AFFC044660B33E4B454935221A703D4B90
:10F8F00014225A7207F1600019F00DFD3E4907F11C
:10F90000700019F008FD4FF6E07307F1700207F17F
:10F9100060013A4809F058FD07F1700019F0BBFC8E
:10F9200007F1600019F0B7FC6420F5F799F9BB699D
:10F930001B683B672C4B3A6F1A602C4B1D7054E1CF
:10F940000123424631462F4809F07AFC054600283B
:10F950007FD04FF4D770F0F762FF012858D12146CD
:10F960004FF4D770F0F7EEFE274907F1600019F069
:10F97000D2FC264907F1700019F0CDFC46F22C3379
:10F9800007F1700207F160011E4809F01DFD07F143
:10F99000700019F080FC07F1600019F07CFC24E194
:10F9A000F516030058120300D2160300D616030002
:10F9B0001A120300161203001E1203002212030083
:10F9C000E6180300BCBBFF1F0988FF1FC4C5FF1F4B
:10F9D00095C6FF1F3C88FF1FA4BAFF1FB8BAFF1FC0
:10F9E00096C6FF1F4CC4FF1FC48EFF1F6BC7FF1FAF
:10F9F000CCBAFF1F061903000B190300E0BAFF1F62
:10FA00000F190300F4BAFF1F4B150300151903006B
:10FA100001214FF4D770F0F795FEBD4907F1600062
:10FA200019F079FCBB4907F1700019F074FC4FF430
:10FA3000FC6307F1700207F16001B74809F0C4FCEC
:10FA400007F1700019F027FC07F1600019F023FCA2
:10FA5000CBE0012342463146B04809F0F1FB0028D3
:10FA600000F0C3804FF48A70F0F7D9FEAC4CAD497A
:10FA70000230C0B21E28207007F1600088BF2570D8
:10FA800019F049FC217807F1700019F064FC07F1C6
:10FA90006001002307F17002A04809F095FC07F10E
:10FAA000700019F0F8FB07F1600019F0F4FB217801
:10FAB0004FF48A70F0F744FE97E00E2DDFF8A8921D
:10FAC0003AD13288313A0023524523701BDCFA695F
:10FAD000132A18DC944A1370944BFF221A70944A2C
:10FAE00001231370934A23701370237002200323A1
:10FAF0008BF80030F5F78AF9F2F718F8002108467C
:10FB0000F6F7C2FA71E0B7F81C8083481FFA8AF64C
:10FB100001234246314609F093FB002802F0F786A4
:10FB2000854D2B78FF2B02F0F286844B1A78012A40
:10FB300042F0ED8602F0EFBD0F2D56D1804C2678B5
:10FB400096B907F170057F49284619F0E4FB0F23A9
:10FB500000937D4802960195DC2323222D2109F094
:10FB6000D7FC284619F097FB00217848744D13F014
:10FB70007CF80121754813F072F82178734801EB85
:10FB80004101490000232722323114F041FBB7F82C
:10FB90001C806F481FFA8AF601234246314609F05D
:10FBA0004FFB002803F051822B781F2B03F24D826C
:10FBB00068496648F0F7E7FC2978674B31225A54C8
:10FBC0000131C9B229700A22C1F1200107F1700088
:10FBD00019F0D4FB61484FF6E07207F1700109F0AB
:10FBE000BDFB07F1700019F056FB5D4B4FF4A0729E
:10FBF0001A805C4BF0221A805B4B1B78012B06D1DC
:10FC00005A4A5B495B48F0F793FE05F026BCC820D2
:10FC1000F3F74AFB4FF4CC70F0F701FE032256498C
:10FC2000212888BFFF2017F01FFB05F016BC0A2B08
:10FC30001ED194F85830002B3DF4B9AB002D7DF463
:10FC4000B6AB4E4B1878A38B83427DF4B0AB012545
:10FC5000F4F774FEE5834A494A48F0F794FCE18BD7
:10FC60004848F0F75BFEFDF7A2BB0A2B3DF49FABC3
:10FC70000B2B7DF49CAB94F85830002B3DF497ABE4
:10FC8000A38B092B05D1404A337812789A4233D19D
:10FC90003BE00A2B04D13D4932780978914234D0B7
:10FCA0000A2B29D00B2B02D13278FF2A2DD00B2B17
:10FCB00022D00C2B02D13278FE2A26D00C2B1BD05E
:10FCC0000D2B03D199F80020022A19D00D2B13D047
:10FCD0000E2B3DF46CAB0F2B3DF469AB98F8002074
:10FCE00042FA03F3DB077DF562AB40F21910F0F73F
:10FCF00096FD50B9FDF75BBB0023E383FDF757BBCF
:10FD00000123E3832384FDF752BB0123F5E700BF02
:10FD10004015030015190300F4BAFF1F08BBFF1FAD
:10FD200056C6FF1F1B190300B8C4FF1F0988FF1F19
:10FD3000C4C5FF1F95C6FF1F7990FF1F5BC7FF1F3C
:10FD40000088FF1F8F110300E0BAFF1F08C6FF1FC6
:10FD50006CBBFF1FCC160300C4C4FF1F1CBBFF1FDE
:10FD60000488FF1F3E88FF1FFD87FF1FA08601003C
:10FD700025080000388EFF1FA95401004188FF1F8D
:10FD80007D1B0300848AFF1F88BAFF1F96C9FF1FCF
:10FD9000122B0CD100238BF80030BB8B7B84A7F88F
:10FDA00020A0AC4B386ABA8C18609A8050E00A2BBD
:10FDB0001DD1E38B00228BF800208BB9A649184691
:10FDC000CA18703392F827500A2D08BFD083B3F5B4
:10FDD000EE6FF5D1A14B207F18700125E58315E06A
:10FDE0009E4BE283FF201870F4F73AFF5DE00B2B87
:10FDF00040F08C81A68BA6F10903032B2AD8984BDF
:10FE00001B7803F0FD03012B5FD0FF20F4F728FFE0
:10FE1000FDF73EBB934DA28B2978914248D12B70C0
:10FE2000297840F2AB10F0F78DFC00228A4B8E4807
:10FE3000114693F82760092E3DD01432B2F5AA7FFF
:10FE400003F17003F5D12B78E38300238BF80030A6
:10FE5000FF20C9E70D2E00F0BF800E2E00F0E280DB
:10FE60000F2E00F01D8140F21910F0F7D8FC002889
:10FE70003DF40EABE28B7D4D00238BF80030002A61
:10FE800040F02B8101232A78E383B3401343DBB294
:10FE9000FF202B70F4F7E4FE228C002A40F024812E
:10FEA000297840F2C710F0F74DFC0125FDF7F0BAB4
:10FEB000D2B22A70B4E793F85860002EBDD08618ED
:10FEC000367C002EB9D0D983B7E7002362498BF87E
:10FED0000030184691F827200B2A07D1DAB2904556
:10FEE00004D08A8B093A92B2032A73D90133112BB9
:10FEF00001F17001EED15E4BA18B1B785D4DE68B5D
:10FF0000002B14BF4FF4807000200B2914D11EB9B0
:10FF10000123E383FF2157E0574B00212970E18340
:10FF20001880564B1A78564BA82000FB0233002548
:10FF30000026C3E90E5648E00C294FF0010E0CD103
:10FF40001EB9A4F81EE0FE213EE04B4B18804D4B3D
:10FF50000021E18319802970E3E7474A474B26BB1C
:10FF600009290CBF48494949A4F81EE091F80080CE
:10FF70001B781FFA88F1FF2B118008D0404AA82671
:10FF8000404606FB03261CF00FFAC6E90E01404B63
:10FF90003B491B7885F80080A82202FB0318002249
:10FFA0000023C8E90E2329780FE01B781080002178
:10FFB000FF2BE18307D0324AA82101FB0323002154
:10FFC0000022C3E90E12002129704FF4F170F0F7FE
:10FFD000B9FB3DE7C88389E72E4D2B780022022B21
:10FFE0008BF8002004D10123E38303232B7014E05A
:10FFF000032BE2834FF0010102D1228429700CE02F
:020000021000EC
:10000000012B4FF0020009BF287028702384194685
:1000100018BF218420460FF093FE002120460FF0E8
:100020008FFE15E700238BF800301B4A1B4B1B7813
:10003000127803F00F0302F00F02013201339342F2
:10004000C8BF002399F80020638402F0F002134334
:100050003BE000BF7EC7FF1FB0BCFF1F4188FF1FF2
:1000600064C5FF1F7990FF1FA4BAFF1F89BAFF1F45
:1000700020C4FF1F95BAFF1FBAC5FF1F0A88FF1FC4
:100080008890FF1F94C9FF1F88BAFF1F96C9FF1FE2
:100090000188FF1FA4C5FF1FD68EFF1FD58EFF1F2F
:1000A00000238BF80030AE4B1B781B09591CAD4B5D
:1000B0001A7899F80030120901329142C8BF002124
:1000C00003F00F03618443EA0113DBB289F80030C7
:1000D00099F800104FF4E47079E7E3832A7801235C
:1000E000B34022EA0303D3E694F822300133DBB2B3
:1000F0000132934208DDA08B29780122824000233F
:1001000021EA0202E3832A706384C9E6102B7DF49E
:10011000BFA9BAF14F0F21DCFB69632B0ADC924ABD
:1001200018215172BA691268FA6200238BF8003004
:10013000F96A0DE0FB698C2B7DF7AAA98A4A142184
:100140005172BA6912683A630023396B8BF8003038
:10015000864A1160864AFE20137045E6BAF1910F77
:100160007DF796A9FB69782B7DF792A97E4D002635
:1001700028468BF80060F0F71AFC20236B72BB69ED
:100180001B683B64794B3A6C1A60794BFE201E70F9
:10019000F4F766FD774B1E7087E60320F4F736FE12
:1001A000744B4FF0010983F800900423A7F87030D6
:1001B000714B702404FB0B34704B1A88704B1988F8
:1001C00022FA09F221FA09F100265023283A2839A7
:1001D00088F8006087F86060A7F872602046009396
:1001E0000296019592B289B20FF0F8FD4A4607F1E6
:1001F00060012046F0F7CAFB07F170012046F0F7D6
:10020000BEFB4946204684F8589098F800200FF02D
:10021000A9FD314620460FF093FDE6E40123224676
:100220003146584809F00CF860B1574B1978FF294E
:1002300008D0564A535C2BB1013B18205354F5F7B4
:1002400023FFD2E4012322463146514808F0F8FF4B
:1002500020B14D4B1978092940F2BB800123224679
:1002600031464C4808F0ECFF804698B1464C4A4D68
:1002700021780139C9B240F207202970F0F762FAFB
:10028000464B2A781A70FF21002318202370F5F7B7
:10029000FBFEAAE4012322463146414808F0D0FF84
:1002A000054688B1384C3C4D2178297040F2072032
:1002B000F0F748FA394B2A781A70FF21182084F891
:1002C0000080F5F7E1FE90E40123224631463548EF
:1002D00008F0B6FF90B12C4C2F4E21780131C9B2F5
:1002E00040F207203170F0F72DFA2C4B32781A705B
:1002F000FF2118202570F5F7C7FE76E4012322467A
:100300003146294808F09CFF054680B11E4B1A78FB
:10031000013AD2B2FF2A1A7002BF244A12781A7028
:1003200019783839C9B21820F5F7AEFE5DE401231B
:10033000224631461E4808F083FF00283AD0124B6F
:100340001A491A7809780132D2B291421A7038BF2C
:100350001D7019783839C9B21820F5F795FE44E4B4
:10036000D58EFF1FD68EFF1F4CC4FF1FC48EFF1FEC
:100370006BC7FF1F3C88FF1FB0BCFF1F3E88FF1FDD
:100380000488FF1FB8BAFF1F94C5FF1F78C5FF1F61
:10039000CCBAFF1F08BBFF1FE08EFF1F21C4FF1F49
:1003A0001CBBFF1F30BBFF1F44BBFF1F22C4FF1F2E
:1003B00058BBFF1FFB692C2B44DD2246012331462D
:1003C000BA4808F03DFFBA4A50B11378092B39D822
:1003D00006E00131C9B218201970F5F755FE04E4A2
:1003E000B44BF9691B88313B8B420DDCB24BB349EE
:1003F000187808701978117019783839C9B218202E
:10040000F5F742FEFFF7F1BB1178FF293FF4EDABA2
:10041000273EF82E3FF6E9AB503C6E2C3FF6E5AB9D
:10042000FB69A3F1BE08642303FB08F86FF06D03BA
:1004300098FBF3F8A24B182003F80180F5F724FE8F
:10044000FFF7D3BB9E4E4FF4FE7440F20725A4F590
:10045000FE732046F15C0134F0F774F9AC42F6D13A
:10046000FB69934C2C2B4FF000030CDC934A237058
:100470001370944A0E20FF218BF800001370F5F7DB
:1004800003FEFFF7B2BB0193AC230093302213238A
:100490004FF496718C4814F06BFDFF2118202170E9
:1004A000F5F7F2FDFFF7A1BB01232246314687484D
:1004B00008F0C6FEB8B17E4B1978FF2913D0814DE4
:1004C000834B2A780B2000FB0232525663320ADB40
:1004D0002A7800FB023316205A5C013A5A54F5F789
:1004E000D3FDFFF782BB0123224631466F4808F057
:1004F000A7FE58B16E4B1978092907D80131C9B246
:1005000016201970F5F7C0FDFFF76FBBFB692C2BA8
:1005100007DD012322463146644808F091FE002899
:100520003DD0634D2B780A2B39D1DFF89881DFF865
:10053000A09100240B2698F8000098F8003006FBE4
:10054000039306FB0040195D00F516700134F0F7C7
:10055000F9F80B2CEFD1FB69584C2C2B4FF0000312
:100560000BDC584A2B701420FF218BF800002370FD
:100570001370F5F789FDFFF738BB0193AC230093A7
:10058000302213234FF496714F4814F0F1FCFF21F1
:10059000162029702170F5F777FDFFF726BB04239D
:1005A000224631464B48454D08F04AFE58B1404B73
:1005B000FF211970434B2970002216201A70F5F79D
:1005C00063FDFFF712BB042322463146424808F080
:1005D00037FE58B1364BFF2119703A4B2970012272
:1005E00016201A70F5F750FDFFF7FFBA04232246D4
:1005F00031463A4808F024FE58B12D4BFF211970BE
:10060000304B2970022216201A70F5F73DFDFFF7D6
:10061000ECBA042322463146314808F011FE58B1A5
:10062000234BFF211970274B2970032216201A70C3
:10063000F5F72AFDFFF7D9BA0423224631462948A7
:1006400008F0FEFD58B11A4BFF2119701D4B29709F
:10065000042216201A70F5F717FDFFF7C6BA2B789B
:10066000FE2B41D1A6F12703F82B3DD8A4F1690355
:10067000552B39D80E4A134B11781B78144A0B208E
:1006800000FB0322FB69A3F1BE08C82303FB08F8A3
:1006900016206FF0540398FBF3F8A8F1640802F8F1
:1006A0000180F5F7F1FCFFF7A0BA00BFCCBAFF1F3D
:1006B00094C5FF1F3E88FF1F21C4FF1FE08EFF1F50
:1006C00078C5FF1F96C6FF1F08C6FF1FB8BAFF1FD9
:1006D00057C6FF1FE0BAFF1FF4BAFF1F08BBFF1F7A
:1006E0001CBBFF1F30BBFF1F052322463146B54808
:1006F00008F0A6FDA0B1B44BB44C197820780139AC
:10070000C9B200F5F7702970F0F71CF82378B04AE9
:100710002978D1541620FF21F5F7B6FCFFF765BA0A
:10072000052322463146AB4808F08AFD90B1A74C1C
:10073000A54B20781978297000F5F770F0F702F8CA
:100740002378A34A2978D1541620FF21F5F79CFC81
:10075000FFF74BBA0523224631469F4808F070FD4B
:10076000A0B1994B994C197820780131C9B200F5A4
:10077000F7702970EFF7E6FF2378954A2978D1546E
:100780001620FF21F5F780FCFFF72FBA052322463C
:100790003146924808F054FD054690B18A4A1378D4
:1007A000013BDBB2FF2B137002BF8D4B1B78137024
:1007B000864B19786431C9B21620F5F765FCFFF74E
:1007C00014BA052322463146864808F039FD002830
:1007D00036D07D4A8249137809780133DBB29942D9
:1007E00013707A4B38BF157019786431C9B216206E
:1007F000F5F74AFCFFF7F9B90123324629467A4852
:1008000008F01EFD10B12178FF2934D101233246B2
:100810002946764808F014FD10B12178092969D9D4
:10082000FB692C2B32DD0123324629466F4808F044
:1008300007FD58BB2178FF2902D0BAF1260F62DCF0
:10084000FB692C2B3FF7D1A9AC2200238DE80C00CB
:100850004FF4967113233022654814F089FB5A4BEC
:10086000FF211970634B14208BF800001970F5F705
:100870000BFCFFF7BAB9604A535C002BC6D0013BB2
:1008800015205354F5F700FCFFF7AFB923780A2B76
:10089000D0D1594E40F2D7156FF4EB73EB182846C0
:1008A000F15C0135EFF74EFFB5F5F17FF4D1FB694F
:1008B0002C2B4FF000030CDC4E4A23701370434A7C
:1008C0001420FF218BF800001370F5F7DDFBFFF714
:1008D0008CB90193AC230093302213234FF496710B
:1008E000434814F045FBFF2115202170F5F7CCFBA0
:1008F000FFF77BB9344B0131C9B215201970F5F7F8
:10090000C3FBFFF772B9FB694F2B99DDBAF5907FF6
:10091000BFF66BA9BE2B3FF768A9384B364A1B7848
:10092000032BFB694FF01500A3F1BE081ABF642327
:1009300003FB08F8C8EB08286FF06D0398FBF3F889
:1009400002F80180F5F7A0FBFFF74FB901234246FB
:1009500031462B4808F074FC002859D04FF4D6706B
:10096000EFF75DFF002853D0264907F1500018F03B
:10097000D2FC254907F1600018F0CDFC234907F1AE
:10098000700018F0C8FC46F22C3307F1500107F153
:10099000600200931A4807F1700308F05DFD07F14B
:1009A000700018F078FC07F1600018F074FC07F193
:1009B000500018F070FC00214FF4D670EFF7C2FE23
:1009C000FFF713B96CBBFF1F94C5FF1F96C6FF1F2F
:1009D000C88EFF1F80BBFF1F94BBFF1FA8BBFF1F5C
:1009E00022C4FF1FBCBBFF1FB8BAFF1FCCBAFF1F3A
:1009F00008C6FF1FE08EFF1FB9C4FF1F64C5FF1F9D
:100A0000E0BAFF1FFB1403006C190300E514030098
:100A1000012342463146D34808F012FCD8B140F2D7
:100A2000AD10EFF7FCFEB0B1002140F2AD10EFF7D2
:100A300089FECD4907F1700018F06DFC46F22C32AA
:100A400007F17001C74808F089FC07F1700018F041
:100A500022FCFFF7CAB8012342463146C14808F0DC
:100A6000EFFBD8B140F2AD10EFF7D9FEB0B90121DC
:100A700040F2AD10EFF766FEBB4907F1700018F0C9
:100A80004AFC4FF4FC6207F17001B64808F066FCBE
:100A900007F1700018F0FFFBFFF7A7B801234246EB
:100AA0003146B24808F0CCFB002834D0B04CB148F5
:100AB0002378132B94BF05330A3323702378642BD8
:100AC00084BFAB4B05224FF0000188BF1A7012F0B3
:100AD000CCF8217840F20710EFF734FEA64907F171
:100AE000700018F018FC217807F1600018F033FC52
:100AF0004CF2186307F1600207F170019B4808F09F
:100B000063FC07F1600018F0C6FB07F1700018F0F5
:100B1000C2FBFFF76AB8012342463146974808F006
:100B20008FFB50B34FF4D270EFF779FE0230C4B2AE
:100B3000292C28BF0424924907F1700018F0EBFB20
:100B4000214607F1600018F006FC07F170014CF235
:100B5000186307F16002894808F036FC07F160006D
:100B600018F099FB07F1700018F095FB21464FF43F
:100B7000D270EFF7E7FDFFF738B801234246314660
:100B8000804808F05DFB054638B11720FF218BF83F
:100B90000000F5F779FAFFF728B8012342463146FD
:100BA000794808F04DFB8146002873D040F2AF1021
:100BB000EFF735FE0130C4B2052C744907F150003F
:100BC00025D918F0A8FB724907F1600018F0A3FBC3
:100BD000704907F1700018F09EFB46F22C3307F1C4
:100BE000600207F150010093674807F1700308F0B5
:100BF00033FC07F1700018F04EFB07F1600018F0AD
:100C00004AFB07F1500018F046FB2C463BE018F079
:100C100082FB5F4907F1600018F07DFB214607F178
:100C2000300018F098FB07F1300107F1400018F090
:100C3000DCFB594907F1400018F088FC014607F138
:100C4000700018F0D2FB4FF4FC6307F1600207F16B
:100C5000500100934C4807F1700308F0FDFB07F1C9
:100C6000700018F018FB07F1400018F014FB07F1B2
:100C7000300018F010FB07F1600018F00CFB07F1D2
:100C8000500018F008FB214640F2AF10EFF75AFD74
:100C9000FEF7ABBF012342463146404808F0D0FA88
:100CA000002800F0838040F21D10EFF7B8FD07F137
:100CB000500401283A4907F1700607F16005204603
:100CC00027D118F028FB3749284618F024FB314972
:100CD000304618F020FB46F22C33049328235F2281
:100CE000EB21009303963C23029501942B4808F0D6
:100CF0004FFC304618F0CFFA284618F0CCFA2046C0
:100D000018F0C9FA494640F21D10EFF71BFDFEF737
:100D10006CBF18F000FB2349284618F0FCFA224962
:100D2000304618F0F8FA4FF4FC63049328235F224E
:100D3000EB21009303963C2302950194174808F099
:100D400027FC304618F0A7FA284618F0A4FA2046E7
:100D500018F0A1FA012140F21D10EFF7F3FCFEF7A5
:100D600044BF00BF08BBFF1F851B0300F4BAFF1F71
:100D7000FF87FF1F08C6FF1F7D1903001CBBFF1F55
:100D80008519030030BBFF1F44BBFF1F94190300EC
:100D90009B190300E61803004116030058BBFF1F10
:100DA000A2190300A7190300D41803000123424627
:100DB0003146BE4808F044FA20B1BD4B1B78002BE9
:100DC0003EF413AF012342463146B84808F038FAE2
:100DD00078B1B84B1B8863B1B74B1D221A70002045
:100DE0000923002200218BF80030F3F709FCFEF7FD
:100DF000FCBE012342463146AC4808F021FA70B1EE
:100E0000AC4B1A885AB9AC4B1E211970002009232B
:100E100000218BF80030F3F7F3FBFEF7E6BE012369
:100E200042463146A54808F00BFA00283EF4DDAEF4
:100E3000A34C23780133DBB2092B237084BF00233A
:100E4000237021780020EFF77DFC9E4907F17000A8
:100E500018F061FA21780A22013107F1600018F0D8
:100E60008DFA002307F1600207F17001934808F042
:100E7000ABFA07F1600018F00EFA07F1700018F0F5
:100E80000AFAFEF7B2BE0123424631468B4808F00B
:100E9000D7F9044608B38C4907F1600018F03BFA13
:100EA0008A4907F1700018F036FA07F160014FF433
:100EB000FC6307F17002814808F086FA07F17000C0
:100EC00018F0E9F907F1600018F0E5F901214FF495
:100ED000E270EFF735FCFEF788BE0123424631464B
:100EE0007B4808F0ADF900285BD04FF400714FF457
:100EF000D970EFF735FC4FF440714FF4DA70EFF72B
:100F00002FFC4FF4FC614FF4DB70EFF729FC4FF43A
:100F1000E8614FF4DC70EFF723FC4FF4C2614FF44B
:100F2000DD70EFF71DFC4FF4C0714FF4DE70EFF78A
:100F300017FC40F6FF714FF4DF70EFF711FC40F63D
:100F4000FF714FF4E070EFF70BFC4FF47F614FF44B
:100F5000D870EFF705FC21464FF4E270EFF7F2FB93
:100F600021461220F5F790F85A4907F1600018F071
:100F7000D2F9594907F1700018F0CDF94FF4FC632C
:100F800007F1700207F16001514808F01DFA07F1FE
:100F9000700018F080F907F1600018F07CF9FEF796
:100FA00024BE0123424631464C4808F049F9002846
:100FB0003EF41BAE4A4810F08FFFFBF74BFB49494C
:100FC00007F1700018F0A7F94FF4FC6207F1700107
:100FD000424808F0C3F907F1700018F05CF9FEF719
:100FE00004BE012342463146344808F029F920B3B3
:100FF00023783D4D032B20D83C493D48EFF7C3FAF9
:101000003C4A2978138801311B010233C9B213808D
:1010100029700A22C1F1040107F1700018F0AEF93D
:101020004FF6E07207F17001334808F097F907F1C5
:10103000700018F030F9FEF7D8BD01234246314662
:10104000234808F0FDF818B12378274D032B57D912
:10105000012342463146214808F0F2F8002870D0BA
:101060002378214D032B6CD824492148EFF78BFAC4
:10107000204A2978138801311B010433C9B2138037
:1010800029700A22C1F1040107F1700018F076F905
:101090004FF6E07207F17001174808F05FF907F1A9
:1010A000700018F0F8F8FEF7A0BD00BF6CBBFF1F82
:1010B00064C5FF1FC08EFF1F96C6FF1F80BBFF1FAA
:1010C0008DC7FF1FC2190300211A0300AB1E0300C6
:1010D00094BBFF1F2A1A0300311A0300A8BBFF1F8D
:1010E00034C5FF1F351A03000088FF1F8713030054
:1010F00008C6FF1F58C7FF1F1CBBFF1FD8160300E1
:10110000AA49AB48EFF73FFAAA4A29781388013178
:101110001B010333C9B2138029700A22C1F10401F3
:1011200007F1700018F02AF94FF6E07207F170012C
:10113000A14808F013F907F1700018F0ACF8FEF7B9
:1011400054BD0123424631469C4808F079F820B34B
:1011500023789B4D032B20D89A499548EFF713FA33
:10116000944A2978138801311B010533C9B21380D1
:1011700029700A22C1F1040107F1700018F0FEF88D
:101180004FF6E07207F170018B4808F0E7F807F1BD
:10119000700018F080F8FEF728BD01234246314662
:1011A000894808F04DF820B32378854D032B20D8CB
:1011B00086497F48EFF7E7F97E4A2978138801319D
:1011C0001B010633C9B2138029700A22C1F1040140
:1011D00007F1700018F0D2F84FF6E07207F17001D5
:1011E000754808F0BBF807F1700018F054F8FEF7E6
:1011F000FCBC012342463146754808F021F820B373
:1012000023786F4D032B20D872496948EFF7BBF95B
:10121000684A2978138801311B010733C9B213804A
:1012200029700A22C1F1040107F1700018F0A6F834
:101230004FF6E07207F170015F4808F08FF807F190
:10124000700018F028F8FEF7D0BC01234246314662
:10125000614807F0F5FF20B32378594D032B20D8C0
:101260005E495348EFF78FF9524A297813880131C4
:101270001B010833C9B2138029700A22C1F104018D
:1012800007F1700018F07AF84FF6E07207F170017C
:10129000494808F063F807F1700017F0FCFFFEF70B
:1012A000A4BC0123424631464D4807F0C9FF20B394
:1012B0002378434D032B20D84A493D48EFF763F983
:1012C0003C4A2978138801311B010933C9B21380C4
:1012D00029700A22C1F1040107F1700018F04EF8DC
:1012E0004FF6E07207F17001334808F037F807F164
:1012F000700017F0D0FFFEF778BC0123424631465C
:10130000394807F09DFF18B123782D4D032B2CD9B8
:10131000012342463146354807F092FF00286BD042
:101320002378274D032B67D831492148EFF72BF954
:10133000204A2978138801311B010A33C9B213806E
:1013400029700A22C1F1040107F1700018F016F8A3
:101350004FF6E07207F17001174807F0FFFF07F141
:10136000700017F098FFFEF740BC22491048EFF7D5
:101370000AF9104A2978138801311B01C9B2138078
:1013800029700A22C1F1040107F1700017F0F6FF7D
:101390004FF6E07207F17001074807F0DFFF07F131
:1013A000700017F078FFFEF720BC00BFD4160300D2
:1013B00008C6FF1F58C7FF1F1CBBFF1FBCBBFF1F7A
:1013C0000088FF1FBF1A0300D0BBFF1F9018030047
:1013D000E4BBFF1F5D150300F8BBFF1FF7120300FE
:1013E0000CBCFF1F7313030020BCFF1F34BCFF1F86
:1013F000E814030049150300012342463146BD4865
:1014000007F01EFF20B32378BB4D032B20D8BB4928
:10141000BB48EFF7B8F8BB4A2978138801311B01A4
:101420000B33C9B2138029700A22C1F1040107F1FC
:10143000700017F0A3FF4FF6E07207F17001B24899
:1014400007F08CFF07F1700017F025FFFEF7CDBB0A
:10145000012342463146AD4807F0F2FE20B323781F
:10146000A54D032B20D8AA49A548EFF78CF8A54A2B
:101470002978138801311B010C33C9B213802970FC
:101480000A22C1F1040107F1700017F077FF4FF64F
:10149000E07207F170019C4807F060FF07F17000EF
:1014A00017F0F9FEFEF7A1BB0123424631469948E9
:1014B00007F0C6FE20B323788F4D032B20D8964922
:1014C0008F48EFF760F88F4A2978138801311B01A4
:1014D0000D33C9B2138029700A22C1F1040107F14A
:1014E000700017F04BFF4FF6E07207F1700186486D
:1014F00007F034FF07F1700017F0CDFEFEF775BB63
:10150000012342463146854807F09AFE20B32378EE
:10151000794D032B20D882497948EFF734F8794A7E
:101520002978138801311B010E33C9B21380297049
:101530000A22C1F1040107F1700017F01FFF4FF6F6
:10154000E07207F17001704807F008FF07F17000C2
:1015500017F0A1FEFEF749BB012342463146714810
:1015600007F06EFE20B32378634D032B20D86E491D
:101570006348EFF708F8634A2978138801311B01A3
:101580000F33C9B2138029700A22C1F1040107F197
:10159000700017F0F3FE4FF6E07207F170015A4841
:1015A00007F0DCFE07F1700017F075FEFEF71DBBBB
:1015B0000123424631465D4807F042FE10B12378D0
:1015C000042B1CD0012342463146594807F038FE0F
:1015D00058B3217849B3484B49480139C9B2197009
:1015E00001EB410108234CF2186449008DE8180012
:1015F00027220623323113F0BBFCFEF7F6BA122481
:101600008BF80040F0F792FA4A4B18783D4B00F502
:10161000D8701988EFF7A4F800212046F4F734FDBC
:10162000354B00221A70FEF7E0BA012342463146DC
:10163000414807F005FE00283EF4D7AA0220F3F740
:10164000E5FB3E4B12241C70F0F770FA0021204697
:10165000F4F71AFDFEF7C9BA394911F81230FD2B1B
:101660003CF621AD013301F81230A9E0354AF969A1
:1016700012881D3A8A423CF722AD334A1678082E6A
:101680003CF61DAD963B9BB2192221462A4808F034
:1016900035F8B8F8002078230093963A00231921F2
:1016A000EFF781F8264B03F8160089E0264B1878EF
:1016B00009287CF40DAD254E3378002B3CF408ADA1
:1016C000013B01213370F4F7DFFC31780CE01E4B55
:1016D000187809287CF405AD1C4C2378013323705D
:1016E0000121F4F7D1FC2178194814F08DFFFCF7A3
:1016F0003FBD00BF48BCFF1F0088FF1F75130300DC
:1017000008C6FF1F58C7FF1F1CBBFF1F5CBCFF1F85
:101710006E2F030070BCFF1F462F030084BCFF1F09
:10172000F41D030098BCFF1F1D88030030BBFF1F82
:10173000F4BAFF1FE08EFF1F08BBFF1FFD87FF1FCE
:101740002988FF1F3E88FF1F94C5FF1FFC87FF1FCE
:1017500010C5FF1FAC4AF96912881D3A8A423CF74E
:10176000CCACAA4A1678092E7CF4C7AC963B21462D
:101770009BB21922A648A74C07F0C0FFB8F800207A
:10178000FF23009319210023963AEFF70CF801216B
:1017900020703046A5E79D4B1B780A2B7CF4B6AC35
:1017A0009D4A1378002B3CF4B1AC013B07E0974B0A
:1017B0001B780A2B7CF4B3AC974A1378013313706F
:1017C00001210920F4F760FCFCF7D2BC8E4AF969CC
:1017D00012881D3A8A423CF7ACAC8C4A12780A2A2D
:1017E0007CF4A7AC963B9BB219222146884807F0AF
:1017F00085FF328878230093963A00231921EEF76B
:10180000D2FF854B1870DBE70123FCF7A9BC01234D
:101810002A462146814807F013FD18B17B4B1B78FF
:101820000B2B31D0BAF1190F22DD7D4E3388A3F195
:101830007D0292451CDA744AF96912881D3A8A427F
:1018400016DC724A12780B2A12D1963B9BB21922EF
:1018500021466F4807F052FF328878230093963A6A
:1018600000231921EEF79FFF6E4B1870FCF779BC2F
:1018700001232A4621466C4807F0E2FC80B3634B03
:101880001B780C2B2CD109E0664A1378602B02D808
:101890000233FCF765BC6223FCF762BC4FF4D470E2
:1018A000EEF7BDFF012807D100214FF4D470EEF709
:1018B00049FF4FF4FC6405E001214FF4D470EEF7CA
:1018C00041FF1F24594907F1700017F024FD5648C5
:1018D000224607F1700107F041FD07F1700045E075
:1018E00001232A462146524807F0AAFC18B1474B6B
:1018F0001B780C2B3ED001232A4621464D4807F089
:101900009FFC00286ED0414B1B780C2B6AD14A4CAF
:101910002378082B75D1052323702178474814F0CC
:101920002CFD217807F1500017F015FD07F150014B
:1019300007F1600017F059FD414907F1600017F009
:1019400005FE014607F1700017F04FFD002207F178
:101950007001384807F002FD07F1700017F09BFC9A
:1019600007F1600017F097FC07F1500017F093FCA7
:10197000FCF7FEBB334C23780133DBB2062B23701C
:1019800001D9002323702078F0F79CF80320F1F7A9
:1019900047FC2D4907F1600017F0BDFC217807F1E5
:1019A000500017F0D8FC07F1500107F1600017F064
:1019B000C5FD014607F1700017F017FD002207F181
:1019C00070011B4807F0CAFC07F1700017F063FCB8
:1019D00007F1500017F05FFC07F1600017F05BFCA7
:1019E000FCF7C6BB01232A4621460F4807F028FC16
:1019F00000283CF4BDAB054C2078082826D9FCF71C
:101A0000B7BB082388E700BF3E88FF1F94C5FF1FB0
:101A100008BBFF1FFC87FF1F3B88FF1FF4BAFF1F97
:101A20000488FF1F368EFF1F1CBBFF1F2D160300EF
:101A300030BBFF1F44BBFF1F23C4FF1F10C5FF1F88
:101A40003D160300E88EFF1F37160300B74942001A
:101A50008E180D4673780133DBB2092B737001D9F0
:101A6000002373702A4400F267105178B04EEEF7ED
:101A700069FEB04907F1700017F04DFC2378AE48BD
:101A800005EB430307F170015B7836F8132007F08C
:101A900065FC07F1700017F0FEFB2378A74859009A
:101AA0005A18294403EB82024B7836F8133001931D
:101AB000092300932C320A23732113F059FAFCF7FF
:101AC00057BB0123424631469D4807F0B9FB48B158
:101AD0009C4B1B78082B05D001210820F4F7D4FA81
:101AE000FEF783B8012342463146974807F0A8FB2A
:101AF00030B90123424631468F4807F0A1FB20B19F
:101B0000904B1A78082A994616D00123424631464E
:101B10008B4807F095FB40B90123424631468B487C
:101B200007F08EFB00283EF460A8864B1A78082A3E
:101B300099467EF45AA850E0854D864C2B78864E07
:101B4000A82202FB034393F891200AB9FF2203E085
:101B5000FF2A08BF3278013A83F89120012107203B
:101B6000F4F792FA4FF6FF71744811F07EF899F885
:101B70000030724803EB430203EB82024FF000088F
:101B800009232D328DE8080112B25A23642113F083
:101B9000EFF999F80030694803EB430203EB820246
:101BA0002D32434612B2672112F032FB2B78A82265
:101BB00002FB034407F17000337894F89110424619
:101BC00008F002FA07F170015C4817F021FA07F1FA
:101BD000700017F060FBFEF708B85D4E5D4C33787F
:101BE0005D4DA82101FB03412A7891F89130013A1B
:101BF000934201D1FF2303E0FF2B0CBF00230133ED
:101C000081F8913007200121F4F73EFA4FF6FF7179
